:020000040800F2
:1000000000500020D143010895D200081FA6000827
:1000100093D2000891D200088FD20008000000009F
:100020000000000000000000000000008DD2000869
:100030008BD200080000000089D20008090D0108D9
:100040006D4401086D4401086D4401086D440108C8
:100050006D4401086D44010877F2000881F2000840
:100060007FF200087DF200087BF2000801550008CD
:10007000F1540008E1540008D1540008C1540008AC
:10008000AD5400089B5400086D4401086D440108FC
:1000900059D300086D4401086D44010879F2000845
:1000A0006D44010865A300086D44010855A30008CC
:1000B00045A3000835A3000825A30008F958000847
:1000C000FD580008F1580008F55800086D44010873
:1000D0006D4401081D5400086D44010813540008C4
:1000E00075F200086D440108812C01080000000031
:1000F0000000000000000000000000000000000000
:0C01000000000000000000005FF808F1A3
:100110002DE9F04FB0F908300546D8B2522885B025
:100120000C4617460B8100F0328700F238813628E2
:1001300000F0D18600F2D180222800F00B8563D830
:10014000032800F0078347D8012800F0E88202283E
:1001500000F0F482F52895E8480041F00C809E42BA
:100160000FBFFF23591C296013F8021BAF4A16BFAB
:100170002B6082F82F3082F82F1092F82F30FF2B4F
:100180004FF0000340F0F187A94A1846904699586D
:1001900001B108801433F02BF9D100264FF0140977
:1001A000A44BA54D31463022A4481E702E7018F085
:1001B00033FF8DF80F60A14E9DF80F300B2B40F2EE
:1001C000AD8723682A78591C21601A70002F00F02F
:1001D000BF829B4B3B60BBE2052800F0FA82C0F077
:1001E000E9820A28B6D1974813F004F9002396490A
:1001F000984240F3AD825A1892F8D45422680133E1
:10020000561C26601570F3E72A2800F0F8850DD8F3
:10021000262800F09C85282800F0DA85242899D12A
:10022000894B204699680AF012FF91E2322800F0CB
:100230001286342800F0B3842C288BD1824D0B68B1
:1002400095F85C22591C21601A70B5F86E12204690
:100250000AF011FFB5F86A1220460AF00CFFB5F853
:100260006C1220460AF007FF236895F86522591C96
:1002700021601A70B5F8781220460AF0FCFEB5F835
:100280007A1220460AF0F7FE236895F87022591C6E
:1002900021601A70236895F87222591C21601A7027
:1002A000B5F8761220460AF0E6FE236895F85F223C
:1002B000591C21601A70D5F8601220460AF0C7FE5A
:1002C000236895F86422591C21601A70236895F8F8
:1002D0007322591C21601A703AE2442800F01787F3
:1002E00025D83B2800F02C840AD8382800F0408517
:1002F0003A287FF42FAF002120460AF0A8FE27E21B
:10030000402800F0B085422800F0BA853D287FF4EF
:1003100021AF4D4B226893F8B212501C206011702F
:1003200093F8B1222368591C21601A7010E24B28FF
:1003300000F06D850ED8462800F0DF85C0F03586C8
:1003400049287FF407AF414B2046B3F848100AF024
:1003500092FEFDE14F2800F00386502800F0E7856B
:100360004D287FF4F7AE0026394D3A4F3B780235E1
:100370009E4280F2ED81236815F8022C591C216001
:100380001A7015F8011C204601EB810101EB810177
:1003900001F2EE2189B20AF06EFE0136E6E76F281F
:1003A00000F0928300F2F280652800F0478200F2AC
:1003B000B7805C2800F05A8650D8542800F0EE85AB
:1003C0005A287FF4C7AE204D0B6895F8FF21002A0C
:1003D00000F040865A1C0A6008221A700B685A1CEA
:1003E0000A6001221A70236895F8D520591C2160F3
:1003F0001A70236895F8D420591C21601A70B5F83A
:10040000D21020460AF037FE1349D5F8D80013F071
:10041000A9FD16F02BFB81B220460AF02CFE2368C2
:1004200095F80322591C21601A7091E1AC05002057
:10043000441C0020121C0020111C0020803A0020C7
:100440002DB40008EC34002018300020F80F0020F4
:1004500094320020281700200000C842602800F0D5
:100460004186642800F0D4815E287FF473AEC04DCD
:10047000002120460AF0FFFD002120460AF0FBFD86
:100480002B682046598D0AF0F6FD23685A1C22601D
:1004900000221A702B6893F831102368581C2060D2
:1004A00019702B6893F840102368581C206019704D
:1004B0002B6893F841102368581C2060197023683A
:1004C000591C21601A702368591C21601A70236816
:1004D000591C21601A702B68A649986C13F042FDD4
:1004E00016F0C4FA81B220460AF0C5FD2B68A14976
:1004F000586C13F037FD16F0B9FA81B220460AF0B5
:10050000BAFD2B6893F833202368591C21601A70B8
:100510002B6893F834202368591C21601A7017E166
:10052000692800F0EF8016D8672800F0F18140F2CA
:10053000C18100251426904FDFF8748206FB0573F5
:10054000197B002940F05C82204601350AF093FDBA
:10055000082DF3D1FCE06D2800F0558200F25C829A
:100560006C287FF4F7AD854D204629880AF083FD7D
:10057000698820460AF07FFD0A23B5F90410204659
:1005800091FBF3F189B20AF076FDE1E07C2800F0FE
:10059000208538D8742800F02D8321D8722800F0E7
:1005A000598300F2B08370287FF4D4AD00227049E3
:1005B0000B68985C23685D1C256018700B681344F9
:1005C000987A23685D1C256018700B681344187DA9
:1005D000236801325D1C0A2A25601870E8D1B7E053
:1005E000772874D0782800F0A18175287FF4B2AD07
:1005F000634A12F8013F002B00F0AA802168481CD2
:1006000020600B70F5E7A02800F091834AD87E287F
:1006100000F00B85C0F0EF8496287FF49BAD594B1A
:100620002046B3F858100AF026FD574B204619888B
:1006300089B20AF020FD554B20461968C1F3C0036A
:10064000C1F380029B0043EA4203C1F3400213431B
:10065000C1F3401243EAC20301F0100119430AF04A
:100660000AFD12F003FE014620460AF0F0FC484B5A
:10067000204693F81C242368591C21601A70454BAE
:1006800019886429A8BF64210AF0F5FC23685A1C64
:10069000226002221A70404B1A782368591C21608C
:1006A0001A7055E0F12800F07A81FE2800F03483BA
:1006B000F0287FF44FAD364D2046B5F822120AF0EF
:1006C000DAFCB5F8201220460AF0D5FC40E0002103
:1006D0004FF00C0C314D324805F1100700F1300E8F
:1006E00095F82E30994233DA0022CE5D0CFB02F3EE
:1006F00013F80E80B04501F0158301321F2AF5D1A1
:100700000131EDE70025274E274F33789D421FDA50
:1007100037F8151020460AF0AEFC0135F5E70B68F6
:100720005A1C0A6000221A700B685A1C0A60187062
:100730000B685A1C0A601F221A7006E200231B4D28
:100740002268595D0133501C042B20601170F7D1D1
:100750000120FAE10B685A1C0A60187001200B682E
:100760005A1C0A6018700B681A180A600622E3E720
:10077000881E002000002041441C00202A26002062
:100780006F91010818000020201C0020AC250020DB
:1007900018300020EC0F0020221C0020AC050020A7
:1007A0007091010828170020181800200BB10108CB
:1007B000642500200023B34D2268595D0133501C8D
:1007C000042B20601170F7D1002120460AF053FC61
:1007D000BEE70023AC4D2268595D0133501C0B2B42
:1007E00020601170F7D10023A84D2268595D0133B4
:1007F000501C082B20601170F7D10023A44D2268F3
:10080000595D0133501C072B20601170F7D19FE711
:100810000B6820465A1C0A60E7221A709D4B93F819
:10082000B3220B68591C21601A70236804215A1CDA
:10083000226000221A700AF00AFC89E7964B2046D3
:10084000B3F858100AF017FC944B2046198889B267
:100850000AF011FC924B20461968C1F3C003C1F3A2
:1008600080029B0043EA4203C1F340021343C1F3F9
:10087000401243EAC20301F0100119430AF0FBFBE6
:1008800012F0F4FC014620460AF0E1FB814B2046C1
:1008900093F81C242368591C21601A70814B198815
:1008A0006429A8BF64210AF0E6FB002120460AF073
:1008B000E2FB4DE77C4E00253289B2F5007F94BF04
:1008C000012704277319196B204691FBF7F10435B2
:1008D00089B20AF0D0FB0C2DF4D10025734EAB1970
:1008E000B169D86C13F0F2FB16F0C0F8043581B290
:1008F00020460AF0C0FB0C2DF1D100256C4EAB193F
:100900009989204604350AF0B6FB0C2DF7D11FE774
:10091000684B0A6803F1100153F8040B8B4242F84C
:10092000040BF9D123681033236011E7594D0026D9
:100930002F464FF00E08B5F8721120460AF09BFBC7
:10094000B5F8741120460AF096FBB5F876112046EA
:100950000AF091FB236895F87821591C21601A70E0
:10096000236895F87921591C21601A70236895F83D
:100970007A21591C21601A70236895F87B21591C33
:1009800021601A7008FB06732046D3F87C110136EB
:100990000AF05DFB082E05F10E05CCD1D8E63D4BE3
:1009A00003F17001226893F80201551C2560107054
:1009B000226893F80301551C25601070226893F893
:1009C0000401551C25601070226893F80501551C20
:1009D00025601070226893F80601551C2560107080
:1009E000226893F80701551C25601070226893F85F
:1009F00008010733551C994225601070D2D1A7E633
:100A000038F81510A0E5204600210AF020FB00214F
:100A100020460AF030FB9BE6274B4FF6FF751B88FC
:100A20000A68FF2BA8BFFF23511C21601370234BC2
:100A300020461968A942A8BF294621EAE17189B276
:100A40000AF019FB1E4B204619880AF014FB114BC3
:100A500093F845221B4B62B10A211B68204659437B
:100A6000A942A8BF294621EAE17189B20AF003FB35
:100A70006EE61968204601F30F0189B20AF0FBFA0D
:100A800066E600BF10B1010815B1010821B10108E7
:100A90002AB101081830002018000020201C002076
:100AA000AC250020EC0F0020B0250020F80F00201E
:100AB000F4250020AC050020F8140020F4140020D8
:100AC0004A0E0020600C0020B94D2B681A780B6884
:100AD000591C21601A702B689A782368591C216070
:100AE0001A7000232A681A44517922680133501C75
:100AF000032B20601170F5D12B6820461A7A2368E9
:100B0000591C21601A702B68DA782368591C2160FF
:100B10001A702B681A792368591C21601A702B6887
:100B200059890AF0A8FA2B685A7A2368591C21605F
:100B30001A702B685A782368591C21601A7007E6CE
:100B400001200B685A1C0A601870608140B205B021
:100B5000BDE8F08F0C27974A974E02F1500192F8AA
:100B60001D34043207FB036393F8380023685D1CCF
:100B700025601870236892F81A045D1C25601870AF
:100B8000236892F81B045D1C25601870236892F896
:100B90001C045D1C914225601870E0D1D8E5854B9E
:100BA00003F15A01226893F87204551C25601070F5
:100BB000226893F86D04551C25601070226893F824
:100BC0006E04551C25601070226893F86F04551C44
:100BD00025601070226893F87004551C2560107011
:100BE000226893F871040633551C994225601070F1
:100BF000D8D1ADE501264FF00C0B704FDFF8B8816E
:100C000007F1100908F1300A002597F82E309D42AF
:100C100004DB002E3FF49CAD0026F5E7002215F81A
:100C200009100BFB02F313F80A00884201F06D80F3
:100C300001321F2AF5D10135E7E7216813F801EBEE
:100C400001F1010CC4F800C081F800E0991A81425A
:100C5000F3DBF0E7574D2046B5F86A120AF00BFABD
:100C6000B5F8CC1020460AF006FAB5F8CE102046AA
:100C70000AF001FAB5F8D01020460AF0FCF9B5F8F0
:100C8000B81220460AF0F7F92268531C23600023AB
:100C900013702268511C216013702268511C21605E
:100CA0001370226895F84512501C2060117022685C
:100CB00095F86712501C2060117022682046511C64
:100CC000216013700A23B5F90C1291FBF3F189B27C
:100CD0000AF0D1F9236895F83822591C21601A705E
:100CE000236895F83C22591C21601A70236895F8F6
:100CF0003B22591C21601A70236895F83D22591C2B
:100D000021601A7024E501232268511C21601370B0
:100D10000133092BF8D11BE50025294E36F81510B3
:100D2000204601350AF0A7F9042DF7D110E5254B2F
:100D3000204619680AF08BF9234B204619680AF0FF
:100D400086F9224B204619680AF081F900E5194D11
:100D50002046B5F8E4110AF08EF9B5F8E8112046FE
:100D60000AF089F9B5F8EC1120460AF084F9EFE4AD
:100D7000104B226893F83812501C206011702268C2
:100D800093F83C12501C20601170226893F83B12BB
:100D9000501C20601170226893F83D12501C206096
:100DA000117093F83F222368591C21601A70CFE418
:100DB000380E00201830002070910108AC0500208A
:100DC000CE1E0020E8F7FF1FECF7FF1FF0F7FF1F14
:100DD000BF4D2046B5F840120AF04DF9B5F8421261
:100DE00020460AF048F9236895F84422591C2160EE
:100DF0001A70B5F8461220460AF03DF9A8E4B44B43
:100E000093F8B3220B68591C21601A70A0E4B04D0E
:100E10000B6895F8B622591C21601A70236895F862
:100E2000B722591C21601A70B5F8B81220460AF092
:100E300022F9236895F8BA22591C21601A70B5F876
:100E4000BC1220460AF017F9236895F8BE22591CF7
:100E500021601A707CE49E4B93F867220B68591C42
:100E600021601A7074E40023994D5A1992F85412B3
:100E700022680133501C082B20601170F5D167E403
:100E8000934D0B6895F8B322591C21601A70A9681C
:100E900020460AF0DCF8236895F85C22591C216092
:100EA0001A70B5F8E41120460AF0E5F8B5F8E81133
:100EB00020460AF0E0F8B5F8EC1120460AF0DBF81D
:100EC000B5F8401220460AF0D6F8B5F8421220468E
:100ED0000AF0D1F83CE47E4D7E4F05F12806002350
:100EE00095F9DA22D957914200F025870C333C2B33
:100EF000F8D10835B542F2D12AE40DF099FC00286A
:100F00000CBF022203222368734D591C21601A7002
:100F1000298820460AF09BF8E96820460AF097F8ED
:100F20000DF066FC014620460AF091F810E401201D
:100F30000B685A1C0A601870654B226893F8C91434
:100F4000151825601170226893F8C71415182560CC
:100F5000117093F8C824236819182160FFF7ECBBBF
:100F600000250B6820465A1C0A601D700B685A1C2D
:100F70000A601D700B685A1C0A6029461D700AF031
:100F800066F8294620460AF062F8FFF7E1BB0B68D5
:100F90005A1C0A6000221A70FFF7DABB0B685A1C51
:100FA0000A6000221A70FFF7D3BB00234B4D226862
:100FB000595D0133501C0B2B20601170F7D1204676
:100FC00000210AF044F8002120460AF040F8FFF71B
:100FD000BFBB3F4D2046B5F8E8100AF04CF8B5F815
:100FE000EA1020460AF047F8B5F8EC1020460AF05F
:100FF00042F8FFF7ADBB364B226893F84C12501CF9
:1010000020601170226893F84D12501C20601170FE
:10101000226893F84E12501C20601170B3F8EE1045
:1010200020460AF028F8FFF793BB294B226893F873
:10103000FC11501C20601170226893F81812501C8B
:101040002060117093F80E222368591C21601A70D9
:10105000FFF77EBB95F8FE21591C21601A702368AA
:1010600095F8F821591C2160FFF7BCB9184E0B68A0
:1010700096F801221A4D591C21601A702B682046DF
:10108000198C09F0F8FF2B682046598C09F0F3FF02
:10109000B6F80412204609F0EEFFB6F80612204614
:1010A00009F0E9FF2B682046998C09F0E4FF2B68D2
:1010B0002046D98C09F0DFFFB6F80812204609F067
:1010C000DAFFB6F80A12204609F0D5FFFFF740BB59
:1010D00018300020683500207802002015B1010882
:1010E000881E0020B74B226893F81912501C20600C
:1010F0001170226893F82412501C2060117093F82C
:101100000F222368591C21601A70FFF721BB002AA7
:101110003FF41EABAC4B1360FFF71ABB9DF80F30CA
:1011200009FB03831B7BC3B19DF80F3009FB0383CD
:101130001B6993B19DF80F304A2109FB038318699D
:101140002B7846F823000EF04DF82B7856F8230044
:101150000EF078F82B7801332B709DF80F300133A7
:10116000DBB28DF80F30FFF727B82268511C2160E1
:101170001370FFF7EDBA4728A6EB030648D12846BF
:1011800009F03FFF052E07463FD9284609F04FFFDB
:101190000026054694E80C009B1A103B8B4AAB4294
:1011A000A846B8BF9DB2D3683946DB1B9D42204696
:1011B00088BF9DB2914609F04AFF3EB929462046B4
:1011C00009F059FF23685A1C22601E70D9F80C30B0
:1011D0007A199A42D4F800A088BFDD1B0DF006FCF6
:1011E0002A46514638460DF03FFC236803442360ED
:1011F000002E3FF4ADAA002280457FF7A9AA2368FC
:101200000130591C21601A70F6E701268025C1E7DC
:101210005B2800F05C8300F2DD80372800F01F853A
:1012200062D8292800F02A8420D8232800F0F781EA
:1012300005D80B2800F052854FF0FF3085E42528B3
:1012400000F011842728F7D1284609F0F0FE5D4E02
:10125000C6F8E401284609F0EAFEC6F8E801284687
:1012600009F0E5FEC6F8EC01FFF772BA2D2800F090
:101270001D8409D82B28DFD15A1C2A601A78514BBB
:1012800083F8B322FFF764BA332800F0B18435281D
:10129000D2D15A1C2A6019780E29CDD89A1C2A60FE
:1012A0005A78032AC8D80626464806FB010181F869
:1012B0007224DA1C2A609A7881F86D241A1D2A603B
:1012C000DA7881F86E245A1D2A601A7981F86F2421
:1012D0009A192A605A7981F87024DA1D2A609B795C
:1012E00081F87134FFF734BA432800F089843BD881
:1012F0003C283FF42DAA23D839289DD119465A1CE1
:101300002A6011F8020B2F4A042E82F83802296055
:10131000597882F83C1203F103012960997882F828
:101320003B1203F104012960D97882F83D127FF65F
:101330000FAA591D29601B7982F83F32FFF708BABE
:101340003E2800F0438141287FF476AF00231D48FA
:101350002A68511C296011781A180133082B82F869
:101360005412F5D1FFF7F4B94C2800F0F9830AD8EC
:10137000482800F06D834A287FF45EAF284609F0C4
:1013800056FEFFF7E5B94E2800F00E8451287FF491
:1013900053AF0F4A92F83020012A3FF6D9A91946D7
:1013A0005A1C2A6011F8020B064A82F8C904296007
:1013B000597882F8C714D91C29609B7882F8C83400
:1013C000FFF7C6B9183000202D320108780200203E
:1013D000AC050020D22800F0CD807ED8CA2800F0CD
:1013E000038152D85F2800F0AC8247D85D287FF493
:1013F00023AF5A1C2A601B78BB4FDFF8F8822846BF
:10140000D7F8009088F8013209F011FEA9F8200001
:101410002846D7F8009009F00AFE052EA9F8220008
:1014200023D9284609F003FEA8F80402284609F04B
:10143000FEFDA8F806022846D7F8009009F0F7FD4F
:10144000A9F824002846D7F8009009F0F0FD0D2EE9
:10145000A9F8260009D9284609F0E9FDA8F80802EC
:10146000284609F0E4FDA8F80A0208F0B1FB06F0EE
:10147000E5F938680EF064FCFFF76AB9612800F0FE
:10148000B982C8283FF464A9D6E6CE2800F0C58208
:1014900010D8CC2800F0DF80CD287FF4CDAE934B60
:1014A0001B7859073FF554A94FF4C872904B1A8026
:1014B000FFF74EB9CF2800F02381D0287FF4BCAECF
:1014C0008A4B1B7858073FF543A908F00DFF09F038
:1014D000C3FB09F021FAFFF73BB9DA2800F0D98104
:1014E0001BD8D42800F06A815ED3D62800F05A8138
:1014F000D9287FF4A1AE284609F099FD7D4EA6F8C3
:10150000E800284609F093FDA6F8EA00284609F00D
:101510008EFDA6F8EC00FFF71BB9EF2849D018D8CC
:10152000DB2800F0CE81DC287FF486AE19465A1CF9
:101530002A6011F8020B6F4A82F8FC012960597881
:1015400082F81812D91C29609B7882F80E32FFF7B6
:10155000FFB8F22800F06B81FA287FF46DAE634B80
:101560001B785B073FF568AE09F076FB09F0D4F90C
:10157000FFF7EEB85A1C2A60187806060BD45B4BAE
:101580001B785D073FF5E4A8022828BF002008F07B
:1015900001FBFFF7DDB800F07F00032828BF002023
:1015A00008F0DAFAFFF7D4B8284609F040FDFFF753
:1015B000CFB8284609F03BFD4E4EA6F82202284639
:1015C00009F035FDA6F82002FFF7C2B85A1C2A60C0
:1015D0001A46484912F8020B81F8B2022A605B7879
:1015E00081F8B132FFF7B4B83F4B1868431E00F1E1
:1015F00009062A68511C2960114611F8027B03F87C
:10160000017F296051789E42997202F1030129609D
:1016100092781A75EDD10EF001FBFFF799B85A1CBC
:101620002A601A78132A3FF607AE00204FF00C0C00
:10163000991C296030495F7801F1300E0CFB00F6EF
:101640000EEB060898F80880B84500F0A383013037
:101650001F28F3D1F0E5092E7FF6EEAD27485A1C7E
:1016600007682A601A4612F8021B804639702A6001
:101670005B78791DBB700023022B14BF4FF0640E02
:101680004FF0FF0E28680133421C2A600278724531
:10169000A8BF7246032B01F8012BEDD1831C2B60F0
:1016A0004378642B28BF64233B72C31C2B60837870
:1016B000FB70031D2B60C37828463B7109F0B7FC13
:1016C0000A2E78810CD02B68D8F80020591C29608C
:1016D00019780B2E51721FBF991C29605B785370CB
:1016E00011F056FEFFF734B8881E0020282600208F
:1016F000780B00201830002070910108380E00206F
:10170000284609F094FCCB4EA6F86A02284609F058
:101710008EFCA6F8CC00284609F089FCA6F8CE007D
:10172000284609F084FCA6F8D000284609F07FFC82
:10173000A6F8B802284609F085FC284609F082FC84
:10174000284609F07FFC2B6828465A1C2A601A4656
:1017500012F8021B86F845122A605B7886F8673219
:1017600009F070FC284609F062FC2B6800EB800051
:101770005A1C4000A6F80C022A601A4612F8021BF6
:1017800086F838122A605A7886F83C22DA1C2A60D9
:101790009A7886F83B221A1D2A60DB7886F83D325B
:1017A000FEF7D6BF0026A44F284609F040FC27F8D4
:1017B00016000136082EF7D1FEF7CABF0F2E7FF4B0
:1017C0003BAD5A1C2A601E78072E3FF635AD2846E1
:1017D00009F02DFC0E22974B02FB0636A6F872018B
:1017E000284609F024FCA6F87401284609F01FFCDD
:1017F0002B68A6F876015A1C2A601A4612F8021BBA
:10180000284686F878112A605A7886F87921DA1CF9
:101810002A609A7886F87A211A1D2A60DB7886F881
:101820007B3109F0EEFBC6F87C01FEF791BF5A1C34
:101830002A601A780F2A3FF6FFAC991C29607D4870
:101840005978C2EBC202024482F80211D91C296005
:10185000997882F80311191D2960D97882F804114A
:10186000591D2960197982F80511991D2960597946
:1018700082F80611D91D2960997982F8071103F1C0
:1018800008012960DB7982F808310EF089F9FEF74A
:101890005FBF5A1C2A601A46664E12F8021B284681
:1018A00086F84C122A605A7886F84D22DA1C2A6093
:1018B0009B7886F84E3209F0BAFBA6F8EE00FEF7E8
:1018C00047BF5E4B186808F02DFAFEF741BF5A1C5F
:1018D0002A601A46574F12F8021B284687F8FE1155
:1018E0002A605A7887F8F821DA1C2A609A7887F8F3
:1018F000D5201A1D2A60DB78042BA8BF042387F8A3
:10190000D43009F094FB072EA7F8D20009D9284655
:1019100009F08DFB12F0D2FA494912F023FBC7F807
:10192000D8002B686A689A4207D05A1C2A601B7834
:10193000003318BF012387F8033208F049F9FEF796
:1019400007BF284609F073FB3C4F284609F06FFBA0
:101950002846D7F8008009F06AFBA8F82A00284634
:1019600009F070FB2B683A68591C2960194611F878
:10197000020B82F8310029605978284682F840101D
:10198000D91C29609B7882F8413009F05BFB28461E
:1019900009F058FB284609F055FB2846D7F8008087
:1019A00009F045FB12F08AFA264912F0DBFAC8F872
:1019B00048002846D7F8008009F039FB12F07EFA7B
:1019C000204912F0CFFA112EC8F844003B460CD93A
:1019D0002A683868511C2960114611F8026B80F89A
:1019E00033602960527880F8342018680EF016F9B8
:1019F000FEF7AEBE19465A1C2A6011F8020B0D4ABA
:101A000082F819022960597882F82412D91C2960B9
:101A10009B7882F80F32FEF79BBE0B4B1B785A0760
:101A20003EF596AE094A137843F004031370FEF7AF
:101A30008FBE00BF18300020241C0020881E00200C
:101A40000AD7233CCDCCCC3D2826002034260020CC
:101A50000DF03CF80023C94A1370C94A1370C94AF3
:101A60001360FEF775BE0023C74E2846B36009F029
:101A7000C8FAB3681843B060FEF76ABE284609F09A
:101A8000D6FAC14EA6F84002284609F0D0FA2B68D3
:101A9000A6F842025A1C2A601B78284686F844326F
:101AA00009F0C5FAA6F84602FEF752BE5A1C2A6093
:101AB0001B78B54F284687F85C3209F0B8FAA7F8CA
:101AC0006E02284609F0B3FAA7F86A02284609F020
:101AD000AEFA2B68A7F86C025A1C2A601B78082EF5
:101AE00087F865327EF634AE284609F0A0FAA7F8EA
:101AF0007802284609F09BFA0C2EA7F87A027EF6A7
:101B000027AE2B6828465A1C2A601A4612F8021B78
:101B100087F870122A605B7887F8723209F087FACA
:101B2000102EA7F876027EF613AE2B6828465A1CB4
:101B30002A601B7887F85F3209F063FA2B68C7F8D0
:101B400060025A1C2A601A78162E87F864227EF6E4
:101B5000FFAD9A1C2A605B7887F87332FEF7F8BDF8
:101B60005A1C2A601A46884E12F8021B284686F82C
:101B7000B6122A605B7886F8B73209F058FA2B68FB
:101B8000A6F8B8025A1C2A601B78284686F8BA3292
:101B900009F04DFA2B68A6F8BC025A1C2A601B7883
:101BA00086F8BE32FEF7D4BD5A1C2A601E78112E6C
:101BB0003FF642AB9A1C2A605A7806F59E73724E25
:101BC000284606EB4306327109F031FA40F6CA03A3
:101BD0009842A8BF184640F2EE239842B8BF184674
:101BE0001923A0F2EE2090FBF3F07071FEF7B0BD68
:101BF0005A1C2A601A78644B83F86722FEF7A8BD46
:101C00005A1C2A60604E1B78284686F8B33200239F
:101C1000B36009F0F6F9B36818432B68B0605A1C3A
:101C20002A601B78284686F85C3209F000FAC6F86C
:101C3000E401284609F0FBF9C6F8E801284609F056
:101C4000F6F9C6F8EC01284609F0F1F9A6F84002C9
:101C5000284609F0ECF9A6F84202FEF779BD072202
:101C6000B6FBF2F2C2EBC203F61A7FF4E5AADFF884
:101C700020915FFA82F8F3B243453EF469AD2968DA
:101C80004B1C2B6091F900000021D9F8003003EBC8
:101C9000C10797F90220824204D001310529F6D10B
:101CA000FFF7CABA0136002F3FF4C6AAB87028461B
:101CB00009F0BDF92A6838801146531C2B6011F8D1
:101CC000023BFB70296053783B71D31C2B609378E7
:101CD000BB71131D2B60D3787B71CCE700211122DF
:101CE0002A4817F099F9102E4FF0000328BF10264C
:101CF0002549B342BEF42CAD2A68501C28601078E8
:101D00005A1882F8D4040133F3E743445A6B10465F
:101D1000019211F06FFB002E7EF48DAF019A1346F5
:101D2000FEF794BF034493F8382023685E1C2660B6
:101D30001A70FEF7E5BC23682046591C21601A7012
:101D4000B5F8D81209F097F9236895F8DB22591CE9
:101D500021601A70236895F8DC22591C21601A70E2
:101D6000236895F8DE22591C21601A70236895F8C3
:101D7000DD22591C21601A70FFF7BBB86C1D0020D2
:101D80006D1D0020701D002018300020EC34002054
:101D90006435002002F5837031440F4A91F8301009
:101DA00002EB80025171D91C296099780020917151
:101DB000191D2960D978D171591D29601B791372B9
:101DC000064B1A68064B1A600FF05DFA054B80F05F
:101DD00001001870FEF7BCBC18300020881E0020DF
:101DE000B40B00200C0000202DE9F04F904AA5B064
:101DF00013780690012B904607D18E498E4A0968C8
:101E0000496A11808D49098851808D4C94F800A051
:101E1000BAF1000F00F02E83072B02D108F0A2FBCD
:101E20000890884B1A68994612F4806F04D086484F
:101E300083680BB185499847854B864E1B78C3B1A3
:101E4000854BB3F90620B6F86C329A4211DC96F84D
:101E5000B332012B01D0192B02D196F8FC2042B9E4
:101E60000E2B06D0082B04D000227C4B9A80002336
:101E7000E36096F836526DB3794B1B889F0729D0E3
:101E8000784B79491F6A384612F014FA002840F05E
:101E9000C580384614F062FE216912F063F814F030
:101EA000E5FDB0F5617FA8BF4FF4617012F006F850
:101EB0006E4912F057F811F07CF80746284611F0E9
:101EC000FDFF394612F04EF814F0D0FD634BDA886E
:101ED0001044D880664B96F871721B780237FFB2B7
:101EE000002B53D0634A4FF07E51D2F8F45044F6A1
:101EF00020629542A8BF1546B5F57A7FB8BF4FF46A
:101F00007A755D4AADB2D2F800B0A582DBF83C200C
:101F100007931046059212F0E1F9079B002835D08F
:101F20004FF47A71B5FBF1F5642191FBF5F5142DB1
:101F3000A8BF1425D9F80010A06911F4805F4749A3
:101F400018BFBBF838E000F1010CB1F9061004EB42
:101F5000400014BF4FEA5E0EBBF938E0AC45818308
:101F6000A8BF0020C4F818C0A8BFA061A069059A46
:101F700004EB4000808B091A09B20029B8BF49421E
:101F80007145D8BF4FF07E523C490A6096F87022E6
:101F9000002A45D1324A1288002A46D10025284B12
:101FA000A3F84650324B1B78002B40F0AD80344BE9
:101FB0001878002840F05182224D2B681A0340F116
:101FC0004C82304C2378033B052B16D8214B1C4EFA
:101FD00093F8C934002B00F00F82012B00F010821F
:101FE000F26F96F880301344B3F5807FA8BF4FF4AA
:101FF00080738342D4BFF367F0672378023B092BD9
:1020000000F21C82DFE813F001020D02B5021A0291
:102010001A02F8020B03A705C405D405002055E7F2
:10202000022A33D0032A00F0E880174A528831E0B0
:10203000CC1E002008150020CE1E0020EC0F002032
:102040000C07002000170020F80F00204E0C002085
:102050000C0000201830002018180020500C002020
:10206000C63A0020882500208FC2753CD06D393AD1
:10207000BA0B002018000020881E00200400002059
:10208000681D0020DC05002028170020A28A02F528
:102090007A7292B2002B00F0CB80724B196898F8DC
:1020A0000030B2FBF1F1481C00B2092BA4F8440047
:1020B00006D16D4D6D4B2E886D881E805D80DA8057
:1020C00000236B4DB4F94680DFF89C9105F1080EB2
:1020D000BB42C0F29A80674BA3F84610654AB2F93A
:1020E000460000287FF75AAF00231D461946DFF847
:1020F00078E1B2F9446002F1500C4832BB42C0F2C0
:102100009D8000293FF44EAF5B4B00261B78DFF823
:102110009491002B18BF0225584BD3F80080584BE0
:102120001B780A9308F105030793AE4240F3BC8085
:10213000544B93F8730200285BD0534B1B689D00EF
:1021400057D5524B1B88590653D44A4D504E95F8DB
:102150007030834211D085F8700011F0AFFE4D4908
:1021600011F000FF4C49074611F0F4FD10F021FF7B
:102170007060384610F01DFF6867D6F80480656807
:102180004146284611F0EEFEE768666F814631460B
:10219000384611F0E7FE0146484611F0D9FD3F49A7
:1021A000814612F087F808B9DFF8F0903C494846BC
:1021B00012F08AF808B9DFF8E89041463846C4F8CA
:1021C000049011F0CFFE31460746284611F0CAFEB2
:1021D0000146384611F0BEFD3049054612F06AF856
:1021E00000B92E4D2E49284612F06EF800B92C4D3C
:1021F000E5600022204B1A70D9E696F87222C2EBF5
:10220000421102EB8102D20043E735F9132039F97C
:1022100013C008FB02F292FBF0F23EF813602EF8B6
:1022200013C0ACEB0606324425F8132001334FE708
:10223000B4F84630013BA4F846304FE732F91310AA
:102240003CF81350414391FBF6F1022BA5EB010141
:102250001D46B8BF02252EF81310EDB201335146CA
:102260004CE700BFDC220020500C0020CE1E0020D6
:10227000540700200C070020BA0B0020380E002065
:10228000CC1E002018300020181C0020C63A002068
:102290000400002035FA8E3CDB0FC93F00C0F94432
:1022A00000C0F9C40AD7233C022E15BF98F80000DD
:1022B00098F8010098F802B098F809B011F0FEFD06
:1022C000494611F04FFE4FF08041074612F006F8E4
:1022D00060B14FF08041384611F03AFDB24911F03B
:1022E00041FE0146384611F035FD0746730005935F
:1022F000AE4B33F9160011F0E1FDAD4911F032FE9D
:1023000020F00043AB4A0593059B42F826000C32AF
:10231000824642F82630BBF1000F20D0584611F01B
:10232000CDFD494611F01EFE83465146504611F040
:1023300019FE059911F016FE594611F013FE594683
:102340000C904FF07E5011F003FD0C9A01461046A0
:1023500011F000FD0146504611F004FE82469649F8
:10236000384611F0FFFD514611F0FCFD079B074672
:1023700013F8010B079300B311F0A0FD494611F0CB
:10238000F1FD059911F0EEFD8C49824611F0A6FF92
:1023900068BB0021504611F083FF50BB51464FF0FF
:1023A0007E5011F0D5FC01464FF07E5011F08EFEAC
:1023B0000146384611F0D6FD07460A9B0C2B05D185
:1023C000384611F0ABFF7E4B720098527D4938467B
:1023D00011F070FF00B97B4F7B49384611F074FF54
:1023E00000B9794F794BB200D75001369DE6494686
:1023F000DAE74FF07E51D7E7B06F0FF0DCFBEFE587
:102400000CF006FAC0F17F00EAE50022704BDA67B3
:10241000C3F884206F4A1268C3F88820032323700E
:102420000CE06C4B6A4E1A68D6F8883064339342DD
:1024300004D240200DF0BEF9002874D00DF0E6F96A
:102440000646002800F0348401232370604B93F883
:10245000A12012B1002283F8A1205F4B1B78072B2B
:1024600005D108F07FF8089BC01A554B98800022D0
:10247000574B1A70584C2378072B02D108F072F88A
:102480000B90DFF86891D9F810504F46002D32D1EB
:10249000D9F804304846984768B389F82550B9F808
:1024A0001C30DFF84C811BB2C8F80030B9F81E3080
:1024B00099F826101BB2C8F80430B9F8203040460D
:1024C0001BB2C8F8083005F0A1FA444B1E88444BF3
:1024D0001B68002E40F03E849B79002B00F0B384F3
:1024E000EFF31283F02282F312883E4ADBB2C9F87E
:1024F000102083F31188384D2A78072A05D108F077
:1025000031F80B9BC01A2E4B1880314B93F8F020FA
:102510001C460592002A00F07185013A83F8F020EC
:1025200025B0BDE8F08FDFF8CC804027C146D6F853
:10253000843018F8030068B104F0BEF8F36F013F6F
:1025400003F1FF33F367D6F8843003F10103C6F8D3
:102550008430ECD1D6F8843019F80330002B7FF4A6
:102560006DAFC6F884304FF0FF33C6F888300423CF
:1025700055E71D4A5021A2F10C0301932523029235
:1025800000934920A2F10A03163A04F0D3FB002875
:102590007FF454AF4FF0FF320D4BC3F88400C3F803
:1025A000882007233BE700BFD7A36841500C0020D9
:1025B0006F12033B6407002000004843A4707D3F76
:1025C000CE1E002000C0F94400C0F9C4100700204E
:1025D0000C07002008350020CC1E0020F40F00203E
:1025E0005C100020357B0008B2930108F80F002032
:1025F000D41400203C930108052300210093AA4B2A
:1026000002910191A3F10802532004F093FB0028EA
:102610007FF414AFA54BC3F884000823FFE64020E5
:102620000DF0C8F800287FF409AF7423A0489F4E2E
:1026300090F81C14D6F8847003FB010292F88023F2
:10264000492F01F24184DFE817F04A004F005D0096
:10265000630066006C007000740078007E008200E9
:102660008E0098009C00A500A900AD00B100BA0042
:10267000C300CC00D500DE00E700F000F900060141
:1026800010011A01240185018F019901A301AD01F7
:10269000B301BD01C301C901CF01D501DB01E101D6
:1026A000E701ED01F301F901FF0105020B0211023F
:1026B00017021D022102250229022D0231023702D2
:1026C0003D0249024D025102550259025D0261026A
:1026D000650269026D02710275027F02830275490B
:1026E00075480DF0CBF907E0744B754A00937549B6
:1026F000754B76480DF0C2F9D6F884300133C6F830
:1027000084309BE6724A734973480DF0B7F9F3E7DA
:1027100072497348E5E790F8C82490F8C7147148E7
:10272000F3E7B0F8CC107048DBE7B0F8CE106F4894
:10273000D7E74FF07E516E48D3E7B6F88C20B6F855
:102740008E106C48E1E76C4B6C481989C9E7D6F8E4
:102750009030DB0403D590F838126948C1E70C23A8
:10276000C6F88430C8E790F83B3290F83D2290F8E4
:102770003C1264480DF082F9BEE7B6F89410624846
:10278000AFE72B681F05B7D5B0F94022B0F9421268
:102790005E48BAE75E4B5F48996CA2E790F8FE117D
:1027A0005D489EE790F8F8115C489AE759430C237E
:1027B00003FB0211014491F88213594891E75943F0
:1027C0000C2303FB0211014491F88413554888E758
:1027D00059430C2303FB0211014491F8831352481F
:1027E0007FE759430C2303FB0211014491F88B133B
:1027F0004E4876E759430C2303FB0211014491F83C
:1028000085134B486DE759430C2303FB0211014428
:1028100091F88613474864E759430C2303FB0211E0
:10282000014491F88A1344485BE759430C2303FBA6
:1028300002110144B1F88C13404852E759430C236C
:1028400003FB0211014491F8893391F888233C4835
:1028500091F887138EE703FB01013A4891F848335A
:1028600091F83E2391F8341384E703FB01013648C5
:1028700091F8493391F83F2391F835137AE703FB38
:102880000101324891F84A3391F8402391F8361308
:1028900070E703FB01012E4891F84B3391F8412377
:1028A00091F8371366E700BF609501080C07002018
:1028B0001830002040B201084CB2010810B10108E4
:1028C0005DB2010863B201082AB101086EB20108C5
:1028D00021B1010815B101088EB20108EC340020C5
:1028E000A2B20108B0B20108C1B20108D0B2010819
:1028F000DFB20108EFB20108B025002001B30108E2
:102900000BB3010818B3010831B301083CB3010847
:10291000F80F00204FB301085BB301086EB3010844
:1029200083B301088DB3010897B30108A4B301086C
:10293000B1B30108BBB30108C6B30108D3B30108A2
:10294000E5B30108F4B3010805B4010817B40108A0
:1029500027B4010803FB0101A44891F84C3391F816
:10296000422391F8381305E703FB0101A04891F8D1
:102970004D3391F8432391F83913FBE603FB010132
:102980009C4891F84E3391F8442391F83A13F1E6BC
:1029900003FB0101984891F84F3391F8452391F8D2
:1029A0003B13E7E603FB0101944891F83C1398E6DA
:1029B00003FB0101924891F8513391F8472391F8B4
:1029C0003D13D7E603FB01018E4891F8521388E6C8
:1029D00003FB01018C48B1F8541382E603FB0101AB
:1029E0008A48B1F856137CE603FB01018848B1F828
:1029F000581376E603FB01018648B1F85A1370E6D6
:102A000003FB0101844891F85C136AE603FB0101B2
:102A10008248B1F85E1364E603FB0101804891F837
:102A200064135EE603FB01017E4891F8651358E6E6
:102A300003FB01017C4891F8661352E603FB010198
:102A40007A48B1F86C134CE603FB01017848D1F8E1
:102A5000701346E603FB0101764891F8741340E6D3
:102A600003FB0101744891F875133AE603FB010179
:102A70007248D1F8781334E603FB01017048D1F8AD
:102A80007C132EE690F84C126E482AE690F84D1210
:102A90006D4826E690F8FF116C4822E690F8001287
:102AA0006B481EE690F801126A481AE6B0F8082250
:102AB000B0F80412684828E6B0F80A22B0F8061206
:102AC000664822E6B0F8160211F0F8F9644911F0F0
:102AD00049FA11F023FC0146624802E690F8191207
:102AE0006148FEE590F824126048FAE590F80F126C
:102AF0005F48F6E590F8B0125E48F2E590F8701283
:102B00005D48EEE590F872125C48EAE5B0F876129E
:102B10005B48E6E590F85C125A48E2E590F8D5107B
:102B20005948DEE590F8D4105848DAE5B0F8D210EC
:102B30005748D6E54A49D0F8D80011F013FA11F0F9
:102B4000EDFB01465348CCE590F8F9115248C8E531
:102B500081685248C5E5524B1B68990115D5514E05
:102B6000B6F898308BB9D6F89C3018A91893069B04
:102B70000E20199303F044FE4FF48053A6F89630CC
:102B80000A232370069803F087FE03F019FE55E42C
:102B9000444B93F8A020002AF4D0414A12689201D5
:102BA000F0D493F8A130002BECD109232370ECE78B
:102BB0003D4B3C4E1A68D6F88830C83393420FD24A
:102BC0003A4B93F8C9744FB9B06F08F0C8FA96F849
:102BD000A230B767022B01D106F00EFE01231EE4DE
:102BE00013F044FD0028EBD128E400BF37B40108FE
:102BF00047B4010858B4010869B401087BB401085E
:102C00006BB4010885B401089AB40108AAB401089C
:102C1000B8B40108CAB40108E0B40108FBB4010863
:102C20000AB5010821B501083AB501084EB50108F9
:102C300068B501087DB5010893B50108AAB501087A
:102C4000BFB50108D5B50108D1B50108E1B5010846
:102C5000EDB50108FFB5010812B6010826B6010856
:102C60000000C8423EB601084CB601085CB6010837
:102C70006DB601087DB6010896B60108AAB601082E
:102C8000C7B60108E4B60108F9B601080EB7010895
:102C900023B7010835B701084AB7010858B701083A
:102CA000181C00200C0700200835002018300020D8
:102CB000A94991F8CA34002B3FF4CFAB2B68DF044D
:102CC0004FF000034CBFB1F8EC50B1F8D050A34F17
:102CD00037F913200133AA420CBF304646F00100F9
:102CE0000C2BC6B2F4D19E4D9E4BC6B11B6803F5AA
:102CF0009C530833C5F8A4302378012B7FF4ADAB87
:102D000095F8A130002B7FF4A8AB91F8C934D3B16A
:102D100004F0DEF8012385F8A130FFF79EBB1A68A6
:102D2000D5F8A4309342E7D82378012B3FF495AB34
:102D300095F8A130002B3FF490AB04F0ABF885F888
:102D4000A160FFF78ABB80200EF014FB00287FF4FF
:102D500084ABDDE75B78D9F8482007934FF47A73AA
:102D6000B3FBF2F3AB46C3EB431203EB8203DB008E
:102D70009BB2059323787C4C0C937C4B04F13C096B
:102D8000B3F90630CDF820800693059B5B080E93BF
:102D9000059B4FEA850A9E4202BF002349F8253071
:102DA0002361089B53F8250059F82530034449F85E
:102DB000253011F083F8226902F10108B8F1010F02
:102DC000C4F8108040F0A180002360602060A36000
:102DD000089B012E1A464FF000034AF802304FF0CC
:102DE0000002634B4AF8032040F0E280206901288A
:102DF00040F3AF80013811F061F80146E06811F04E
:102E000065F914F0F3F80C9B8046032B05D113F001
:102E10002DFE4FF0010B03B20693079B002B00F031
:102E2000BD80184611F04AF8414611F039FA0028E1
:102E300000F0B480BBF1000F03D04C4BBDF818205C
:102E4000DA8004F0ECFCDFF84C914FF0000BCA463E
:102E5000DFF84481474C464B54F82B0053F82B3095
:102E60004FEA8B05C01A44F82B0011F027F8424BAB
:102E7000996911F077F899F800300146032B06D1D3
:102E8000059013F0F3FD394B059923F81B003B4ADD
:102E90003B4BA8581B6898479AF800300146082B0E
:102EA00006D1059013F0E2FD304B059923F81B0085
:102EB000344A354BA8581B689847344A344B01466E
:102EC0001B68A85898470BF1010BBBF1030F48F89A
:102ED000040FC0D1002E3FF40EABBD69F86C29463B
:102EE00011F0F4F813F0C2FD29462060386D11F09E
:102EF000EDF813F0BBFD29466060786D11F0E6F83F
:102F000013F0B4FDA060FFF7F6BA226810901146E6
:102F10000F9210F01DFF0A90404610F0CFFF0146BF
:102F20000A9811F0D3F80F9A114610F013FF109B76
:102F3000014680466060184610F00AFF0A9911F0B9
:102F400011F8A16810F006FFC4F80080E060A060EE
:102F50003EE7002055E700BF18300020241C002069
:102F60000C07002008350020B4070020CE1E0020EA
:102F7000E0140020D4140020F80F0020B41000202A
:102F8000501000204414002054100020A4140020ED
:102F900058100020CC1E0020401000200E9A5AF835
:102FA00009301344059A93FBF2F3104A42F80A30B1
:102FB0000135032D04F114047FF4EAAEBBF1000FD8
:102FC00003D00B4BBDF81820DA80012E08D1002267
:102FD000084B30461B689A621A63DA620CF09EFD59
:102FE000054A1388013B13802DE700BFE014002041
:102FF000CE1E002008150020F40F0020A84B93F8E7
:103000000122002A00F0458193F8F831013BDBB240
:1030100084F8F0302B78072B02D107F0A3FA0D903B
:10302000A04B4FF07E501B6806939F4B1B680A9382
:10303000D4F8F4301946089310F08AFE9B4B1968B7
:1030400010F090FF4FF07E51079011F033F910B956
:103050004FF07E5307934FF0000B4FF07E55944B8B
:103060000B93944B944F53F82B80002140464FEA2A
:103070008B0457F82B6011F009F9D0B9F43757F8E1
:103080002B903046494610F063FE824620F0004106
:10309000404611F005F958B10021504611F01EF9D3
:1030A000002800F0F8804946404610F053FE0646DE
:1030B0003E51824BB3F8009019F0030F3ED0BBF1A4
:1030C000020F3BD0069B93F8340010F0F7FE7C4BC8
:1030D000E15810F047FF069B804693F833A0CAF1F1
:1030E000000010F0EBFE07460146404611F0D8F80C
:1030F00040B9504610F0DEFE4146074611F0DAF8BE
:1031000000B947466F4B33F91B00654B03EB4B038C
:10311000B3F92032C01A10F0D1FE6B4910F022FF33
:103120000146384610F014FE19F0010F0C9000F023
:10313000EF80664B196810F015FF06460B9B304672
:1031400053F8049F49460B9310F002FE8246604BF1
:103150000A98E15810F006FF514610F003FFBBF14A
:10316000020F804606D15B4A5B4B01461B68106824
:1031700098478046594B29460898E75811F090F82F
:10318000B0B1574B1968574B186810F0EBFE079910
:1031900010F0E8FE544BE15810F0E4FE514610F0F8
:1031A000E1FE0146384610F0D5FD07464B4BE05096
:1031B000BBF1020F40F076813946404610F0CAFD5F
:1031C0004A4EC6F80C01404611F0A8F8C6F818019E
:1031D000384611F0A3F80023C6F82401C6F83031B0
:1031E000434B1B7813B90022424BE2500BF1010B09
:1031F000BBF1030F7FF435AF3F4C2278072A05D18E
:1032000007F0B0F90D9BC01A3C4B58802378374D1E
:10321000012B40F0B08107F0A5F93949D5F83C31D0
:10322000364A0968C31A93805B1A0990D380C5F89F
:103230003C011C4B1C68334B1B680B9313F48053ED
:103240000C93314B00F0F583304AD5F848111278D1
:10325000C988560758BFD5F84421B3F906305CBF7A
:10326000D28AA5F84021D5F84421D68A701A834223
:1032700000F3B681B5F84C11108BB5F88E8007912C
:10328000A5F84031181A10F019FED5F8503107464C
:10329000B8E10123BCE64146484610F059FD06E777
:1032A00018300020881E0020BC0B00209422002033
:1032B000401000208822002010070020C63A00207D
:1032C000640700202A260020CDCCCC3D78220020A7
:1032D0004C22002048250020442500205C0B0020C3
:1032E0000400002084220020582200200C07002027
:1032F000680B002010080020CC1E0020CE1E0020ED
:10330000DC22002000170020500C0020282600207E
:103310009C4BD3F864809F6E4146384610F0C0FF46
:10332000002878D04146284610F012FD964B804682
:10333000B3F90000B3F9023080EAE07183EAE37286
:10334000A1EBE071A2EBE372914266DD0028D8BFE9
:10335000404210F0B3FD8D4910F004FE069B074675
:1033600093F83630012B069B93F835005CD1AE28DC
:1033700000F29580C0F1AF0010F0A0FD844910F07C
:10338000F1FD8146394610F0E3FC494610F09EFEFF
:103390002946074610F08EFF00B92F460021384617
:1033A00010F092FF00B900277A4B0021D3F800906B
:1033B000484610F07FFF002834D12946404610F0DF
:1033C000C7FC754910F0CEFD494610F07FFE294636
:1033D00010F0C0FC0146384610F0C4FD80466F4B2B
:1033E0000C98196810F0BEFD29460746404610F0BB
:1033F00061FF00B9A8460021404610F065FF08B9FA
:103400004FF000084146384610F0ACFD014630460A
:1034100010F0A0FC91E6394685E7002BCCBF18469A
:10342000584296E70021D6E7002835D0C0F1640065
:1034300010F044FD5A4910F095FD0146814628469A
:1034400010F086FC574910F08DFD394682465648EB
:1034500010F07EFC0146504610F084FD494610F005
:1034600079FC4C4B196810F07DFD07460021384669
:1034700010F020FF98B92946404610F069FC394603
:103480008046454810F022FE0146404610F06AFD95
:10349000294610F05FFCA1E73E4B1F68E6E74FF0BE
:1034A00000089CE7414B1A68069B93F84030632B59
:1034B00012D83F4B0C92E1583E4B186810F052FD69
:1034C0002946824610F0F6FE0C9A00B9AA4610462C
:1034D000514610F047FD02461146304610F042FDBD
:1034E000494610F035FC344E8246A15910F030FCAC
:1034F000324B196810F0EAFD8146314B44F806A0C2
:10350000E1580A9810F02EFD494610F02BFD2D4B86
:1035100006461B780B2B04D110F000FF2A4B23F832
:103520001B002A4A2A4B31461B68A0589847294A53
:10353000294B01461B68A0589847814639464046AA
:1035400010F008FC494610F005FC244E305140466E
:1035500010F0E4FE06F10C0A4AF80400384610F0B8
:10356000DDFE06F1180848F80400484610F0D6FEC3
:103570002436305134E6072B7FF45BAE06F0F2FFC1
:10358000099056E60C0700202A260020CDCCCC3D21
:103590006666E63F802200200000C8427C220020B0
:1035A0000AD7233C610BB63B000034437022002055
:1035B0007007002074220020400800208422002090
:1035C00064220020CC1E0020CE1E00209C22002061
:1035D00098220020E4220020E02200201008002091
:1035E00072189342C0F21182B5F88C20A5F84031D0
:1035F0009B1B581A079210F061FC0746B5F85481DE
:10360000D5F858310893079BDFF840A3A3EB0800D7
:1036100010F054FC0023D4F82C900D9009F10045D3
:10362000069315AEB04B069A514653F8220010F09F
:1036300099FC2946834610F033FE002840F00B82A7
:103640004946584610F036FE00B9CB46069B46F870
:1036500023B00133032B0693E4D1A44B1B6843B37F
:1036600094F831202AB30B9A940722D5A04A1478F3
:10367000FCB1D87810F01EFC0546204610F01EFC68
:103680000146284610F06EFC9A4B0446188810F04C
:1036900011FC0146204610F019FD9749044610F030
:1036A00009FE00B9944C4FF07E51204610F00CFEFC
:1036B00008B94FF07E544FF0000A0026D1468F4BD8
:1036C0008F4D1B7805F5B2750A93169B0DF1600BB3
:1036D0000E93159B0F93179B109355F8043C119371
:1036E0000A9B9E42C0F2B9815146484610F030FB19
:1036F000834B4FF07E51C3F8F400044610F0EEFD0A
:10370000002800F0F98121464FF07E5010F0DEFCD9
:103710000024064618AD0A9BA34200F3E4814FF053
:103720007C560025774BDFF8EC91DB780E93764BD7
:10373000B3F800A0754B0FFA8AFB1C78744B04F0A9
:103740000404B3F906706E4BD3F8442103F5B27349
:103750000F930B9B089203F010030B930A9B9D425F
:10376000C0F0F7812CB96B4B6B4A0A99A14200F269
:103770002782634CD4F82432002B00F05D8394F848
:103780002932192B00F2938001229A40634B134097
:10379000002B00F08C80624B1B88D80540F116820C
:1037A000604B1A88ADF860205A889B88ADF862207B
:1037B000ADF864304FF47A724FF461615A48B0F951
:1037C000023003F5E163534393FBF1F3A3F5FA737E
:1037D000ADF87830B0F9003003F5E1635A4392FB5D
:1037E000F1F24C4BA2F5FA721B88ADF87A20A3F2E5
:1037F000DC53474AADF86630D4F844311188DB8A8F
:10380000C91AADF868105188C91AADF86A109188C4
:10381000C91AADF86C10D188C91AADF86E101189AB
:10382000C91AADF870105189C91AADF87210918992
:10383000D289C91AD31AADF876300023ADF87410C6
:1038400019463A4A22F813100133082BFAD164279B
:10385000374B384A1B68384C0793384BDFF8CC900D
:103860001B680893364B1B78C3EBC30313440B93BD
:103870000B9B934240F0D88100254FF00E0964273E
:103880002E4B304ED3F8008009FB0583B6F9024079
:1038900093F90600444394FBF7F4E8B274800CF00B
:1038A000A3F901352044082D26F8020FECD1264D4E
:1038B000224E2B6813F0200F69D000200CF094F9F1
:1038C0001A4C0746208001200CF08EF9184B6080BE
:1038D0001B6819065BD50A4B1349D3F84C321B7889
:1038E000012B40F0128233E010080020F014002079
:1038F000EC140020F8140020713DAA3F5C25002044
:103900000C070020441800206A1D002028260020F3
:103910001818002064250020241C002032413003A8
:10392000C63A0020500C00202A260020AC050020BA
:10393000181C0020D1210020360900204822002038
:10394000D0210020AA050020001700206F12833A22
:10395000326892F9063092F91420C3F1000EB1F9E1
:103960000230B1F9001003FB0EF34FF0320E514359
:103970006FF0310293FBFEF391FBF2F291FBFEF14B
:103980009BB21A44BA1A22800B44184460803368F0
:10399000A24A03F17004B2F90200B3F90010B3F9BE
:1039A0000270884203DB87423946A8BF01460E33C6
:1039B0009C4222F8021FEED1994CD4F8503293F970
:1039C0000430002B40F0B68194F82932013B182BCB
:1039D00000F20482DFE813F0F6010202020255024F
:1039E0000202020202024A0202020202020202026F
:1039F00002025C02020202020202020202025502FA
:103A00006902020202025C02F601B5F840319842F6
:103A100005DBB5F84C31B5F88E80079333E4B5F883
:103A20008C30B5F854810793D5F8583100270893A6
:103A3000E9E5B3F90600D5F844311B8BC01A10F044
:103A40003DFAD5F85C3107460893B5F88C30B5F8E7
:103A50008E800793D7E5AB46F8E5119B93F90100FB
:103A6000404210F02BFA109910F07CFAE96810F03F
:103A700079FAA96813900E9810F074FA6968129098
:103A80000F9810F06FFA129A0146104610F062F982
:103A9000139B0146184610F05DF94FF07E511290CD
:103AA000204610F01BFC129BB0B94BF826305BF897
:103AB000263049461846129310F010FC129B38B974
:103AC0001946504610F0F6FB08B9129B9A464B4631
:103AD00001361035994603E62146184610F042FAA1
:103AE0004BF82600E3E755F82400314610F03AFA87
:103AF00045F8240001340EE60899384610F0E6FA3D
:103B00004FF07E51054610F0D5FB08B94FF07E55B9
:103B10000021284610F0D8FB00B900254FF07C5159
:103B2000204610F01FFA06460146284610F0B8FB62
:103B300000287FF4F6AD31464FF07E5010F008F9C2
:103B40002946064610F0B6FB00287FF4EAAD2E4663
:103B5000E7E50F9A2B019958304610F003FA18AB9D
:103B600053F8251010F0F6F80D9910F0FBF912F04B
:103B70007DFF0E9A404400B26B0029F81500DAB1BF
:103B8000504504DB079A9042A8BF104600E050461B
:103B90000B9A29F803006AB164B10C9A52B91093D8
:103BA0000EF07CFE30B9089B1A8B9742BCBF109B6D
:103BB00023F809B00135D1E58045E3DD4046E7E76C
:103BC00032F8141023F814100134CEE51549D4F856
:103BD000040110F0C7F910F0A1FB1249ADF8600024
:103BE000D4F8080110F0BEF910F098FB0D49ADF8BB
:103BF0006200D4F80C0110F0B5F910F08FFB0C9BAB
:103C000000B2ADF86400002B3FF4D4AD089BDB8A12
:103C10009F42BCBF4042ADF86400CBE5AA0500203E
:103C20000C0700203333333F937933B1012115332F
:103C300001FA03F307990B4065D00E21089B92F817
:103C400000E092F904B001FB0E3CBCF90230BCF973
:103C5000001056785B1A9BB203FB0BFB9BFBF7FB38
:103C600092F905104FEA530A0A91D178ABEB0A0B8F
:103C70000FFA8BFB750051BB24A90D4435F8301C9D
:103C800021800120DCF80A1000FA06F63142B4F96E
:103C9000005092F9021018BF4FF0FF30694391FBBA
:103CA000F7F159450ADB0A9D6B4393FBF7F3A3EB4E
:103CB0000A0B0FFA8BFB8B45A8BF8B4639F81E30D9
:103CC00000FB0B3B29F81EB002340732D0E50DF1A2
:103CD00090084544B4F9000035F9305CA84208DA90
:103CE0000144884203DC8D422846A8BF0846208054
:103CF000C7E7C6DD411AA94203DB8842A8BF0846D0
:103D000005462580BDE72380DEE73368B1F9022050
:103D100093F906E002FB0EF24FF0320E92FBFEF238
:103D20003A44228093F91420B1F90030534393FBB5
:103D3000FEF32AE60023DFF8AC81A4F8543204F540
:103D40001677B4F95492B9F1070F3FF73DAE94F8E6
:103D500056327BB9D4F85032588810F0ABF801468F
:103D60001C205F4B00FB09701A680FF025FA012335
:103D700084F85632B4F9549238F9190010F09EF8CC
:103D800001461C2000FB09700EF0DEFF12F06EFEF3
:103D90000E22B4F95432316828F8190002FB0312DC
:103DA00038F91300B2F90010B2F90220884203DB9F
:103DB0008242A8BF0246114628F813100133A4F826
:103DC0005432BEE7D4F850321B78002B48D0454B14
:103DD000598900200BF074F8012305932B689A068B
:103DE00003D494F82932052B0ED13E4E0598318824
:103DF0000BF066F8059B7188581CC0B20BF060F898
:103E0000059B0233DBB205932B68DB0214D5D4F893
:103E1000383300241D78344EE0B22B18DBB2112B5E
:103E20000AD8059A2B19104436F81310C0B2013481
:103E30000BF046F80E2CEFD12C4C94F828220AB146
:103E40000CF062F82A4B1B78072B05D106F08AFB91
:103E5000099BC01A274BD88001232370FEF760BB53
:103E6000254B197811F00401B1D1B2E71D4E0020A5
:103E7000F1880BF025F8318901200BF021F802239D
:103E8000ABE7184E002031890BF01AF87189F3E77F
:103E90000226144FB01E37F81610C0B201360BF0D0
:103EA0000FF8082EF6D1062397E70E4E069BD81E74
:103EB00036F81310C0B20BF003F8069B0133072B42
:103EC0000693F3D1042388E712F0D0FB00283EF4D8
:103ED000B5AA4FF48053A6F896300A23FEF79FBA8E
:103EE000DC220020AC050020181800200C07002060
:103EF000CC1E0020CE1E0020282600202DE9F04FE9
:103F0000AC4B00F59C4808F12008C3F80080AA4B90
:103F100087B01D780746002D6ED0A84A12689042DF
:103F200001D9013D1D70A64B1A689B4612F4805FB3
:103F300005D0A44B1B68D90701D405F0EFFDA24BB7
:103F40001C68E07C002800F08081A04A637D013875
:103F500032F910001BB1C0F53B60083000B2A0F58B
:103F60007A70B0F57A7FA8BF4FF47A7020EAE070DB
:103F70000FF0A4FF96490FF0F5FF10F0F5F9954BFF
:103F80001880DBF80030DFF880A213F4807F00F0A7
:103F9000D981914BDFF860929F4205D999F80220B0
:103FA00012B9012289F8022099F80220002A00F0B3
:103FB000C981844999F8215008689AF8002000F0D6
:103FC0008063012D02F004080093019100F07581D7
:103FD00012F0080F0CBF00270227804C804E99F882
:103FE0002020052A00F2AA81DFE812F06901CF0142
:103FF000DA01FD010D02290205F07EFB8146794CB4
:10400000714EDFF8F8A1A94546DC42F201024FF4F7
:104010007A796B4BB7FBF9F91B6813400193724B2C
:1040200006D0724A12781A70714A1178714A11706A
:104030001B78009323B16F4B1E7886F00103009329
:104040000F230025DFF8C4B1DFF880A184F8243005
:1040500005F052FB85424DDB94F824305F4A0F2B6C
:104060000CBF0123002384F8D230634B40F0D08092
:1040700054490968480100F1CB801268D9689A60F8
:10408000521AC82A02D9012283F8212094F8B830A4
:10409000013384F8B83046E7072DD8BF3368E9B25A
:1040A0005648D8BF595DDAF804309847032D1DDC17
:1040B000326805F1130302EB830E32F82310BEF8C9
:1040C000022098B1431A4FF47A705843531A90FB68
:1040D000F3F040F2EE2300F57A709842B8BF18462C
:1040E00040F6CA039842A8BF184680B224F81500CB
:1040F000013588E7009A6B00DAB134F91500324ACD
:1041000080B21268918C81424FEA850103D8B2F8DF
:1041100026E0864520D23A4A515889450BD23AF8D2
:104120000300019AEAB92AF8030001350BF1060BE6
:104130008EE70098E3E7E8B2029305F0F3FA032D67
:10414000029BEEDC012101FA05FE94F8241021EA1D
:104150000E0184F82410E4E7294E09F59672725096
:10416000DFE7032194F8B8C003EB050EBCFBF1F1C7
:1041700001EB4101ACEB0101C9B2714404EB410117
:10418000C88494F8B91029B9BCF1020FCBD9012128
:1041900084F8B910BBF80010BBF802000844BBF863
:1041A00004100844174900B2C852032190FBF1F0F3
:1041B00080B2B8E734170020401800203C180020D7
:1041C00000170020181C00201418002018180020C8
:1041D000AAF1823F4A0E0020404B4C0008350020D7
:1041E000582600204C0A0020F5160020FC1600205E
:1041F000200200202102002044180020281700205F
:10420000BC0A0020060B002028260020720A00208D
:1042100001219648126801709548DA60017099682A
:104220000025521A5968934E8A4284BF002283F8AF
:10423000212005F061FA8542BFF628AFE8B205F00B
:1042400071FA26F815000135F3E7DBF800301A049F
:104250007FF597AE884AD2F8D430FB1A002BFFF6D0
:1042600090AE92F8E930C2F8D48002EB4303B3F881
:10427000EC10237D89B291FBF3F192F8F430013315
:1042800003F00F0382F8F430134483F8F51003466B
:10429000F532995C01330844102B00B2F9D190FB40
:1042A000F3F000B2002806DB6428A8BF64200FF0FA
:1042B00005FE72495FE60020F9E700278DE6B8F1B8
:1042C000000F32D06C4AB2F80611D2F808010EF095
:1042D000ADFA012807D1642032682168D28800FB3A
:1042E0000212C9F81020009B63B1326812794AB1FA
:1042F0000CF0EAFA032289F820204FF47A72C9F808
:104300001C206CE6012D19D02268D9F810109142BA
:1043100007D20CF0D9FA032289F8202040F6B832EF
:10432000EDE7012289F8202059E6009B4FF48060D8
:1043300043B30EF047FA0022C9F8102017B13846EF
:104340000BF0ECFB4E4D4C4CB5F8EE1005F515702E
:104350000EF06CFA06460EF0A1FA002800F09680E6
:104360009AF800305F0740F19180464BB3F9062080
:10437000B5F876329A42C0F28581012384F80C3177
:10438000012397E00EF00EFAD5E7012D01D10522A9
:10439000C8E73268127A012ABBD00CF095FA1EE603
:1043A000012D04BF052289F82020B8F1000F0CD0A0
:1043B0000327314AD2F80821B2F916102D4A11808C
:1043C0005180918031684988D1802268D9F81410D1
:1043D000914202D3B8F1000F43D147F23052C9F8ED
:1043E0001C2003229EE79AF8002042F002028AF87D
:1043F000002005F093FB2168D9F81C200A44C9F875
:10440000182004228EE7012D12D12268D9F8181045
:10441000914293D21C4B1A781AB9019B1A68D307A0
:104420008CD49AF8002022F002028AF80020AEE72D
:104430002168D9F81C200A44C9F818207EE76420B6
:1044400032682168D28800FB0212C9F810200022CD
:104450004FF4806089F8202089F803200EF0A2F93B
:10446000BDE5012D3FF4BBAD68E700BF2002002091
:1044700021020020181800204C0A002014AE23410D
:1044800018300020500C00200C000020002384F87D
:104490000C31002E7FF474AF0023C4F81031C4F83F
:1044A0001431C4F81831B64B1B6893F83230002B26
:1044B0007FF466AF84F81C319AF80030580725D590
:1044C000DBF80030D90621D5AE4A1278D2061DD4C9
:1044D000DF041BD40EF0E2F9C0B9AB4B1B78002B04
:1044E00000F0EB8095F8B232002E40F0D480002B23
:1044F00000F0E580A54B1A68D4F820319B1A002BF8
:1045000080F2DD8005F00AFB84F824610022134666
:1045100095F8B112B5F86CE2B5F86EC29C4830F966
:1045200012709B087745C4BF63F07F03DBB2013292
:104530006745B8BF43F04003042AF0D194F8252121
:104540009A4240F0C38094F82621F92A02D8013219
:1045500084F826218C4A84F8253113788D4F9046B3
:1045600063B93A68D00740F1B38084F827312EB997
:104570009AF80030DA0701D505F06CFA94F8263184
:10458000142B1AD198F800305BB194F825315F2BC9
:1045900007D19AF8003013F0040600F0B98005F056
:1045A000BDFA9AF8003013F0040206D194F82531D0
:1045B000572B40F0B38003F032F9DBF80030580796
:1045C00026D594F82A319BB19AF8003059070FD5B7
:1045D0006F4BB3F90620B5F86C329A4208DD3B68A0
:1045E00013F0010302BF322284F82A31A4F82E21ED
:1045F0003B68DA0340F1108194F830312BB994F81C
:10460000283113B93223A4F82E31012384F8303134
:1046100000234FF00109604E3B6006F1500831461F
:1046200016F8010C0EF0DCF830B116F8023C3A68CE
:1046300009FA03F313433B6004364645EFD1574B69
:104640001F78002F00F0F880524E554F336813F05A
:10465000020F09D1DBF80030D80540F1CE82514B72
:10466000DB78002B00F0C9823B68990740F1C582D6
:104670004D4B1B8813F0010802D101200EF0A2F867
:104680000023BEE2002E7FF47BAE94F80C31002BA9
:104690007FF476AE00E73BB14FF47A713B4A126883
:1046A00001FB0323C4F8203194F82431002B3FF49C
:1046B0002DAF06F0A5FE002305E0002EF4D110205A
:1046C0000BF02CFA012384F824311FE700223FE786
:1046D0009AF800305B077FF551AF344B1B78002B05
:1046E0003FF44CAF2F4BDB78002B7FF447AF94F8AF
:1046F00027310133DBB2032B84F827317FF63EAF3D
:1047000011B105F00BFA39E7002E7FF437AFF8E767
:104710000B200BF003FA84F8266142E7DBF8001067
:104720004E0717D55A2B15D194F828312BB10123F8
:1047300084F8282184F829313FE794F82A3183F05E
:10474000010384F82A311BB10C200BF0E7F934E7A0
:104750000D20FAE75D2B00F019845B2B00F01D841F
:104760005E2B40F01C84032000F011BC94F825312E
:10477000972B1DD14FF4C873A4F82C311DE700BF4F
:10478000881E0020342600200C0000200835002060
:1047900018180020181C002037340020681D002045
:1047A000AC25002044180020C63A0020F516002051
:1047B000A72B05D1BC4A137843F004031370FCE621
:1047C0000022BB2B059216D10223ADF81630B5F8A6
:1047D0002032BDF814201344A5F82032BDF816206D
:1047E000B5F822321344A5F8223205F0E7F9002388
:1047F00084F82631E1E6B72B02D14FF6FE73E4E7E9
:10480000BE2B03D10223ADF81430E0E7BD2B7FF4BB
:10481000D4AE4FF6FE73F6E794F82831002B3FF440
:10482000F7AE9AF8003013F0040302BF84F8283181
:10483000012384F82931EBE64FF00C099B4E06F179
:104840005A08314616F8010C0DF0CAFFE8B131796B
:10485000B37809FB0140964A013B03EB4303134441
:10486000D0F8382196F803E093420ED0C0F83831E2
:10487000012303FA01F194F8643180F834E123EA6A
:104880000101C0F83C7184F8641106364645D8D160
:10489000884BDFF830921E68874B1B680193874B6B
:1048A0001B78029300230093D9F80420002A6BD0D0
:1048B0001778002F68D0D9F808300199CB1A002B4F
:1048C0000DDB01F5FA730121C9F80830009B01FAEC
:1048D00003F394F8641121EA030384F86431029B22
:1048E000002B51D099F8003051780433DBB2002905
:1048F00040F05281724931F91310B5F86A3203F170
:10490000C80081422ADD92F80280009B94F864215D
:104910001A41D30738D4B8F1000FCCBF02200120D0
:1049200006F052FD7A1E162A41D8DFE812F0350053
:104930004E00580068007F008600A100CD00E9000D
:10494000F50001014000680075008600A100CD005F
:104950009500B000DD000D0119012701C83B994207
:1049600003DA9178C1F10008CFE70122009B02FA37
:1049700003F394F8642122EA030384F86431019B71
:1049800003F5FA73C9F80830009B09F10C090133EB
:10499000042B009388D157E6317801204144FA294D
:1049A000A8BFFA2121EAE17131700DF063FFD4F85C
:1049B00068010BF033F90122009B02FA03F394F82B
:1049C0006421134384F86431DEE7B1780220414466
:1049D0006429A8BF642121EAE171B170E5E731796A
:1049E0008844B8F1640FA8BF4FF0640828EAE8785B
:1049F00086F804800EF0CCFC41460320D5E7B1795F
:104A00000D2041446429A8BF642121EAE171B171FC
:104A10000DF030FF0D2FCAD071790E20414464296A
:104A2000A8BF642121EAE1717171BEE7F179052027
:104A3000414481F30801F171B7E7D4F868210F20F0
:104A400051784144C829A8BFC82121EAE1715170B9
:104A50000DF010FF0F2FAAD0D4F868211220117882
:104A60004144C829A8BFC82121EAE17111709CE71F
:104A7000D4F868211020D17A4144C829A8BFC821A0
:104A800021EAE171D1720DF0F5FE102F8FD0D4F82C
:104A900068211320917A4144C829A8BFC82121EA7E
:104AA000E171917281E700BF342600208634002036
:104AB00080950108380E002008350020F5160020EA
:104AC00018180020800B0020D4F868211120517D97
:104AD0004144C829A8BFC82121EAE17151750DF0F0
:104AE000C9FE112F3FF463AFD4F868211420117D63
:104AF0004144C829A8BFC82121EAE171117554E7D2
:104B0000D4F86821092091784144C829A8BFC82158
:104B100021EAE171917048E7D4F868210A20117BFD
:104B20004144C829A8BFC82121EAE17111733CE7BB
:104B3000D4F868210B20917D4144C829A8BFC82121
:104B400021EAE171917530E7717815204144B1F5A2
:104B5000967FA8BF4FF4967121EAE171717024E746
:104B6000D4F86821162092F841104144FE29A8BFCC
:104B7000FE2121EAE17182F8411016E7D4F868219C
:104B8000172092F8401041446429A8BF642121EA0B
:104B9000E17182F8401008E701297FF40CAF0C2F77
:104BA0007FF409AFBB494FF4966031F9133040F6FA
:104BB00033018B42A8BF0B469278B3F5617FB8BF33
:104BC0004FF4617390FBF2F0A3F5617393FBF0F384
:104BD000B14ADBB212789A423FF4EDAE1846039325
:104BE00004F0BAFF039B384619460DF043FE039BC1
:104BF000581CC0B206F0E8FBDDE601200DF0D2FD46
:104C000001233268520740F12681002B00F02381F6
:104C100001200DF0C7FDA14B1B889B0702D4022089
:104C20000DF0D0FD3B6813F00A0F20D03368DF068B
:104C300040F11581994B1B88580702D404200DF0D0
:104C4000C1FD3368990640F10E81944B1B885A06CA
:104C500002D440200DF0B6FD33685B0607D50A226A
:104C60008F4BB3F9043093FBF2F3A4F86C31336843
:104C70004FF480701F0540F1FA800DF0A3FD95F808
:104C8000B332082B01D00E2B02D140200DF08AFD4B
:104C9000DBF80030590510D595F80433002B40F0AF
:104CA000E9809AF8003013F0040F00F0ED803C200A
:104CB0000CF060FB002840F0E180012384F86E31A5
:104CC000744BB3F90660774B1B685A89964280F2A1
:104CD000F5804FF07E53C4F87031002295F95032C0
:104CE000B5F86A125B429BB295F84D8295F84CC2BA
:104CF0006D4F019340F2E630664B4FEA420E33F9B6
:104D0000123000935B1A03F2F319814500F25981C6
:104D1000002BB8BF5B42022A00F05881634540F384
:104D2000E180A3EB0C0327F80E30009B8B42C0F20E
:104D30005A810132032ADDD1DBF8002012F48052BF
:104D400000F0D280B6F5FA6FA8BF4FF4FA66B6F558
:104D50007A7FB8BF4FF47A76A6F57A764FF0640E74
:104D60006FF0630C96FBFEF304EB43000CFB036354
:104D7000B0F97451B0F97601401B434393FBFEF345
:104D80002B449BB2FB80AAB1484A1268D20011D5CD
:104D9000474AD27872B94FF47A72A3F57A731BB28C
:104DA0001B0393FBF2F3C1F5FA6212B2534301EB1A
:104DB0002331F980394B1B885B0642D5384BB3F958
:104DC00004000A2390FBF3F0B4F86C31C01A00B26F
:104DD0000FF074F837490FF0C5F8374905460EF063
:104DE000B9FF0EF0E6F8804628460EF0E2F80546D8
:104DF000B7F902000FF062F80646B7F900000FF0AD
:104E00005DF8414681460FF0ADF8314683462846AD
:104E10000FF0A8F8014658460EF09AFF0FF07EFA00
:104E20004146388030460FF09DF8494606462846F0
:104E30000FF098F8014630460EF08CFF0FF06EFA36
:104E400078809AF800305E0762D5012007B0BDE88F
:104E5000F04F0CF0CDB902200DF0A4FCE2E60420E6
:104E60000DF0A0FCEDE640200DF09CFCF4E60DF00A
:104E700099FC04E7336813F4002F16E704F0A6FC4E
:104E80003C200CF043FA15E70AF098FB04F0B4FC60
:104E900013E700BF18180020221C0020C63A00208B
:104EA0002A260020380E0020500C0020181C00205C
:104EB0004418002035FA8E3CDB0FC93FB6F5FA6F77
:104EC000187ABFBFB31A5843C2F5FA6290FBF2F0EA
:104ED000C0F164000EF0F2FF47490FF043F8C4F848
:104EE0007001FAE600231EE7B5F86C0286420DDB7E
:104EF000B6F5FA6FA8BF4FF4FA664FF47A73361A14
:104F00007343C0F5FA66B3FBF6F627E70646F4E707
:104F10003A4A1268D50702D594F88C211AB143F0A9
:104F200001038AF80030364BB4F82C111B78354A4F
:104F300018075EBF9AF8003023F001038AF80030AA
:104F4000314B19B131490968890706D430490988BC
:104F500019B930480088642811D9022119701378D2
:104F600023F00103137005F0FDFA2B4B1B68C01AE8
:104F700000283EDB07B0BDE8F04F04F07DBC12789E
:104F8000D20756BF022219701A70ECE701200138CF
:104F9000C0B204F0FFFDFFF710BB0220F7E7562B6D
:104FA00001D104F00BFE98F80030002B3FF4DEAB8B
:104FB00094F825316F2B7FF4D9AB04F04BFDFFF74C
:104FC000FCBA022A4FF4FA737FF4ABAE9845A8BF3F
:104FD00000230198B8BFA3EB08034343BB80009BA9
:104FE0008B42BFF6A9AE37F80E305B4227F80E3081
:104FF0009FE607B0BDE8F08F0AD7233C181C0020BD
:105000003426002028260020CC1A0020AC250020C1
:10501000F40F0020EC0F0020D01A002090F825207B
:10502000034602F0FF0012B1002283F825207047EA
:1050300013B5036B04466A46062190F8440098476E
:10504000C0B101209DF800209DF8013043EA022301
:105050001BB2A3839DF802209DF8033043EA02238C
:105060001BB2E3839DF804209DF8053043EA022338
:105070001BB2238402B010BD13B5436904466A46CF
:1050800006213B209847A0B19DF800209DF80130F3
:1050900043EA022363819DF802209DF8033043EA2E
:1050A0000223A3819DF804209DF8053043EA0223E2
:1050B000E38102B010BD034601225A7453F8043C48
:1050C000143803B118477047026D70B5158804464F
:1050D000ADB2A90606D5036B23B9C36AA3B1908804
:1050E00080B298472B0620D5636AA26A9A42236D44
:1050F00017D0511CA069A162825C9A8023699942F1
:1051000013D30023A36270BDE169928840694E1CED
:10511000D2B2E6614254E169E268914228BFE3619C
:10512000E0E7DA6822F08002DA6070BD0C234343C6
:105130009B4AF0B5D35800019C8A9A4AA4B2E1B2C6
:1051400011F0010F48D0198821F400610904090CFD
:105150001980198889B241F4806119800021117089
:1051600011188C7A6CB392F8344014B9C979FF29BC
:1051700027D1012182F834101118097A022901BFC0
:10518000198889B241F4006119801118897941F0B8
:10519000010119821118097A92F9004001318C42FB
:1051A0000ED1002182F8341092F8351029B1998877
:1051B00021F440710904090C9980002302445371C1
:1051C000F0BD1418A17901F0FE011982E179FF29DF
:1051D000E0D0FF211170DDE78E0745D5BFF35F8F6B
:1051E00011180C7AE4B2012C1AD1897AC1B192F863
:1051F0003410A9B1198821F480610904090C1980BF
:10520000BFF35F8F198B198882F8354089B241F45A
:1052100000711980998889B241F480619980B9E759
:10522000198BBFF35F8F11180C7A022C10D1897A79
:1052300071B192F8341059B1198821F480610904D0
:10524000090C1980998821F480610904090CE5E7AB
:1052500011180C7A032CDDD1897A0029DAD092F862
:1052600034100029D6D0EDE74D0756D5012182F83C
:10527000351011188C7A002C38D092F83440002C5C
:1052800034D00C7A0D69022C198892F900401DD98E
:1052900021F480610904090C19801E8AE1B2F6B27A
:1052A0002E551C88A4B244F400741C808C1C14700D
:1052B0001C8A013149B2E4B26C54998889B241F434
:1052C000806199801988CF05FCD463E789B241F4E5
:1052D000007119801E8AE1B2F6B22E551E8A4C1C4E
:1052E00064B2F6B22E5503311170EBE792F8341028
:1052F00011B91118497A39B1198889B241F400718C
:10530000198011780131EFE7198889B241F4807171
:105310001980012182F83410D4E711F040011ED029
:1053200092F900E0198A17183E69C9B25FFA8EF542
:1053300006F80E106C1C64B23E7AE11C8E421470AA
:1053400005D1998821F480610904090C998011180C
:10535000097A8C427FF41EAF023515701AE72606D3
:105360007FF518AF92F90040651C0BD01518EE6858
:10537000611C345D49B21C822C7A11708C427FF41E
:1053800009AF5FE711701118CC791C828C7A002C60
:105390007FF458AF097A00297FF4FCAE52E700BFD2
:1053A000C8950108DC0B0020F8B507460E46094CED
:1053B000094D206809F041FF3946284609F08FFF62
:1053C0003146284609F08BFF206809F03BFF012099
:1053D000F8BD00BFDC06002000300140022210B4FE
:1053E000047B0168A24043694A6041680A6822F070
:1053F00001021204120C0A60596A9A6A914203D09F
:10540000184610BC0BF0ACBD012210BC83F8442040
:105410007047014858E600BF28360020004853E690
:10542000D43500202DE9F04300234FF00F0E012664
:105430000F8847FA03F2D20723D58C784FEAD308B6
:1054400014F0100F18BF91F8039003F0070504F053
:105450000F024FEA850550F828C018BF42EA09023A
:105460000EFA05F92CEA090CAA4042EA0C02282C93
:1054700040F828200AD1C26806FA03F422EA04029E
:10548000C2600133102BD4D1BDE8F083482CF8D191
:10549000C46806FA03F22243F2E70348D0F8B030BA
:1054A0000BB1A83018477047880200200348D0F895
:1054B00094300BB18C301847704700BF8802002031
:1054C0000248836F0BB17030184770478802002084
:1054D0000248C36D0BB15430184770478802002052
:1054E0000248036C0BB1383018477047880200201F
:1054F0000248436A0BB11C301847704788020020ED
:105500000248836803B11847704700BF8802002033
:105510002DE9F0470C244443814E86B006EB040A83
:1055200080469AF8040009F03BFE05469AF805000B
:1055300009F036FE4FF016091522074608F101035F
:10554000DBB2AA71EB7180F80690C3719AF806007D
:105550000BF030FE34592846A3884FF0640A23F438
:1055600040731B041B0CA38009F06CFE384609F045
:1055700069FE4946284609F035FE4946384609F095
:1055800031FE4FF00809284609F06BFE18B9BAF150
:10559000000F40F0B480284609F04FFE0A2005F0C5
:1055A00029F8284609F04EFE0A2005F023F8B9F143
:1055B0000109E8D1384609F040FE0A2005F01AF842
:1055C000284609F03AFE0A2005F014F8284609F0AA
:1055D00039FE0A2005F00EF8384609F033FE284659
:1055E0001F2109F0FFFD1F21384609F0FBFD4D4B3F
:1055F0004D4F9C4203F5DE331A6901A80BBF42F4FC
:10560000001242F480021A611A610BBF1A691A690A
:1056100022F4001222F480021A61A388434A23F480
:1056200040731B041B0CA3800C2303FB0866F37957
:10563000002B18BF1746238807EB47079BB243F0A0
:1056400001032380A58801F0D9FE039B384825F08B
:105650003F05B3FBF0F02D042D0C0543ADB2A58042
:1056600021884FF4967221F001010904090CB3FB63
:10567000F7F321804FF47A7142439BB2002B92FBE7
:10568000F1F208BF0123013292B243F400432284B5
:10569000A383238800259BB243F001032380238842
:1056A00001A823F4816323F002031B041B0C43F4C1
:1056B000806323804FF480432381238823F0800379
:1056C0001B041B0C23800124737A8DF805508DF880
:1056D00004308DF806508DF8074002F001F8337A57
:1056E0009DF807208DF804308DF805508DF8065090
:1056F0005AB101A801F0F4FF06B0BDE8F0870A2016
:1057000004F078FF0AF1FF3A3DE75A09094903F02E
:105710001F0304FA03F3203241F82230ECE700BF04
:10572000C895010800540040801A060000350C009E
:1057300040420F0000E100E00C23434337B5264A06
:105740000546D458A38A9BB20193019B13F4706F52
:105750001FBF0122214B03EB00131A71019B13F4AD
:10576000E06F1FD0238BA38823F480631B041B0CE2
:10577000A380019B9A0515D423889B0512D4238806
:10578000D8051CD52388D905FCD423889BB243F4C3
:105790000073238023889A05FCD46B1C02D0284612
:1057A000FFF7B6FEA38A23F470631B041B0CA382CD
:1057B0000A4B03EB051500236B7103B030BD238842
:1057C0009BB243F400732380A38823F440731B042B
:1057D0001B0CA380E6E700BFC8950108DC0B002086
:1057E00013B502AA02F8011DD0211D4B9975D87579
:1057F00001210020DA611A621A4A597698761976E0
:105800005975187591888C051FD41188C80516D450
:105810004FF48054118889050CD5013CFAD1124A05
:105820000120138801339BB21380FFF771FE2046DD
:1058300002B010BD118889B241F48071118009490C
:105840008A8892B242F440728A804FF480545A7D22
:1058500012B1013CFBD1E2E71C7D84F00104E6E7D4
:10586000DC0B002000580040201C002010B5D02484
:105870001C4B9C75D875012400201A62DA611A4A03
:1058800058769C7619765C75187591888C051ED4AF
:105890001188C80515D44FF48054118889050BD59B
:1058A000013CFAD1114A0120138801339BB21380C5
:1058B000FFF72EFE204610BD118889B241F4807199
:1058C000118009498A8892B242F440728A804FF46A
:1058D00080545A7D12B1013CFBD1E3E71C7D84F07A
:1058E0000104E7E7DC0B002000580040201C0020EA
:1058F00001201BE401201FE7002017E400201BE724
:105900002DE9F04F85B0804609F058FECE4B1E7849
:10591000002E40F04584CD4D2B685C0540F140845D
:10592000CB4CCC4F637A002B00F040813A68E3689F
:10593000D31A7C2B40F23A814FF02409C64BDFF892
:1059400044A3B3F8EE30E2600093237CAAF12C0B61
:1059500001332374484609F017FE5AF8040F0EF07D
:10596000ADFA0190BBF808000EF0A8FA019A0146C2
:1059700010460EF0ABFBB9490EF0F4FA0EF0CEFC77
:1059800009F1010900B25FFA89F909F0EBFDB9F1FB
:10599000270FDFD1302009F0F7FD002009F0E2FDEC
:1059A00009F0EAFD94F8109019F0030923D141F2AF
:1059B0008833E2689A420BD9102009F0E5FD484689
:1059C00009F0D0FD212009F0DFFD484609F0CAFDAD
:1059D000142009F0D9FDA24BB3F904000A2390FB6F
:1059E000F3F009F0BFFD1C2009F0CEFD002009F006
:1059F000B9FD09F0C1FD237C580740F0AF800220BB
:105A000009F0C2FD0A23B4F9120090FBF3F009F08B
:105A1000A9FD032009F0B8FD924B1B78590740F10E
:105A20005C81009990480CF001FF0522B4F91A300E
:105A300093FBF2F39BB220B92A6812F0100F18BF43
:105A4000002318B209F08EFD2B68884A1A4253D001
:105A5000DFF834B29BF80020002A4DD04FF06409E3
:105A6000DFF818A20620BAF8003009FB0323520021
:105A7000B3FBF2F3B4F81C904FEA09191FFA89F945
:105A800049EA03291FFA89F9C3F3032349EA030901
:105A900009F07AFD0FFA89F009F064FDA38B9BF8F9
:105AA000002001339BB293FBF2F102FB1133216A18
:105AB000A3838B7B012B40F01881392009F064FD12
:105AC000BAF9000009F04EFD282009F05DFD0A2317
:105AD000606A90FBF3F000B209F044FD042009F085
:105AE00053FD634B1B68DB89002B00F0248102F01F
:105AF00077F800B209F036FD02A95E4809F008FD0A
:105B0000132009F041FDBDF9080009F02BFD1B2011
:105B100009F03AFDBDF90A0009F024FD232009F03F
:105B200033FD4E2009F01EFD02A9524809F0F0FC99
:105B3000122009F029FDBDF9080009F013FD1A2013
:105B400009F022FDBDF90A0009F00CFD222009F040
:105B50001BFD452009F006FD09F00EFD237C282BD6
:105B600024D100231720D7F80090237409F00CFDEE
:105B70004EF660204FF03C0AB9FBF0F3B3FBFAF0AD
:105B80000AFB1030000200B209F0ECFC182009F00A
:105B9000FBFC4FF47A70B9FBF0F9B9FBFAF00AFBA1
:105BA000109000B209F0DEFC09F0E6FC94F8283011
:105BB000002B79D0E36A304AA8EB030393423CD927
:105BC000002384F8323084F834302C4B1B88DAB24E
:105BD0001B0A84F84E2084F84F3084F8442084F85F
:105BE00045303A68E36DD21A236E197C4FF47A730C
:105BF0004B439A420DD33B68E36502F045F8013808
:105C0000C0B201289FBF102384F83230022384F8E9
:105C100034300A211A4B626A1B6892FBF1F293FB43
:105C2000F1F384F84C2084F8503012121B1284F8DF
:105C30004D2084F85130C4F82C8094F864A0BAF157
:105C4000000F00F0738421E0681D00200017002081
:105C50003C0C0020083500201830002000007A4459
:105C60002A260020282600206C320020020000088E
:105C7000F0140020809698003F0D0300F8140020D7
:105C8000F4140020DC250020EC140020206F58B113
:105C900094F86430002B7AD040F6B732A36FA8EBAB
:105CA0000303934200F28A8094F88230D7F8009080
:105CB000002B00F0D981D4F88430002B00F0D4817F
:105CC00094F88830013B012B00F2CE81DFF81C8371
:105CD0004FF0010B4FF0000AB5E0BF4B1B68D889AD
:105CE0000523B0FBF3F000B2ACE66E23BAF8000077
:105CF000C97B4343152093FBF0F311B19BB293FB97
:105D0000F2F34FF0640B1FFA83F93A2009F03CFCE0
:105D1000B9FBFBFA0FFA8AF009F024FC3B2009F0EA
:105D200033FC0BFB1A904FF00A0980B2053090FB50
:105D3000F9F000B2C6E6A94B186880F31000D8E667
:105D400099F8003023B1C4F8688089F800A09DE775
:105D5000A36EA8EB0303B3F57A6F97D30123E06E2C
:105D600089F800300BF024FF8146E06E0BF020FF35
:105D700019F07F0F8AD18E2888D194F86430002BD7
:105D800084D1974B23672D2384F874307EE7012359
:105D900084F86430E36F9B78022B0AD8E06E02210E
:105DA000043009F091FB002384F88030C4F8788037
:105DB0007AE70221E06E0BF0F5FEF4E794F8743018
:105DC0009BB9236784F86430E36F9B78022B07D874
:105DD000E06E0121043009F077FB09F08BFBE5E769
:105DE0000121E06E0BF0DEFEF7E7013BDBB284F849
:105DF000743094F8801094F881204BB94B1C013218
:105E000084F8803084F88120E06E08F0EFFFCDE761
:105E1000034613F801EB01320EEB010084F8800019
:105E2000236784F881207146EEE7D4F884000BF0F4
:105E3000BFFE83B27E2B3A6822D184F889A084F811
:105E40008AA088F801A0D4F884000BF0B7FE0146C0
:105E50000028EAD194F88F30002B00F0918063780D
:105E600084F88F00302B40F08B80A3784FEA531ECC
:105E7000BEF1010F4AD084F8900009F0DDFA7FE00E
:105E800098F80120002ADED194F8891089B91B2BDB
:105E900007D1D4F884000BF091FE40BB84F88AB09F
:105EA000D1E70D2B23D184F889B02370A4F88C108E
:105EB000C9E77D2B02D184F88EB0C4E794F88EE058
:105EC000BEF1000F04D080F02000C3B284F88E2011
:105ED0004A1CD2B2092A84F8892063540AD1B4F842
:105EE0008C20C2F1FF02934201D184F88FB088F870
:105EF00001B0A8E7082AA6D8B4F88C00034403EB45
:105F0000132303F0FF03A4F88C309CE703F00F0089
:105F100013F0100328D0334B94F803C02279A4F86F
:105F20009E10A4F89C2003EB0C0182EA0C02C4F83A
:105F30009430C4F8981084F8E02084F890E09B3BFB
:105F40004FF0000894F8E010DFF8A4C0D4F894E013
:105F5000D4F8982072451FD1B8F1000F2AD16345BB
:105F60002DD184F8E1000BE094F8902042B194F830
:105F7000E120013202F00F0282421ED084F89030FC
:105F80004FF00008DFF86CA094F88AE094F8F0B1C4
:105F900094F8F13100228DE113F8012B0EF1010884
:105FA0006345C4F8948081EA02018EF800204FF026
:105FB0000108CBD384F8E010D1E70B4BC0E71A7887
:105FC00094F8E0309A424FF0000284F8902013D009
:105FD000B4F99C10012050E7F0140020F4140020C4
:105FE0006C0C0020DC0C00203F0C00200D00002079
:105FF000440C0020E0950108B348D4F8943000F137
:106000005008C4F89830C4F8940000F5A87300F163
:1060100044010C38C4F8E830C4F8E480A4F8EC205B
:10602000A4F8EE20FAF774F80130434606D1D4F80C
:10603000E420511CC4F8E41002211170D4F8E420CB
:10604000C4F8E4300123C4F8E82084F8F03197E77D
:106050003968A1EB0901012940F2A5800AB184F851
:10606000F131002384F88A3094F80032002B00F0DC
:106070009780D4F80432002B00F092803D68D4F869
:106080000832EB1A632B40F28B800A27DFF8548228
:10609000412009F0B8F9B8F9020090FBF7F080B29E
:1060A00009F0A8F9B8F9000090FBF7F080B209F008
:1060B000A1F9B8F9040090FBF7F080B209F09AF961
:1060C00009F07DF994F80C32D80745D47F4B1B8832
:1060D000D90513D4DA0600F11F829F0600F11E8253
:1060E000580600F11D82190700F11C82DA0700F141
:1060F0001B8213F0020F0CBF01260326744B1F787E
:10610000744BC7F38007DB780BB147F002075320CD
:1061100009F079F9704B188800EB800000EB8000E3
:10612000800080B209F066F9002009F063F9FE20D2
:10613000B4F80E32584340F2FF3390FBF3F0C0B294
:1061400009F048F9002009F045F947EA8600C0B295
:1061500009F040F909F033F994F80C329BB94F205B
:1061600009F051F90BF00EF90BF00CF90BF00AF9EC
:10617000012009F02FF9594B187800F0010009F0BF
:1061800029F909F01CF90A2194F80C32C4F80852D4
:106190000133DBB2B3FBF1F201FB123384F80C32B2
:1061A00005B0BDE8F08FBBF1000F67D00AB184F8ED
:1061B000F131D4F8E4304A4A934294F8F2313BD1B9
:1061C000591C84F8F211B4F9EE1003F00F0343F0F8
:1061D00010030029B8BF43F020038DF80830D4F82D
:1061E000E8309B1A94F8EC208DF80930534084F87D
:1061F000F3310DF10A030021D4F8E8C094F8F3213B
:106200000DF10E05AB422AD2D4F8E400ACEB000E3F
:10621000BEF1000F1ADC09B184F8F32194F8F311F0
:106220005A1C19700023AA4225D302A9322009F072
:1062300019F94FF0000B1BE05A1C03F00F038DF807
:10624000083084F8F2210DF10903D4E7411CC4F8A9
:10625000E410017803F8011B4A400121D2E709B19B
:1062600084F8F321AB42D9D102A9322009F0FAF81F
:1062700084F8F0B1F5E602F8013BD4E73AF81300F0
:1062800010B95B464FF403600133B0F5826FDBB2A7
:106290004FF0010200F0E38073D8B0F5007F00F00A
:1062A000B28021D8B0F5807F00F0C380B0F5887F40
:1062B00000F0BF80BEF1000F7FF4CAAE002A3FF4A9
:1062C000D3AE84F8F131CFE6DC0C0020C63A0020D2
:1062D0002826002044180020F8140020342600202E
:1062E0002C0D00202A260020B0F5047F6DD0B0F5DB
:1062F000806FDFD184F8F13194F8F83142F21071F7
:106300000133DBB2032B88BF012384F8F83194F802
:10631000F83159438F4B1B78D80748BF01319A0792
:1063200048BF023158078C4B48BF04311B88DA073D
:1063300048BF0A31980748BF14311A0648BF2831B0
:10634000D80548BF28315A0748BF6431180748BFED
:10635000C8319A0548BF01F5C871980648BF01F5D4
:106360007A71DA0648BF01F5FA61580648BF01F5AF
:106370007A614FF4806009F08FF8784B83F88A8057
:1063800002E6B0F5E26F65D00FD8B0F5C06F46D029
:10639000B0F5E06F8ED1724A84F8F131116B64234D
:1063A0004B43118993FBF1F126E0B0F5046F49D01E
:1063B000B0F5116F00F0A080B0F5E46F7FF47AAF14
:1063C000674A84F8F131916BE9E784F8F1312B6881
:1063D0009A077FF5D9AD634B197800293FF4D4AD06
:1063E000D4F8F431604ADB7B5BB1138893FBF1F3A3
:1063F0000A214FF40470594309F04EF884F88A805A
:10640000C2E51388F4E784F8F1312B6813F0082F04
:106410003FF4BAAD0A23616A91FBF3F1ECE784F82B
:10642000F1312B6813F0082F3FF4AEAD4F4B1968D4
:10643000E2E784F8F1314E4B1B685B077FF5A4ADB2
:106440000021D9E70A2184F8F1314A4BB3F904302D
:106450005943D1E7424A84F8F131516B9FE784F800
:10646000F131434B1B6813F0200B7FF48DAD2B688B
:106470001A0605D5594609F00FF884F88AB083E565
:10648000D4F8F4315B7C002B3FF47EAD94F8F93105
:10649000032B2FD8DFE803F002192027364A1268B1
:1064A000107892F801E09178090401EB0E21014483
:1064B00001EB03610133DBB2042B14BF84F8F93123
:1064C00084F8F9814FF4826096E72B4A1268907A3B
:1064D00092F80BE0117BE7E7274A1268107D92F8EB
:1064E00015E0917DE0E7D4F8FC21507992F806E0C0
:1064F000D179D9E70021DBE784F8F1312B689B07DC
:106500007FF542AD174B197800293FF43DAD164B8E
:106510001A880A23534345E70D26EFE50926EDE5E2
:106520000426EBE50826E9E50226E7E5E06E0BF038
:1065300045FBC0B201287FF6A9AB0228DFF83C90EA
:106540003FF4FEAB08F0D6FF012389F80030FFF7D7
:106550009DBB00BF28260020C63A00203C0C00202E
:10656000B0250020EC140020F8140020F4140020C2
:10657000AC2500202A260020881E00200D000020C7
:106580002DE9F041884600240C4B93E8E0000544D7
:1065900006440744444501DBBDE8F08137F9142087
:1065A00036F9143035F914001344022293FBF2F348
:1065B000C01A09F0E1F90134ECE700BF500E0020E9
:1065C000F8B52F4B2F4E1C682F4B20601A6804F132
:1065D000300562605A689B68A260E3602B4B04F14F
:1065E00036071A6822615A689B686261A361284B6A
:1065F0001A68E2615A689B6822626362254B1A88B6
:1066000022855A8862859A88DB88A285E38556F8B8
:10661000040F10F02BFA25F8020BAF42F7D11E4BF6
:106620001E481A6BE2865A6B9B6B228763871C4B52
:106630001A88A2875A88E2879A88DB88A4F84020C3
:10664000A4F84230174B04F14402197800238B421E
:1066500010DB154B1B88A4F86C30144B1B68A4F896
:106660006E30134B1B88A4F87030124B5B89A4F872
:106670006630F8BD30F91350013322F8025BE6E7CB
:10668000500E0020401000201C0800202808002088
:1066900034080020500C0020B02500206425002084
:1066A000CE1E00205C250020AC1E0020FC14002023
:1066B0004A0E0020AC05002010B5104B014693F89F
:1066C000C934012B13D10E4A0E4C1078431CDBB297
:1066D00013701B0648BF0023215448BF137008F0F5
:1066E00097F83F2809D9BDE8104008F09BB9064B40
:1066F000BDE81040186808F079BB10BD18300020C4
:106700006C1D00204D210020840700207FB5244C03
:10671000244E254D2549264A264B20B1264800887F
:10672000B0F5805F30D2306891F820101278019077
:106730002878224D1B788DF808008DF809108DF807
:106740000A202946082201A88DF80B3012F030FCEF
:10675000C0B101AB03CBE06069605320FFF7ACFF31
:10676000E06809F0F9F8207C09F0F6F8637C01A8EC
:106770000193A37C0293E37C039309F05DF800226C
:106780000D4B1A8004B070BD306891F82010E060A5
:10679000127828781B7820746174A274E374DCE7A3
:1067A000500E0020181C0020342600204418002021
:1067B000F51600201E0B0020A20700205C0E002012
:1067C0000B4A1388013313800A4A1368013313609C
:1067D000094A138801339BB2202B03BF0023138087
:1067E000064A138002BF938A01339382704700BF29
:1067F000A2070020A8070020A4070020500E0020B8
:1068000038B5234B05461B780C46093B012B3ED877
:106810004520FFF751FF2846FFF74EFF0E2D0ED003
:1068200003D83DB10D2D0FD038BD1E2D07D0FF2D43
:1068300028D038BD2068BDE8384009F08DB8206800
:1068400009F08AF86068F6E7637820789BB180F0F9
:106850008000FFF731FFA468E0B2FFF72DFFC4F31B
:106860000720FFF729FFC4F30740FFF725FF200E9D
:10687000BDE8384020E7FFF71FFF6068BDE83840FB
:1068800009F07AB8034809F088F80020F0E738BD2D
:10689000DC05002020B801082DE9F04F5C4E0546CC
:1068A00030888BB0DFF890815A4C002840F0C680C9
:1068B00098F8C734012B05D198F8C804A0F120013D
:1068C00048424841FFF722FF2846FFF779FE256836
:1068D00049202E46FFF7F0FE4F4BDFF858A118680D
:1068E00009F03AF856F8040B09F036F830460AF089
:1068F000BDFC05F110000AF0B9FC10274FF0010BA8
:10690000564605F11C09DAF800200BFA07F313428A
:1069100003D0D9F8000009F02FF80137132F09F13F
:106920000409F0D1032105F1280009F029F8B8F88D
:10693000CC30B5F92E00C01A09F00EF83368DA042D
:1069400008D5364B1888B5F86C30C01AC0F30D0066
:1069500009F002F833689B0403D5B5F86E0008F01F
:10696000FBFF33681F0403D5B5F8700008F0F4FF8F
:106970000127032105F1300009F002F8032105F198
:10698000360008F0FDFF042105F13C0008F0F8FF97
:10699000234BB5F944001B8805F14609C01A08F0DD
:1069A000DBFF204B93F800A0BA4527DC336898053D
:1069B00005D5B5F96600A0F2DC5008F0DDFF2268CD
:1069C0006260A2601849194B521A92105343032275
:1069D000013393FBF2F202EB42029B1A742202FB98
:1069E000031301222360124B1A7098F8C934012B4B
:1069F00001D108F017F80BB0BDE8F08F39F9020BA0
:106A0000B5F944300137C01A08F0B6FFCCE700BF33
:106A1000A4070020500E0020A8070020A007002097
:106A20009A0700205C250020680E002035C2724FB6
:106A3000480A00209C07002018300020B94BD4F8E9
:106A400074211B689A4207D00AA941F8203D002012
:106A5000C4F87431FFF7D4FEB34BD4F878211B6827
:106A6000934208D00AA941F8203D1E200392C4F8A1
:106A70007831FFF7C5FE98F8C714338898F8C80432
:106A80000B44013BB3FBF0F200FB12339942ACD94B
:106A90000120FFF73BFE2846FFF792FD50202768B4
:106AA0006668FFF709FEA268236810681B686268C1
:106AB000034410683D1DA3EB400008F05DFF002378
:106AC000301D50F8231055F82320521A02A941F81E
:106AD00023200133032BF4D1002508460AF0C6FB1E
:106AE00007F1100006F1100151F8252050F825306B
:106AF0009B1A02AA42F825300135032DF4D1104625
:106B000008F09AFE4FF010090121884A07F11C0B8A
:106B100006F11C0A136801FA09F018420AD0DBF8E2
:106B20000000DAF800308DE80600C01A08F024FFF3
:106B30009DE8060009F10109B9F1130F0BF1040BEF
:106B40000AF1040AE6D1002307F1280006F1280122
:106B500031F902EB30F9022BA2EB0E020DF1080E17
:106B60004EF823200133042BF2D14FF0000B02AB7F
:106B700053F825304FEA8B0B5FFA8BFB2BB103F1F7
:106B800008020F2A54D84BF0010B15F1FF35EED255
:106B900000255846FFF790FDA9460DF1080A0BF0B5
:106BA0000302022A56D0032A68D0012A07D1B9F17C
:106BB000000F45D19146DAF800502D01EDB20AF1EF
:106BC000040A06AB53454FEA9B0BE8D1B9F1000F1D
:106BD00002D02846FFF770FD544B1B6813F4805514
:106BE00006D00125B7F86C20B6F86C10521A029244
:106BF00099040AD50AAA02EB8501B6F86E00B7F827
:106C00006E200135121A41F8202C1A044AD50AAB1D
:106C100003EB8502B6F87010B7F8703001355B1AD7
:106C200042F8203C012D60D1029808F0A5FE3BE01F
:106C30008033FF2B94BF4BF0020B4BF0030BA4E708
:106C4000DAF800004FF0000900F00F002843FFF7CA
:106C500033FDB4E7B9F1000F04D19AF80000FFF753
:106C60002BFDACE7DAF80000C0F303102843FFF770
:106C700023FDDAF800502D01EDB2A0E7B9F1000FC5
:106C800004D19AF80100FFF717FDE6E7DAF80000F3
:106C9000C0F303302843FFF70FFDDAF80000C0F31C
:106CA0000710E4E7002DBDD103213020FFF768FC79
:106CB00003213620FFF764FC04213C20FFF760FC31
:106CC0001B4B44201978FFF75BFC184B1B689B0596
:106CD00006D5B7F96600B6F96630C01A08F04CFE62
:106CE00063682268A36062606CE600206B1E02AAE3
:106CF00052F823204000C0B20AB140F0010013F165
:106D0000FF33F4D2FFF7D8FC4FF0000902AB53F881
:106D1000290008B108F030FE09F10109A945F5DBA9
:106D2000C2E700BF1C1C0020181C00209C0700208C
:106D30005C2500202DE9F74FA3EB020B17460E9BB5
:106D40000D9A4C4C9B1A00936368002914BF0626C9
:106D5000042601330546894626D123689E4240F227
:106D60008680DFF82CA15AF823000CF043FB0B308F
:106D700008F020FD804618B1012003B0BDE8F08F77
:106D800021683D485AF82120032994BF29464946E5
:106D900008F098FE394A1368181A636810600133C6
:106DA0006360374B83F87C81DFF8D090DFF8D0A0A8
:106DB00065680C9B9D4217DB10D1012008F0FAFC9E
:106DC00060B92E4A0A201368013B1360FFF774FC78
:106DD0002368013323604FF0FF33636020688642ED
:106DE00094BF00200120C8E70D9B4BB1009B0D9A7A
:106DF0006B43D25C01239340224A1268134227D08E
:106E000005FB0BF5236807EB05082BBB78590CF045
:106E1000F1FA431D1846019308F0CCFC0028ABD1D1
:106E2000D9F80000019BC01A9AF87C31C9F800001B
:106E3000A3B12C20FFF740FC23689BB9785908F0D8
:106E4000ACFD98F904104B1C02D00F4808F03AFE34
:106E5000636801336360ABE70323DBE701238AF850
:106E60007C31E9E7984498F804100848EEE70020E0
:106E700083E700BF900700202BB801088807002097
:106E8000500E00209C0700203AB8010874CF01087A
:106E90000896010810B50B4C21780B290BD801235B
:106EA0008B4040F6030119400BD113F4C06F02D0A0
:106EB000FF20FFF7A5FC044B1A68044B5A600B2314
:106EC000237010BDDC05002008350020900700204D
:106ED0002DE9F04F874E85B03378012B1CD1864CBD
:106EE00094F8C72422B194F8C8340BB19A4216D34F
:106EF000012384F8C73484F8C83494F8C934012BCA
:106F000084BF002384F8C93494F8C954C5B1012D55
:106F100000F09D800023337005B0BDE8F08F184667
:106F2000114630B191FBF0F500FB151501462846DE
:106F3000F7E792FBF1F293FBF1F384F8C724DAE769
:106F4000802004F039FA07460028E3D0802104F0BD
:106F500005FA6A4B7A791870694B97F9020053F871
:106F600022308021B3F5613F0CBF02220022019242
:106F7000022200922A4604F007F94FF4FA72614B9C
:106F80001860614B1B6803EB4303B3FBF2F3002B68
:106F90005BD0402BA8BF40235C4A13700028B9D0B7
:106FA0005B4D1422002105F5C07012F035F82B4618
:106FB000002005F1180243F88C2B6B6005F58073F7
:106FC000AB60544B94F8C7741A88534B53491A80DA
:106FD000534B94F8C8241860524B97421B6894F89E
:106FE000B3220978039302914F4BA2F119012CBFF0
:106FF00000270127D1F1000E1B684EEB010E012A7C
:1070000094F8672203F4006CC3F3400A08BF4FF002
:10701000010EC3F3C033824294F844920CBF9846E9
:107020004FF00108012104464A1ED2B2531E132B11
:1070300026D8DFE803F01F1F1F1F1F1F1F1F1A2A5C
:107040002A5B4D2A5D464646592A0123A4E7374B61
:10705000DB68002B3FF45EAF08F0D8FB00287FF41C
:1070600059AF4022294B1A709AE7734643B9013150
:10707000C9B2D9E7029B9A42CCBF0023012323B1B6
:107080000123184603FA02F214431429EFD908B178
:10709000234B1C6019200AF0F6F8254B254A18707E
:1070A00000231360244AAB821380244A1268C5F877
:1070B0007421234A1268C5F87821224A13700223EA
:1070C00029E7039B13441B79003318BF0123D6E73C
:1070D000BCF1000F06D009F1FF3BDBF1000343EBED
:1070E0000B03C3E76346C1E73B46BFE75346BDE733
:1070F0004346BBE7DC05002018300020AE07002027
:107100007CA5010884070020DC2200208C070020D9
:10711000500E0020AC1E0020A00700205C2500209F
:107120009C070020881E0020001700207802002005
:10713000AC070020A8070020A40700201C1C00208A
:10714000181C0020480A002010B5204B18B9022254
:107150001B681A8210BD00201D491C680880237816
:107160000A4613F07F0313D1637A990644BF0221C4
:10717000117013F0400F137814BF43F0010323F094
:1071800001031370134B1B681B699847104810BD0F
:10719000012B18D0022B17D1617901F00F039B004E
:1071A00003F1804303F5B84311F0800F1B6805D04D
:1071B00003F03003102BE5D10123E2E703F4405341
:1071C000B3F5805FF7E7084610BD00BF282B00200D
:1071D000E40F0020981E002010B5064C18B90122BB
:1071E00023681A8210BD044B1B689B68984720686F
:1071F0000C3010BD282B0020981E002010B5064C26
:1072000018B9012223681A8210BD044B1B681B6841
:10721000984720680A3010BD282B0020981E0020B7
:10722000084BDA68D10709D4DA68520708D4DB685A
:1072300013F0100F14BF0320042070470120704783
:107240000220704700200240064B596841B1642279
:10725000D8684243B2FBF1F21A8100225A60DA6028
:10726000704700BFE40F00200E4B0F4A1B683E29F9
:107270009BB223F0070303EBC00002444FEA420233
:107280000AD94B09C80604BF03F1FF339BB29B0226
:1072900043F40043136070474B08C90748BF0133EC
:1072A0009B02F7E7505C004006300020054B1B684E
:1072B0009BB223F0070303EBC000034B03445B00C6
:1072C00019607047505C0040023000208B6810B598
:1072D0000C6A026823430C6922F4FF4223434C6981
:1072E00022F0700223438C692343CC6923434C6A08
:1072F00023438C6A234313430360CB6843600B68CA
:1073000083604B68C36010BD036823F001031B0456
:107310001B0C03600023036043608360C360294B40
:10732000984204D1284A536843F00F0326E0274BC4
:10733000984204D1244A536843F0F0031EE0244BE2
:10734000984204D1204A536843F4706316E0214BFD
:10735000984204D11C4A536843F470430EE01E4B1C
:10736000984204D1184A536843F4702306E01B4B3B
:10737000984205D1144A536843F470035360704730
:10738000174B984204D1104A536843F07063F5E7F5
:10739000144B984201D1144AC5E7144B984201D1CD
:1073A000114AC8E7124B984201D10F4ACBE7114B63
:1073B000984201D10C4ACEE70F4B9842DFD10A4ADE
:1073C000D1E700BF08000240000002401C0002405C
:1073D0003000024044000240580002406C0002406D
:1073E0008000024008040240000402401C040240E5
:1073F0003004024044040240580402401F4A10B5C1
:10740000536803F00C03042B21D0082B22D01C4B13
:10741000036053681B49C3F30313CC5C0368E34068
:1074200043605468C4F302240C5D23FA04F48460BE
:107430005468C4F3C2240C5DE340C3605268C2F3D5
:10744000813211440A7CB3FBF2F3036110BD0E4B91
:107450001B68DDE753685168C3F38343C90303F135
:10746000020302D409494B43D2E7516811F4003FAB
:107470000549096818BF4908F5E700BF0010024038
:1074800000127A00209601081000002000093D003B
:1074900010B50446FFF7C4FE012806D10CB905203B
:1074A00010BDFFF7BDFE013CF6E7002C08BF05202C
:1074B00010BD0B88F0B54E88B1F804E00F89CC8878
:1074C000002B3CD1038C23F001031B041B0C038411
:1074D000018B824B89B221F0F301058C4EEA010148
:1074E00041EA07119842ADB289B212D003F50063A8
:1074F00098420ED0B0F1804F0BD0A3F5983398424C
:1075000007D003F58063984203D003F58063984267
:1075100012D125F0020546EA050343F00103018379
:107520000384038B23F00C031B041B0C0383038BCA
:107530009BB21C430483F0BD25F00A05EBE7042B46
:1075400044D1038C4FEA0E2E23F010031B041B0CB6
:107550000384038B4EEA073723F440731B051B0D8E
:107560001F435E4B018C984289B2BFB212D003F523
:10757000006398420ED0B0F1804F0BD0A3F5983342
:10758000984207D003F58063984203D003F58063E7
:10759000984214D121F0200141F0100343EA061370
:1075A0009BB207830384038B23F440631B041B0CEF
:1075B0000383038B9BB243EA0424A4B2BAE721F00D
:1075C000A00146EA010343F01003EAE7082B038C0D
:1075D0003FD123F480731B041B0C0384818B3F4B2E
:1075E00089B221F0F301028C4EEA010141EA071150
:1075F000984292B289B212D003F5006398420ED03D
:10760000B0F1804F0BD0A3F59833984207D003F523
:107610008063984203D003F58063984213D122F42B
:10762000007343F4807343EA06239BB2818303848F
:10763000838B23F00C031B041B0C8383838B9BB273
:107640001C438483F0BD22F42063334343F48073EE
:10765000ECE740F6FF4223F480531B041B0C038429
:10766000818B038C0A40390341EA0E2111431B4AE6
:107670009BB290421FFA81FE12D002F50062904246
:107680000ED0B0F1804F0BD0A2F59832904207D0C7
:1076900002F58062904203D002F58062904215D1DB
:1076A00023F4005343F4805343EA06339BB2A0F81B
:1076B0001CE00384838B23F440631B041B0C838333
:1076C000838B9BB243EA0424A4B2BAE723F4007389
:1076D0005B045B0C334343F48053E8E7002C014028
:1076E0000F4BDA684378D243C2F30222C2F104019D
:1076F0008B400F2121FA02F281780A401343094995
:1077000002781B018818DBB280F80033012350098E
:1077100002F01F0203FA02F241F82020704700BF76
:1077200000ED00E000E100E02DE9F041CB780E88AB
:10773000DA0648BF8A7803F00F0548BF154316F0F4
:10774000FF0F1AD000214FF0010E4FF00F0C02680E
:107750000EFA01F737EA06040BD18C000CFA04F894
:1077600022EA080205FA04F4282B42EA040225D191
:10777000476101310829EBD10260FF2E1CD900219D
:107780004FF0010E4FF00F0C426801F108040EFAA1
:1077900004F434EA06070BD18F000CFA07F822EA4A
:1077A000080205FA07F7282B42EA07020AD14461CA
:1077B00001310829E9D14260BDE8F081482B08BFBA
:1077C0000761D6E7482B08BF0461F1E70F4B1A6841
:1077D00042F001021A6059680D4A0A405A601A685C
:1077E00022F0847222F480321A601A6822F4802215
:1077F0001A605A6822F4FE025A604FF41F029A601F
:107800004FF00062034B9A60704700BF00100240C7
:107810000000FFF800ED00E080F3088870474FF4A7
:107820007A73054AD16DB3FBF1F3C3EB431103EB5C
:107830008103DB0013827047E40F00202DE9F74F2E
:10784000684B694CE36623676367E06D0CF032FBBD
:107850000146054665480CF039FC0CF085FDA36F28
:1078600007465E795EB9A36F1889002873D1A36FAC
:107870009889002840F0928003B0BDE8F08FB042B4
:10788000F1D31B79012B19D100254FF01C0A584B5D
:1078900004F17C09E36604F1D0080AFB0596A36FA6
:1078A00048F8256058790CF005FB01350146E26D7A
:1078B00030460BF081FC032DEFD1D4E7002B35D1FE
:1078C0004C4B4D49E36628460CF04CFB05463046D0
:1078D0000CF0F4FA014649480CF0F8FB0646014664
:1078E00028460CF037FA014628460CF0EFFB04F16D
:1078F000DC03C4F8D03004F1EC03C4F8D43004F154
:10790000FC03C4F8E460C4F8E850C4F8E000C4F82C
:10791000F460C4F8F850C4F8F000C4F8D830C4F8E3
:107920000461C4F80851C4F800019CE70025344BF9
:1079300004F58678E36604F1D00608EB0520A36F12
:1079400046F82500B4F85C20597901350BF098FB16
:10795000032DF2D187E7874289D3254A59892267C7
:107960000BF036FC002581464FF01C0BDFF89880A9
:1079700008F1540A0BFB0586A36F4AF825601889A5
:107980000CF098FA012301460093E26D4B46304615
:1079900001350BF093FB032DECD168E78742FFF430
:1079A0006BAF134AD98962670BF012FC0025804641
:1079B0004FF01C0A134F07F154090AFB0576A36F19
:1079C00049F8256098890CF075FA01230146009367
:1079D000E26D4346304601350BF070FB032DECD1D0
:1079E0004AE700BFBF2D0108E40F00200024F4483F
:1079F000492D0108A12D0108BD37863583F9223EA6
:107A0000E52C010850140020F013002002392DE964
:107A1000F843426804460368806806290DD8DFE809
:107A200001F0040873767B7E810022605B42636014
:107A300003E05B425242236062603C4B1B79002BA7
:107A400060D120680CF03AFA804660680CF036FA93
:107A50000746A0680CF032FA354D0646D5F8CC142E
:107A600040460CF07FFAD5F8D814814638460CF021
:107A700079FA014648460CF06DF9D5F8E4148146D0
:107A800030460CF06FFA014648460CF063F90EF0F0
:107A9000EDFFD5F8D014206040460CF063FAD5F81D
:107AA000DC14814638460CF05DFA014648460CF07D
:107AB00051F9D5F8E814814630460CF053FA0146E6
:107AC00048460CF047F90EF0D1FFD5F8D4146060A9
:107AD00040460CF047FAD5F8E014804638460CF0E2
:107AE00041FA014640460CF035F9D5F8EC1407464A
:107AF00030460CF037FA014638460CF02BF90EF000
:107B0000B5FFA060BDE8F883524222608FE75B4278
:107B100023604042A06090E722606360F9E7524230
:107B20006260F6E7524222605B42F6E710000020F6
:107B3000E40F00202DE9F84F90F8253006461BB9D8
:107B400000273846BDE8F88F436898470746002865
:107B5000F6D0002586F82550B38B1E4C1BB2C4F816
:107B6000F034F38B96F826101BB2C4F8F434338C3F
:107B700004F59E601BB2C4F8F834FFF747FF04F128
:107B80005C0808F2944904F2FC4A04F1D00B5AF85C
:107B9000253059F82500C01A49F825000CF08EF957
:107BA000B1690CF0DFF9E36E01465BF825009847F8
:107BB000094A0146236F52F825009847074A0146B3
:107BC000636F52F8250098470135032D48F8040FDC
:107BD000DDD1B6E7E40F002044140020A4140020F7
:107BE00070B51A4C94F8080510B3D4F80C15CD896B
:107BF000FDB128460CF05EF90646D4F810050CF0ED
:107C00005DF9014630460CF0A3F811490CF0AAF9D1
:107C1000044628460CF052F9014620460CF056FA6C
:107C20000CF07CFB6428A8BF642020EAE070C0B29E
:107C300070BD0D79B4F81435CA7800FB153464238F
:107C4000521B63435043B3FBF0F0EBE7E40F00201B
:107C50000000C84210B50A4CD4F8183558430CF04F
:107C60002DF908490CF07EF9D4F81C150CF072F8C7
:107C7000C4F81C050CF052FBC4F8100510BD00BF81
:107C8000E40F00202FE33E31054B93F82005032835
:107C900004D093F82135984238BF1846704700BF8A
:107CA000E40F002008B5FFF7EFFF012802D00228FB
:107CB00005D008BD0820BDE8084007F02FBF072009
:107CC000F9E738B50E4CD4F80C55AB7CB3B1EB8961
:107CD000A3B1FFF7D9FF032810D0FFF781FF28B920
:107CE000022384F82035BDE83840DBE7EB7C834293
:107CF0002CBF0123002384F82135F4E738BD00BFF1
:107D0000E40F002044F6FB71084BD3F80C251378E0
:107D100003EB431300FB03135078C0EB0030B3FBBD
:107D2000F0F09378B0FBF3F080B27047E40F0020DE
:107D30000B2870B511D009280ED83422144B02FB41
:107D4000003009B1C36863B90022124DD5F8284547
:107D500005F22C53A24208DB70BD0E4BD3F824056C
:107D6000EFE7BDE8704001F075BC53F822109600B3
:107D700088420AD1A21A311D920019449819013C77
:107D800011F030F9C5F8284570BD0132E2E700BFB7
:107D900018000020E40F0020F7B504780546A4B9C8
:107DA000334D344EB5F8A23232460193B5F8A032C5
:107DB000002100930120234601340AF087FB042CA4
:107DC00005F10405EED103B0F0BD2B4911F02CF9FB
:107DD000A8B94FF47A714FF4FA62254BA3F8A012B8
:107DE000A3F8A222A3F8A412A3F8A622A3F8A8122B
:107DF000A3F8AA22A3F8AC12A3F8AE22E3E7284620
:107E00000EF046FC0328044628D828460AF04FFA0C
:107E1000074660B10EF03CFC0125064638460AF0E4
:107E200046FA30B903B0BDE8F0400AF0F5BB0546AC
:107E3000F4E70EF02DFC002DF4D040F2DC53A6F256
:107E4000EE229A42EED8A0F2EE229A42EAD8084BED
:107E5000A63403EB84031E815881B4E70323002278
:107E60000649074803B0BDE8F0400AF077BA00BF02
:107E7000183000209FB80108B2B8010856C60108A2
:107E8000B8B801082DE9F14F05460027544E2B786C
:107E900033B90021012001B0BDE8F04F09F093BAD9
:107EA00005225049284611F0FAF848B900224C49F9
:107EB00043181030C028DA60FAD101B0BDE8F08F65
:107EC00004224949284611F0EAF804462846002CC5
:107ED0003FD10AF0ECF981460028EED00BF08AFA87
:107EE000DFF820A15FFA80FB5AF82480B8F1000F78
:107EF00005D13E4801B0BDE8F04F0AF073BB5A46C9
:107F00004146484611F0CBF8013405460028EBD134
:107F100003469A191033C02BD760FAD1344B03EBC8
:107F2000C402D2F804E0BEF1000F03D013F834C04D
:107F3000654505DB41462F480AF010FA2E4DA6E7AD
:107F40002B01F4180C3473440FCB013584E80F0077
:107F5000EEE70EF09DFB0B28064637D828460AF0C0
:107F6000A6F9054638B302F01BFF01241C4B03EBB6
:107F70000613D86028460AF09AF9054630B102F097
:107F80000FFF174B013403EB0613186128460AF064
:107F90008EF9054630B102F003FF114B013403EBBB
:107FA0000613586128460AF082F930B901B0BDE8DD
:107FB000F04F0AF031BB0446DCE702F0F1FE084B5B
:107FC000032C03EB0616B061F0D162E70B2300220D
:107FD0000A490B4801B0BDE8F04F0AF0BFB900BF35
:107FE00018300020B2B80108D3B80108D8B8010889
:107FF00034960108E7B8010858C40108F3B801082D
:10800000B8B8010844A10108F0B5057889B0064662
:1080100035BB19264A4C4B4F94F871343A460593B8
:1080200094F870340021049394F86F340120734362
:1080300003F56173039394F86E340634734303F5C8
:108040006173029394F86734019394F86C3400934D
:108050002B4601350AF03AFA0F2DDDD109B0F0BDFB
:108060000EF016FB0E28054662DC0624002344436E
:10807000701C8DF81F300AF01AF9314E074658B1BE
:108080000EF006FB032807D8331983F872049DF815
:108090001F3001338DF81F3038460AF008F90746C3
:1080A00068B10EF0F5FA0D2809D8062303FB056325
:1080B00083F86D049DF81F3001338DF81F3004F2F2
:1080C0006E410DF11F02314438460AF0FCF80AF007
:1080D000EEF8074668B10EF0DBFA172809D8062338
:1080E00003FB056383F870049DF81F3001338DF89E
:1080F0001F3038460AF0DBF868B10EF0C9FA0D28D7
:1081000009D8062303FB05659DF81F3085F8710427
:1081100001338DF81F309DF81F30062B9ED00023B1
:1081200004F26D443219335193800AF075FA95E7E1
:108130000E230022044905480AF010F98EE700BF1B
:1081400018300020F9B80108F3B80108B8B80108E0
:108150002DE9F74F037823B903B0BDE8F04F0AF0DB
:108160005BBA5C4900270EF0BBFA3C460546B846B0
:108170004FF0FF36DFF88891DFF888A1DFF888B18B
:10818000B5B90C27544B70B207FB05F2D118D25683
:10819000824200F081800135052DF5D1B8F1000F44
:1081A00035D131464D4803B0BDE8F04F02F06DBF08
:1081B000012F0DD0022F10D01FB928460EF068FAFB
:1081C0000646444900200EF08BFA01370546D7E7F2
:1081D00028460EF05DFA8046F3E74946284610F03F
:1081E000ACFF20B93E49284610F0A7FF08B144F083
:1081F00001045146284610F0A0FF28B959462846E8
:1082000010F09BFF0028DCD044F00204D9E7002CDA
:1082100008BF03240022E4B20192009443461146B1
:1082200002F0B2FF054610B931462E48BBE7424680
:1082300031462D4802F029FF31462C4802F025FF37
:108240002B4B1C68204602F07FFF284602F07CFF83
:10825000002008F0CDFF204609F0B0FC60B10120FD
:1082600008F0C6FF204609F0A3FC0146284606F0A8
:10827000BDFD002008F0BCFF284609F09FFC002847
:10828000E9D0012008F0B4FF284609F091FC01462E
:10829000204606F0ABFDDBE74D68002D3FF47EAFD6
:1082A0003146144802F0F1FE54B169798C4207D08E
:1082B0002246114802F0E9FEE1B2284609F072FCBC
:1082C000EB6A002BB8D00D4802F0DFFE0023EB6212
:1082D000B2E700BF46BA0108683500201FB901089F
:1082E000BDC1010847B9010866B90108D1B9010843
:1082F000401C002083B901089BB90108BBB90108E3
:1083000019B901081CB90108A4C301082DE9F341FA
:108310000178064629B9012002B0BDE8F04109F014
:10832000D5B80024009401940EF0B2F9334B013615
:108330001A68234640B202EBC30595F90210814248
:1083400005D00133052BF6D100252C4604E0002D85
:10835000FBD001248DF80200304609F0A8FF074643
:1083600028B10EF095F90134ADF80000E4B2002612
:10837000DFF88C80384609F09AFF074600B30EF00C
:1083800087F9002258F82210D3B2884203D0013274
:10839000102AF7D1002358F82320904210D1022E42
:1083A0001AD0032E1DD05A1E012ED2B20FD00B2A86
:1083B00003D88DF803300134E4B20136042ED9D14C
:1083C000052C14D802B0BDE8F0410AF025B9042A02
:1083D000F3D88DF80430EEE7052BEED88DF8063093
:1083E000E9E79A1E052AE8D88DF80530E3E76B46E1
:1083F00003CB2860696002B0BDE8F08164350020DD
:108400007CA501082DE9F04F81468A460D460027DC
:10841000644E91B096F8023196F90481099396F86A
:10842000033196F907B10A9396F805310B9396F943
:1084300006310C9396F808310D93B8F1000F41D135
:1084400059480AF0CFF800244FF00E08574FBAF100
:10845000000F00F09280002508FB04F30993099AAD
:10846000504B13440A930126099BAE405344D3F862
:108470007C210A9BD3F87C31534036EA030314BFB6
:108480004FF0010B4FF0000B324206D0009523460F
:108490003A465946484609F0F9FF0A9BD3F87C3121
:1084A000334206D0009523463A46594648460AF0DC
:1084B0000DF801350E2DD6D10134082CC7D111B0DD
:1084C000BDE8F08FBAF1000F55D095F8084195F846
:1084D00002310F94099C0E939C4295F8032195F963
:1084E000041195F8050195F906E195F907C140D108
:1084F0000A9C94423DD188453BD10B9C844238D1A3
:108500000C9C744535D1E34533D10D9C23460F9C1B
:108510001B1B5C425C410F9B039006930E9B0291D8
:1085200001920093CDF814C0CDF810E03B46204AEC
:108530002146484609F0AAFF0D9BCDF814B00693DA
:108540000C9BCDF8088004930B9B194A03930A9B5C
:1085500021460193099B484600933B46013709F0A9
:10856000B5FF102F06F1070605F107057FF452AF9E
:1085700066E70024CFE75446DEE75546094B08FB83
:1085800004360121D6F87C2101FA05F31A4205D000
:10859000009523463A46484609F098FF01350E2DCE
:1085A000EFD189E71830002009C101081EBA01087F
:1085B000FFB901082DE9F04F0446A74FDFF8D0823C
:1085C000A64E89B020460AF015FFC1B221B901209C
:1085D00009B0BDE8F04F15E705223946204610F0F6
:1085E0005EFD0546A0B9014670229D4810F014FDBD
:1085F0000E2428462A469B4904FB00130130082814
:10860000A3F87C21A3F87E21F6D109B0BDE8F08F54
:1086100004224146204610F042FD054600284DD177
:10862000204609F044FE81460028EED00AF0E2FE22
:108630002C46DFF860A25FFA80FB5AF824502DB96F
:10864000894809B0BDE8F04F09F088BE5A4629466E
:10865000484610F024FD01340028EED1814B02463B
:108660009E4603F1700183F8082183F8042183F802
:10867000032183F8022107338B42F4D17B4B03EBB8
:10868000C40494F8D890484505DB2946784809F099
:1086900065FE784C96E7D4F8DC30C0EBC00C634440
:1086A0000EEB0C01D3F800C001F58172C1F802C1D4
:1086B0009988013091809B799371E4E707223146D4
:1086C000204610F0ECFC0546002877D120212046FA
:1086D00010F0D7FC81460AF08DFEC4B284BB664818
:1086E00009F03CFE654D21462846013409F036FE6E
:1086F0000E2CF8D1624809F031FE0024DFF8989181
:10870000584FDFF898810E262146484609F026FE8C
:10871000002506FB04760123D6F87C21AB401A42E3
:108720005849594818BF4146013509F017FE0E2D2A
:10873000F1D15348013409F011FE082CE3D164E76C
:10874000524948460DF0CCFF2C46504D00283ED0F3
:10875000022C18D1009B072B2DD801990D292AD85E
:108760000278722A19D06E2A25D10E203D4A00FBCC
:108770000323012202FA01F1D3F87C2122EA01024B
:10878000C3F87C2115E00DF083FF29464DF8240045
:1087900000200DF0A5FF0134D8E70E20314A00FB80
:1087A00003230122D3F87C0102FA01F10143C3F84B
:1087B0007C11344606E709F02FFFFAE720463349DB
:1087C0000DF08EFF0024314D80B1082C04D109B08A
:1087D000BDE8F04F09F020BF0DF05AFF29464DF8D3
:1087E000240000200DF07CFF0134EDE7082CEED1D1
:1087F000009B0F2BEBD8DDF80490B9F1070FE6D8FA
:10880000DDF808C0BCF10D0FE1D8DDF80CE00EF189
:108810006402C82ADBD8049DFF2DD8D805986428A7
:10882000D5D806996429D2D88842D0DA079C032C7F
:10883000CDD8C3EBC3020B4B134483F8029183F8EA
:1088400003C183F804E183F8055183F8060183F836
:10885000071183F808411CE7B2B8010835BA0108CE
:108860001A31002018300020D8B8010834960108C9
:10887000E7B8010858C40108BCBB01083DBA0108AB
:1088800009C1010801CE010842BA010846BA01082F
:10889000D3B8010844A1010874CF01081BC801081E
:1088A0002DE9F047814688460D460027334CDFF816
:1088B000D0A088B0B8F1000F5DD0B4F97221B5F93D
:1088C00000309A4295F9092053D1B4F97401B5F9F1
:1088D000021088424DD1B4F97601B5F904108842EE
:1088E00047D194F87901297A884242D194F97801E4
:1088F00095F9061088423CD194F97B11881A4142BF
:108900004141069295F90620484605922A7A0E467C
:108910000492EA790392B5F904200292B5F9022093
:10892000009301923B46524609F0B0FD94F97B3129
:108930005246069394F978313146059394F87A318A
:108940004846049394F879310E350393B4F976319F
:108950000E340293B4F966310193B4F96431009393
:108960003B46013709F0B2FD082FA3D108B0BDE89E
:10897000F0870021C5E74646D8E700BF1830002041
:1089800048BA0108F0B5017885B0054600294FD0F6
:1089900000242B78002B50D1082C56D1BDF9003083
:1089A0009AB2072A51D840F2DC54BDF90210A1F264
:1089B000EE2292B2A24248D8BDF90420A2F2EE20E3
:1089C00080B2A04241D8BDF9060081423DDC82421E
:1089D0003BDB914239DCBDF90C5005F16404A4B2D3
:1089E000C82C32D8BDF90E40112C2EDCBDF9087010
:1089F000BEB2B42E29D8BDF90A601FFA86FEBEF1B8
:108A0000B40F22D84FF00E0CDFF874E00CFB03E338
:108A1000A3F87211A3F87421A3F8760183F8797191
:108A200083F87A6183F8785183F87B4105B0F0BD13
:108A3000012005B0BDE8F04032E72D2B03D0A3F1B3
:108A40003002092A16D8072C04DD05B0BDE8F04035
:108A500009F0E2BD28460DF01BFE04AB661C03EBDB
:108A6000440424F8100C15F8013F303B092BFAD9C7
:108A700034468EE7202BE8D101352646F8E700BFC3
:108A80001830002003788B4286BF024B33F8110068
:108A9000002070473C150020034B187E10B10022C7
:108AA00001201A76704700BF3C150020F0B5002564
:108AB00041F221072B46224A517E8E1EECB2B4426F
:108AC00017DB01448C1E013914441144A47E897EB5
:108AD00001EB042189B28B420AD100244FF4AF6626
:108AE00092F83D500130E3B29D4216D8012313762F
:108AF000F0BD04441444A47E83EA0423082413F440
:108B0000004F04F1FF344FEA430318BF7B4014F0D9
:108B1000FF049BB2F3D10135D0E700EB4303D9B298
:108B20005318013111449F7E8B7E03EB07239BB2C8
:108B300073431B1303F5487322F814300134D2E752
:108B40003C15002007298FBF0020034B03EB810158
:108B5000086C80B2704700BF3C1500202DE9F04141
:108B6000174D95F8602012B90020BDE8F081002271
:108B700085F8602095F86120A82AF5D195F8744011
:108B8000002CF1D10F4F104E05F16108403508EB74
:108B90000403D8781B7903EB00200BF08BF93946DE
:108BA0000BF0E0F931460BF0D3F80BF0DDFB45F8A4
:108BB00014000234102CEAD10120BDE8F08100BF7E
:108BC0003C1500200000203E0080BB43034B03EB1C
:108BD0004101B1F87600C008704700BF3C15002085
:108BE0001F4BF0B593F8962019460AB90020F0BD46
:108BF000002093F89740B3F8986003EB440595F88C
:108C00009D7095F89E2083F8960042EA07229642CE
:108C1000ECD193F89B30012B02D0812B14D0F0BD06
:108C20001846102C88BF10234FF0000288BF81F82F
:108C300097300C4B91F89740A3F12705D1B28C42A5
:108C400003F1020302D8F0BD0320EAE713F8026C37
:108C500013F8011C41EA062125F812100132EDE754
:108C60003C150020D915002003788B420CD9074B06
:108C7000890093F8BF200B44D3F8C00002B140082C
:108C800000F5777080B27047002070473C150020D7
:108C9000054B03EB8101D1F8F00000EB8000C00828
:108CA00000F55C7080B270473C1500205E4B10B53B
:108CB00093F83801002800F0B680002293F83B4179
:108CC00093F83C0183F8382193F83A2104F0070126
:108CD00042EA012200F03F01490141EAD401C3F810
:108CE000F02093F83D21C3F8F41093F83E11920060
:108CF00093F83F4142EA901201F0010042EA8022DB
:108D0000C3F8F82093F8400104F00F02D20142EAC0
:108D1000510200F07F01C3F8FC20090193F84121C2
:108D200041EA141193F842415200C3F8001142EA9B
:108D3000D01204F0030193F8430142EA4122C3F840
:108D4000042193F8442100F01F018901D20041EA77
:108D5000940142EA501293F8464193F84701C3F850
:108D60000C2193F84521C3F8081104F0070142EAE9
:108D7000012200F03F01490141EAD401C3F810216A
:108D800093F84821C3F8141193F84911920093F80D
:108D90004A4142EA901201F0010042EA8022C3F8FF
:108DA000182193F84B0104F00F02D20142EA51025C
:108DB00000F07F01090141EA1411C3F82011C3F842
:108DC0001C2193F84C2193F84D41520004F003010B
:108DD00042EAD01242EA4122C3F8242193F84F21FB
:108DE00093F84E01D20042EA501200F01F01C3F87E
:108DF0002C2193F85021890141EA9401D407C3F84A
:108E000028114CBF40F21471AD21C3F83011910705
:108E10004CBF40F21471AD2112F0080F14BF0320B3
:108E20000120C3F8341110BD3C15002008B5084BD3
:108E300003EB8101D1F854010BF03CF805490BF02C
:108E400091F805490AF086FF0BF08EFA80B208BD52
:108E50003C15002001F11F3F00405C446B4B30B5D6
:108E600093F894210AB9002030BD002283F89421A0
:108E700093F89721162AF6D1082112F0800F4FEAB5
:108E8000420218BF82F0D5020139D2B2F5D193F86F
:108E900096015F4D02388142C0F2A78093F8AE116F
:108EA0009142E0D1182293F8994193F89A0183F8FE
:108EB000962193F8982104F0070142EA012200F07C
:108EC0003F014901C3F8542141EAD40193F89B21A1
:108ED000C3F8581193F89C11920093F89D4142EA0F
:108EE000901201F0010042EA8022C3F85C2193F85D
:108EF0009E0104F00F02D20142EA510200F07F010C
:108F0000C3F86021090193F89F2141EA141193F8F5
:108F1000A0415200C3F8641142EAD01204F00301E8
:108F200093F8A10142EA4122C3F8682193F8A221F3
:108F300000F01F018901D20041EA940142EA501277
:108F400093F8A44193F8A501C3F8702193F8A321E5
:108F5000C3F86C1104F0070142EA012200F03F015E
:108F60004901C3F8742141EAD40193F8A621C3F85A
:108F7000781193F8A711920093F8A84142EA901251
:108F800001F0010042EA8022C3F87C2193F8A90194
:108F900004F00F02D20142EA510200F07F01090100
:108FA00041EA1411C3F88411C3F8802193F8AA216F
:108FB00093F8AB41520004F0030142EAD01242EAB6
:108FC000412293F8AC01C3F8882193F8AD2100F059
:108FD0001F018901D20042EA501241EA9401C3F80C
:108FE0008C11C3F89021012030BD6C18E4786240E8
:108FF000082412F0800F4FEA420218BF82F0D50217
:10900000013CD2B2F5D1013145E700BF3C1500204B
:10901000D116002038B5314C054694F8B93143B12A
:10902000D4F8BC3183429EBF002384F8B93184F860
:10903000C031D4F8C43113F001021CD094F8C82117
:1090400094F8C93193420CD00123002184F8C03137
:10905000234B84F8C9211970D4F8CC312B44C4F8BF
:10906000BC3194F8E8317BBBD4F8F801854234BFB9
:109070000020012038BD13F4005308D01346194ACC
:1090800032F8131011BB01330C2BF9D1E9E784F846
:10909000E831D4F8F4319847C307E2D5012300F052
:1090A0000200002814BF1A46002284F8E8310C4B55
:1090B0005A700CBF0123002384F8B931D4F8CC31A5
:1090C0002B44C4F8BC31CCE7012038BD0123002279
:1090D00084F8C031024B1A70F0E700BF3C15002045
:1090E000200200200C17002000207047002070474D
:1090F000024B03EB4101B1F8D00170473C15002051
:10910000024B03EB4101B1F8D00170473C15002040
:10911000024B03EB8101B1F8FC0170473C150020C4
:10912000254BF0B593F834220AB90020F0BD002297
:1091300093F8384283F834221C4494F8385294F857
:10914000371293F8594201EB0521012CB3F836028E
:1091500089B228D193F85A2202F11C05EDB29E186B
:1091600096F83A7296F83942023204EB0724D2B2EA
:109170002044AA4280B2F2D18842D6D1002193F88D
:109180005A520E4805EB4102D2B21A4492F83A42C2
:1091900092F8392202EB042240F8212001310E29F5
:1091A000F0D10120F0BD03F23925545D0132001BDE
:1091B0001E2A80B2F9D1DFE73C15002038170020C5
:1091C00070B5054601F0CEF9324CD4F85C32C4F8E3
:1091D0005C02C31AB3F5FA5F82BF002384F86032E1
:1091E00084F8613294F8603233B9A12D1ED1012286
:1091F00084F861221B22627694F861222AB1E21877
:10920000EDB20133957684F8603294F86052637E53
:10921000AB420AD194F86232052B0ED0062B0FD048
:10922000002384F8613284F8603270BDA22DE3D14E
:10923000012284F861222322DDE70020FFF736FCBB
:10924000E37E1E2BECD100200246013DC3B2AB42AF
:1092500007DB2544AB7E9A42E2D10320FFF726FCD0
:10926000DEE7082123449B7EDBB282EA030616F088
:10927000010F4FEA530301F1FF310CBFDBB283F062
:109280008C0311F0FF01C2F34702EED101301A4600
:10929000DCE700BF3C15002010B5044601F062F980
:1092A00041F288310D4BD3F86422C3F86402821A6C
:1092B0008A4284BF002283F8682293F86822142A25
:1092C00003EB02010CBF0122013281F8614014BF9F
:1092D00083F8682283F8602010BD00BF3C15002091
:1092E00010B5044601F03EF9254BD3F86C22C3F8C3
:1092F0006C02821AB2F57A6F84BF002283F8702262
:1093000093F870224AB9A82C38D183F89620A3F894
:109310009820991881F89A4006E0022A02D183F831
:109320009740F6E7242AF4D993F8971001320231D6
:10933000D2B249008A4283F8702216DA082241F23A
:109340002101B3F89800E4B280EA042010F4004F41
:1093500002F1FF324FEA400018BF484012F0FF020E
:1093600080B2F3D1A3F8980010BD01318A4201BF49
:10937000002283F87022012283F8962010BD00BFDE
:109380003C150020F8B5434C94F87802002859D0D9
:10939000002384F8783294F8793294F87A5205EB05
:1093A000032501F0DFF83C4BADB2B0FBF3F0D4F88D
:1093B0008C32002B47D1A4F89052C4F88C020322BF
:1093C000D4F8943294F893521E7894F8920294F858
:1093D0009872511E631893F879322B4103F00F03F2
:1093E000B34212D20B2B10D808B183420DD02144C6
:1093F00091F879E2A11891F879120EEA070E04EBC0
:10940000830301EB0E21C3F8C0100232112AE0D110
:1094100094F89932ABB194F89A3293B194F87B32C4
:109420001B060ED501F09EF8D4F874321B49643047
:109430001BB15A68121A002A28DB194AD360043279
:109440000A600120F8BD9842B9D0C31A012BB2D1ED
:1094500094F89222002AAED0B4F8903294F8BF105B
:1094600092002244EB1A49B16FF01301DB0293FB27
:10947000F1F303F50063C2F8C0309CE76FF013010D
:109480009B0293FBF1F303F58063F4E703F108011A
:109490009B68CDE73C15002020A10700B0170020F5
:1094A0002002002010B5044601F05CF841F288313A
:1094B0000E4BD3F89C22C3F89C02821A8A4284BFC6
:1094C000002283F8A02293F8A0220F2A0DD8511C65
:1094D000C9B21A441029E4B282F8794214BF0022BA
:1094E000012283F8A01283F8782210BD3C150020D9
:1094F00010B5044601F036F840F6AC51104BD3F8E5
:10950000A422821A8A42C4BF002283F8A82293F8B8
:10951000A8228AB90F2C11D1C3F8A402511CC9B2D8
:109520001A44192982F8394114BF0022012283F814
:10953000A81283F8382101E0182AEFD910BD00BF26
:109540003C15002010B5044601F00CF8124BD3F87E
:10955000AC2202F57A72904284BF002283F8B022D6
:1095600093F8B01219B9C3F8AC02052204E002293D
:10957000FBD993F8962102328A420CDD481CC0B216
:109580008242CCBF00220122194483F8B00281F844
:10959000954183F8942110BD3C15002010B5044678
:1095A00000F0E0FF214BD3F8B422C3F8B402821AD2
:1095B000B2F5FA7F84BF002283F8B82293F8B8226C
:1095C00082B993F8B91249BB552C17D101211F203C
:1095D00083F8591283F8B94283F83802A3F8362287
:1095E00083F85A12991881F8394293F838120139E0
:1095F0008A4216D1012283F8342210BD202C0FD1CB
:10960000022183F85A124FF6FF7183F8592283F82A
:10961000B94283F83842A3F83612E3E78C42E1D02E
:1096200010BD013283F8B822FAE700BF3C150020D4
:1096300010B5074C94F89A2242B104F2BA21D4F83A
:10964000D00205F0D6FB002384F89A3210BD00BF8B
:109650003C150020194B2DE9F0411C680746092CE8
:10966000984607DC0023164A9C4206DC0025144E6F
:10967000A54208DD0020BDE8F08152F823108F429A
:10968000F8D00133F0E756F82530681C7BB980002C
:10969000621B011F92003144304401340FF0A2FCE0
:1096A00046F82570C8F800400120BDE8F0811A7D19
:1096B0003B7D9A42EBD30546DAE700BF0C1500204C
:1096C000101500202DE9F04105460F460446094ECD
:1096D00006F10808217809B9BDE8F08105480FF0C6
:1096E000D0FC20B140453EBF801B631B3B5401347E
:1096F000F0E700BFA19D0108094B93F8D42262B99D
:10970000D3F8D82293F8EC1192F820200432D2B288
:109710008A4228BF0A4683F8D42293F8D4027047BD
:109720003C150020124970B5D1F8D83245005C19BB
:1097300094F828600A462EB1022E0FD05319B3F8C0
:10974000DC0270BD022805D90328F7D1D1F8C42165
:10975000D20401D5D88A70BD988C70BD94F82900C8
:1097600000EB800000EB800000F2EE2080B270BDC4
:109770003C15002008B500F0F5FE0222064B83F8E8
:109780000423064AC3F800031268C3F81023012219
:1097900083F8292308BD00BF3C15002008350020B0
:1097A00008B500F0DFFE0222074B00F5B71083F882
:1097B0000423D3F8102300F5587002F2DC52C3F8EA
:1097C0000003C3F8102308BD3C15002070B5054602
:1097D0000024084EA359AB4207D1284601F0BFFC34
:1097E000CC22002130190FF017FCCC34B4F5197FCE
:1097F000F0D170BD681800202DE9F04F012085B030
:1098000001F0DAFD00241A4EDFF868A006F54B7B64
:1098100008B1022C02D905B0BDE8F08F4FF0CC0999
:1098200009FB04F806EB0807D7F82C5315B10134EF
:10983000E4B2EDE70322C378012190F902005AF85F
:109840002330009201952A4601F09EFC039050B10E
:109850004A4629460BEB08000FF0DEFB039B013460
:10986000C7F82C33E4B2012001F082FDD0E700BF3D
:109870003C1500207CA5010810B50D4C94F890050E
:1098800001280CD00AD302280CD000F06BFE00F5A2
:10989000F42000F59070C4F8940510BD002007F086
:1098A000A7FCF2E7034B186805F0BEFCEDE700BF2C
:1098B0003C1500205435002010B501240B4B1C70C2
:1098C00008F06EFB002008F005FB204608F002FBC4
:1098D0000E2008F0FFFA204608F0FCFA08F044FBDE
:1098E000BDE81040024808F05FBA00BFA435002070
:1098F000A535002073B504780546002C44D0002619
:1099000004F10A03ADF8043008F04AFB9DF80500A5
:1099100008F0E0FA9DF8040008F0DCFA0E2008F0E8
:10992000D9FA1C4B187808F0D5FA304608F0D2FA6C
:10993000204608F0CFFA002008F0CCFA002008F00A
:10994000C9FA002008F0C6FA002008F0C3FA002087
:1099500008F0C0FA002008F0BDFA002008F0BAFABA
:109960006B68013C187808F0B5FA6B6814F0FF04D6
:1099700003F101036B60F3D108F0F6FA064802B078
:10998000BDE8704008F010BA4FF485730126ADF8B9
:109990000430B9E7A4350020A535002038B50546C8
:1099A000064C206800B938BD4368EB1A002BFADB7F
:1099B0008368236003689847F3E700BFB01700206F
:1099C0002DE9F047064689464FF000474FF0000862
:1099D000038A8589ADB21D400DB9BDE8F087B5FA9F
:1099E00085F327FA03F2D2431B3B91B23182154033
:1099F000042BF1D8DFE803F02925211A0300D9F858
:109A0000244084B1013CA4B2C9F82480D9F820A034
:109A1000BAF1000FE0D0DAF80030504621469847FE
:109A2000DAF804A0F4E7B48DA4B2EFE7D9F80000A7
:109A3000B18E036889B29847CEE7D9F80400318F18
:109A4000F7E7D9F80800B18FF3E7D9F80C00B6F8BA
:109A50004010EEE738B5264C94F8B03243B1254DAE
:109A60002B782BB9FDF7DBFE0123234A2B701370F3
:109A7000224B1B88002B39D121490B7813F0010FA1
:109A800003F004022CD08ABB1E48006845012DD487
:109A9000980725D40A2243F00C030B701A4BB3F934
:109AA000043093FBF2F3194A1380194B1B681B0314
:109AB00007D5802007F05EFC08B1FFF787FEFDF7B1
:109AC00007FA4FF47A71134B05201A6894F8B232F2
:109AD00001FB0323104A1360BDE8384006F01EB8AE
:109AE00022B9BDE83840012001F06EBC38BD00BF8E
:109AF00018300020D41A0020D80B0020F40F0020CA
:109B000028260020181C00202A260020B80B002040
:109B100000170020083500206C0B0020002208B53B
:109B20000A4B1A700A4A137859070DD523F004031B
:109B30001370084B1B681B0301D5FDF7ABF9BDE89B
:109B40000840042005F0EABF08BD00BFD80B002084
:109B50002826002000170020022828BF02200A4BD8
:109B60000A4A1870742392F81C144B43D11881F8D8
:109B700080030C2103F2823301FB0030044B1044BC
:109B8000186009F005BC00BF221C0020183000201E
:109B9000380E0020012828BF012010B50446064BCE
:109BA00083F81C0401F058F800F0B6FE601CC0B247
:109BB000BDE8104001F008BC1830002008B501F0E5
:109BC0004BF800F0A9FEBDE80840012001F0FCBB05
:109BD0002DE9F0413D4CB4F80432B4F806229A4223
:109BE00028BF0023B4F80A2228BFA4F80432B4F82E
:109BF00008329A4224BF0023A4F8083294F8FF31B7
:109C0000002B5AD0072B58D0012384F8F83184F860
:109C1000FE3100232E4D84F8033294F8032294F889
:109C2000FE31002A4BD0102B38BF1023294D84F869
:109C3000FE3194F8FE010AF041F929460AF092F942
:109C4000804694F8F87138460AF038F941460AF02F
:109C500089F994F8D4500146022D96BF1E4B1D4E33
:109C600053F8256030460AF039FB88B1414630464A
:109C70000AF02CFA0AF052FB1028A8BF1020012885
:109C8000B8BF0120C0B2B84228BF384684F8F801F6
:109C900094F8D5307BB1013D032D0CD831464FF0FF
:109CA0007E500AF013FA0CF0E1FEB4F8D23098427C
:109CB00038BFA4F8D200BDE8F081084DADE7032B12
:109CC00038BF032384F8FE31B3E700BF183000200B
:109CD0006F12833A6F120338B89D01086F1203396F
:109CE000F8B52C22002104460FF096F964230022D7
:109CF00023855223052184F82A3004252346104663
:109D0000074FD65D0132052A9E70D9701D7198717A
:109D1000597103F10803F4D101232380F8BD00BF7A
:109D2000C49D0108F0B50F250571222545710E254A
:109D3000C5733525457619253A22857121252C23B1
:109D400042700574162253250370427528232D2274
:109D500085764FF4FA75322114274B2683720273ED
:109D6000037200223723458546244FF07C55077542
:109D70008775C6764372C3744677C562C1728470B4
:109D8000C1704273C27582730276C171417442849C
:109D900080F8281080F8333080F83430234B4FF4AB
:109DA000827C4364002383644FF4AF734FF0010E51
:109DB00003874FF07E536425A0F824C04FF0A00C19
:109DC00080F81EE080F832E080F84070C3634FF006
:109DD0000A0E034640F2726780F835600584A0F8E9
:109DE00026C080F8312080F8415080F8362000F1FC
:109DF000240683F84E5083F84F5083F8502083F8A0
:109E0000511083F8522083F856E083F85720A3F8C6
:109E1000587083F8534083F8544083F855400C330E
:109E2000B342E6D180F84C20F0BD00BF00002041D5
:109E30002DE9F84F40F2EC42002104460FF0ECF817
:109E40005A2184F801124FF49671A4F80612C82121
:109E5000A4F80812642140F2011340F6C412A4F8D9
:109E60000A122B253021A360A4F8F0219C2308229C
:109E700084F8FD1184F83B526E2121254FF4C870FF
:109E8000237084F8FE210023012284F8381284F81C
:109E90003C520A212325A4F8040284F8391284F8DC
:109EA0001C34A4F8F23184F8FF3184F8F82184F8E6
:109EB000003284F8F93184F8FA21A4F81C32A4F8AD
:109EC0001A32A4F81E3284F8FC3184F8183284F86F
:109ED0000E3284F8193284F8502284F80F2284F864
:109EE000242284F83A2284F83D52A4F84002372014
:109EF00084F84802E44884F84B12014684F83E2274
:109F000084F83F32A4F84232A4F8463284F844225E
:109F100084F8492284F84A3200EBC305AA7912F08A
:109F2000010200F0BB812B7984F81C3300231A4610
:109F3000C8188579AE0741BF0579A01880F81D5370
:109F40000132582B40F0B181012284F8052384F8B6
:109F5000062384F8262384F82A2384F8282384F807
:109F6000302384F85D2284F8662240F2DC5205201A
:109F7000A4F86A2240F24C4284F814031020A4F89A
:109F80006C2240F26C7284F827032120A4F86E2220
:109F900040F2753284F82B032020A4F8782240F692
:109FA00043020023002784F829031F20A4F87A2203
:109FB0002646224684F80433C4F80873C4F80C73A8
:109FC00084F8103384F8113384F8123384F813338F
:109FD00084F8153384F82F3384F82E0384F85C3228
:109FE00084F85E3284F85F3284F86532032BCCBF8C
:109FF0000120002082F87C020CBF05201E200133C6
:10A00000122B82F87D0202F10202EFD100231E2200
:10A0100084F8673284F8682284F86932022284F86E
:10A02000713284F87332062384F8702284F8743213
:10A03000132240F246534FF47A704FF4FA6584F8D5
:10A040007222A4F8763204F52D7204F5297323F8F0
:10A05000040C23F8025C04339342F8D14FF0050E50
:10A0600084F8B2E24FF0190E84F8F4E14FF0030ED9
:10A07000012284F8B3E240F22E4E002384F8B1228C
:10A0800084F8B52284F8B42284F8D4207F4AA4F856
:10A09000CCE04FF4F07EC4F8D8201A4684F825337B
:10A0A00084F8B032A4F8D2E0A4F8CE50A4F8D000DE
:10A0B000C81885796D0741BF0579A01880F8DC5074
:10A0C0000132582B03D00B2A03F10803F0DD0123E2
:10A0D00040F2DC5284F8FC304FF4C873A4F8F0204E
:10A0E000A4F8FE3032220023A4F8F2201A4684F8A5
:10A0F0000031C81885792D0741BF0579A01880F86F
:10A10000F4500132582B03D0072A03F10803F0DD85
:10A1100040F27E53A4F8E83040F2EA53A4F8EA3063
:10A1200040F2B453A4F8EC3032230022A4F8EE300D
:10A1300004F5337104F530731A7303F8012B994257
:10A14000FAD100222B254FF02A0E4FF0200C4FF0B1
:10A15000250811464E481356022B00F0BB8000F331
:10A16000AA80002B00F0B1800132052AF3D100252E
:10A170004FF001094FF00A0A4FF0280B04F5367032
:10A1800004F54D78FFF7ACFD4046FFF7CBFDA4F892
:10A190002052A4F82252A4F80C5284F8F59104F548
:10A1A00015713C48A4F816A284F8F6B184F8F7B10A
:10A1B000FFF788FA4FF448734FF47A71642284F8F9
:10A1C0004F92A4F8343284F8BE9223464FF4FA69D1
:10A1D00040F2DC5C5A204FF0FF0E84F84C5284F8B9
:10A1E0004D5284F8365284F8BA5284F84EB284F84C
:10A1F000B6A284F8B7A2A4F8B812A4F8BC2204F15D
:10A200007005A3F87211A3F87491A3F876C183F8CE
:10A21000782183F8790183F87A0183F87BE10E33A2
:10A22000AB42EED1002384F8E231042384F8E33119
:10A2300004F1C003F7601036B342FBD1012284F869
:10A24000C72484F8C8242C22002384F8CB2423229A
:10A2500084F8C93484F8CA3484F8193384F81A337A
:10A2600084F81B330C4B84F818231A681B79C4F844
:10A27000E52484F8E934414604F56A707422BDE8A7
:10A28000F84F0EF0A4BE00BF1CA5010800009040CE
:10A29000C49D010868BA010810B1010801330C2BF4
:10A2A0007FF43AAE84F81C2340E6072A03F1080342
:10A2B0007FF73EAE48E61E2B11D01F2B7FF454AF24
:10A2C00084F8D71284F8CB124EE784F8CC3284F8A5
:10A2D000C03249E784F8CE5284F8C2E244E784F8F9
:10A2E000D6C284F8CA823FE710B50A4C2046FFF771
:10A2F0009FFD094B04F54D721A6094F88033074AAC
:10A3000013700C2202FB0343054A03F282331360ED
:10A3100010BD00BF18300020881E0020221C002025
:10A32000380E002001490248FFF74ABB501B0020AD
:10A330000008004001490248FFF742BB281B0020EB
:10A340000004004002494FF08040FFF739BB00BFD6
:10A35000001B002001490248FFF732BBD81A002039
:10A36000002C0140FFF7F6BF254B10B55343254A9B
:10A37000254C12680139B2FBF3F20388013AA0427E
:10A3800089B292B29BB212D004F50064A0420ED002
:10A39000B0F1804F0BD0A4F59834A04207D004F55B
:10A3A0008064A04203D004F58064A04202D123F06F
:10A3B00070039BB2154CA04206D004F58064A04205
:10A3C0001CBF23F440739BB203800F4B81859842DE
:10A3D00002850FD003F5006398420BD003F540636C
:10A3E000984207D003F58063984203D003F5806359
:10A3F000984201D1002303860123838210BD00BF50
:10A4000040420F0074020020002C01400010004068
:10A4100073B504460068FFF7A7FF2168184A0B8848
:10A4200002F114009BB243F001030B80002350F8AB
:10A430003350DC00A9421ED12244557E012400265F
:10A4400001A88DF804508DF805408DF806608DF850
:10A450000740FDF745F91B2D0BD1192301A88DF8F5
:10A4600004308DF805408DF806608DF80740FDF743
:10A4700037F902B070BD0133042BD8D10025DDE7D8
:10A48000B89D01080B4B800A98420FD004D8B0F554
:10A49000801F09D0FE207047074B984208D04933EF
:10A4A0009842F7D100207047012070470220704782
:10A4B000032070470100100002001000F8B5046886
:10A4C00005462046FFF7DEFF032840D86B794FEAA8
:10A4D000930E39B976460227A589B740ADB225EA71
:10A4E0000705A5810A2606FB00E61C4D05EB86073D
:10A4F00079607A6131B19A080223A18993400B43B4
:10A500009BB2A38128214143154A01F12003134442
:10A51000EFF31286502787F3128810310A44042182
:10A52000176817B11F6013680433013902F1040280
:10A53000F6D11960F3B283F31188282303FB00508E
:10A54000436A2BB1A3899BB243F00103A381F8BDF9
:10A55000A38923F001031B041B0CF7E7D41A002086
:10A56000D81A00201F4B70B55B681F4AC3F308035D
:10A57000A3B9EFF312838BB91C4910688C6800BF34
:10A5800013689842F9D14FF47A72194BD3F8A81096
:10A5900002FB01F31B1BB3FBF1F31FE0EFF312848B
:10A5A000102383F31288114D1149AE682B6813F400
:10A5B000803F1EBF0123C1F8A430AE681568D1F8F2
:10A5C000A400E2B282F311884FF47A72D1F8A81095
:10A5D000284402FB01F39B1BB3FBF1F302FB0030A9
:10A5E00070BD00BF00ED00E00835002010E000E085
:10A5F000D41A002038B50446FFF7B4FF0546FFF72C
:10A60000B1FF401BA042FAD338BD10B5044604B9CF
:10A6100010BD4FF47A70FFF7EDFF013CF7E708B586
:10A620000E4B93F8AC3003F00503052B0DD10C4B0A
:10A630000C48B3F900100C4B1A780023934208DB46
:10A6400005F062FC3220FFF7E0FF002006F0D0FDAD
:10A65000FEE720F813100133F0E700BFD41A002002
:10A660006A1D0020642500205C2500202DE9F843A8
:10A6700081460B25DFF86C80013D04D1174A184B49
:10A68000DA60BDE8F883002006F0B2FD3227052429
:10A6900009F10106D8F8000004F0C6FD012006F01B
:10A6A0004BFB3846FFF7B1FFD8F8000004F0BCFDC3
:10A6B000002006F041FB3846FFF7A7FF3CB1013C04
:10A6C000E8D14FF4FA70FFF7A0FFFA27E2E7013E66
:10A6D000E0D14FF47A70FFF798FFCDE70400FA0558
:10A6E00000ED00E054350020014B186804F07EBBFB
:10A6F000001F00200E4B98420AD0A3F578439842E1
:10A7000011D003F5806398420FD04FF0FF307047AF
:10A710000022084B03EB02135A89013292B25A818C
:10A72000588980B270470122F3E70222F1E700BFA7
:10A7300000300140300200202DE9F8434F4C060163
:10A74000A7190546387A06F035FD01233A7A02F05A
:10A750001F015209022A03FA01F365D0032A68D0C7
:10A76000A719787904F01CFD12230135EDB283712D
:10A770008046C571F87904F013FD4FF01309C571D7
:10A7800080F80690B87904F00BFD14231B21837127
:10A79000C571404604F026FDF87904F001FD07215B
:10A7A00004F020FDB87904F0FBFC1B2104F01AFD35
:10A7B000387938B104F0F4FC1F22C5718271494622
:10A7C00004F010FDA3592E4A934237D102F560429E
:10A7D000D16841F48051D160D16821F48051D160B9
:10A7E000A219127B002A44D1012202201988344484
:10A7F00001F4415141F445710A4302431A809A8B96
:10A80000207922F400621204120C9A8307221A8221
:10A810001A8892B242F040021A8068B304F0C0FC79
:10A82000BDE8F84304F00EBD164AD1680B43D3606F
:10A8300096E7144A11690B43136191E7124A934258
:10A840000AD102F5EC32116941F4804111611169BC
:10A8500021F480411161C3E70C4A9342C0D102F553
:10A86000EA32116941F400411161116921F400419A
:10A87000F0E700221046B9E7BDE8F8833002002077
:10A88000003001400010024000380040003C004011
:10A8900010B5427A044632B1036800F10A014068FB
:10A8A00098470023637210BD024A936823EA0000B0
:10A8B000906070471830002010B5134C23789C2B03
:10A8C0001FD140F2EC4362889A421AD12379BE2B01
:10A8D00017D194F8EA34EF2B13D105220B490C4819
:10A8E0000EF0DDFB68B90B4914F8013B83EA000266
:10A8F0008C42D2B203D11B1A5842584110BD1046A7
:10A90000F2E7002010BD00BF00F8010810B10108F7
:10A91000E5FC0108ECFC01082DE9F047FFF7CCFF4E
:10A9200010B90420FFF7A2FEA54CFEF739FF40F254
:10A93000EC42A44920460EF04AFB94F81C34A24D88
:10A94000012B84BF002384F81C34742394F81C2446
:10A950009E49534303F54D7222442A60E21892F84F
:10A96000802303F282330A700C2101FB0233984AE0
:10A970002344136094F8D430042B40F0FE80B4F8E4
:10A98000D030B3F57A7F03D24FF47A73A4F8D03085
:10A99000A368904A1A4012B943F00103A360A36868
:10A9A000DE0702D58C48FFF77FFFA368580402D565
:10A9B0008A48FFF779FFA368190702D58848FFF78F
:10A9C00073FFA3689A0103D546F20900FFF76CFFF5
:10A9D000A3689B0415D58348FFF766FF4FF400403A
:10A9E000FFF762FF94F84432012B03D14FF400606B
:10A9F000FFF75AFF4FF48030FFF756FF4020FFF774
:10AA000053FF4FF4367800274FF0FF09764E774B0F
:10AA10001E6034F80820530803F07733900800F0E4
:10AA20003330D31A1B1AD00800F011301B1A03EB75
:10AA3000231303F00F3393FBF9F012F00101C0EB85
:10AA4000002018BF0137A3EB000318BFFFB2012B92
:10AA50000DDD022B40F0AF8011B112F42F7F06D133
:10AA600004EB080004F0A0FD002800F0A48008F129
:10AA70000808B8F5407FCCD1013F022F00F29B803F
:10AA8000FFF7A6F808F084FC0021302258480EF0A9
:10AA9000C3FA2A68574B00201A6006F0F4FB564BA5
:10AAA000564980F001001870554BA1F14E021A6012
:10AAB0006423002594F8B602524A4343524FC833E8
:10AAC00053609560D560156155619561D56182F8D7
:10AAD000205082F821504D4A3960EA3911604C49C2
:10AAE000B4F8162289460A804A4AD06A904600285D
:10AAF00050D1494B494A03F2CB111360A3F11C0218
:10AB00007A60474AB4F8F0011160464A03F1140133
:10AB10001660454A454D1160454A03F18A011160AE
:10AB2000444A03F1FA011160434AFB33136009F010
:10AB3000C5F9424909F016FA6860B4F8F20109F063
:10AB4000BDF93E4909F00EFA94F8F5313C4A2B72F2
:10AB500094F8F431B4F834626B723A4B28601A609E
:10AB6000304609F0ABF90146374809F0AFFABDE8C5
:10AB7000F047364B1860FEF7FDBD002B7FF408AFA1
:10AB8000B4F8D230B3F5F07F84BF4FF4F073A4F87B
:10AB9000D230FDE6DFF8BCA0B9F8000009F08AF970
:10ABA000D8F82C2001460AEB05001C3508F004FB00
:10ABB000542DF1D19DE72648FFF792F860E700BFDA
:10ABC0001830002000F80108881E0020221C0020F8
:10ABD000380E00200960000208600002092000020F
:10ABE00001600002094000026C32002014180020AD
:10ABF000800B0020B40B00200C0000201C33002030
:10AC00005826002044180020841B0020E81F002044
:10AC1000921F0020B02500200031002054080020A1
:10AC20006C080020500800205C090020102600203D
:10AC30004822002058090020440A002017B7D138C4
:10AC40003661023D40260020C0C9FB481C07002099
:10AC5000F0320020941F00202DE9F743FEF7A0FDFD
:10AC60009C234A4E40F2EC413370BE233371EF23F4
:10AC700086F8EA3400231846718086F8EB34F25CDB
:10AC800001338B4280EA0200F9D186F8EB040427F5
:10AC900000203F4C3F4BDFF80491636003F18833A1
:10ACA0006360013F17F0FF0739D034233A4DE3606A
:10ACB00005F17848A8F5FC38C8F30903002B40D00B
:10ACC00000234FF4005056F808800193FCF7E0FB96
:10ACD0000428E6D123694FF4005043F001032361B7
:10ACE0001FFA88F32B80FCF7D3FB042847D1AB1C59
:10ACF0000193019B4FEA1848A3F800804FF40050DD
:10AD0000FCF7C6FB2369042823F001034FEAC34381
:10AD10004FEAD3432361C4D104354D45C8D11C4A01
:10AD20000428136943F08003136102D1FFF7C4FDC7
:10AD300010B90520FFF79AFCFEF71CFD03B0BDE833
:10AD4000F0834FF43020FCF7A3FB0428A9D123693A
:10AD50004FF4302043F0020323616561236943F01F
:10AD600040032361FCF794FB2369042823F00203CA
:10AD70004FEAC3434FEAD3432361A1D091E723694C
:10AD800023F00103DB04DB0C23618AE71830002089
:10AD9000002002402301674500F80108ECFC01088F
:10ADA0002DE9F84302780346202A00F10100F9D08A
:10ADB000092AF7D02D2A4BD10346444D1C460026C4
:10ADC000DFF80C81234614F8012BA2F13007F9B209
:10ADD000092943D92E2A09D127463D4CA0463B4696
:10ADE00017F8010B3038C2B2092A44D91A7802F098
:10ADF000DF02452A63D15A782D2A4CD1012702332C
:10AE000000240A20013B13F8012F303AD1B209295E
:10AE100047D9B4F59A7F28BF4FF49A744FF07E500B
:10AE2000A046DFF8B090B8F1070F3DD8DFF8A0805A
:10AE300004F00704002C3DD1002F42D001463046DB
:10AE400009F044F90146284609F08CF8BDE8F8837A
:10AE50002B2A08BF03464FF07E55AFE741463046E8
:10AE600009F080F80646384609F028F8314608F01F
:10AE700071FF0646A6E709F021F8214609F026F9F8
:10AE80000146304608F066FF41460646204609F076
:10AE900069F80446A3E72B2A14BF013302330027C5
:10AEA000AEE700FB0424AEE7494609F05BF8A8F1E1
:10AEB0000808B8E7414609F055F8013CBAE74FF0F9
:10AEC0007E500146304609F04DF8BBE7000080BFD8
:10AED0000000204120BCBE4C002330B50C4687B09A
:10AEE0000021054600930193029309F0F7F92949DF
:10AEF00000283DD0284608F02DFF274909F032F8F8
:10AF000009F00CFA054680EAE07003A9A0EBE570B1
:10AF100006F047FA002DACBF20232D2303A88DF89F
:10AF2000003008F067FA012826D130238DF801306F
:10AF30008DF802308DF8033003A968460EF092F8C0
:10AF4000684608F057FA0338C5B22A4669462046D3
:10AF50000EF0DEF800231149635520460EF082F80A
:10AF60000DEB050120460EF07DF8204607B030BD00
:10AF7000284608F0EDFEC0E7022805D130238DF801
:10AF800001308DF80230D7E7032804BF30238DF855
:10AF90000130D1E76F12033A00007A44B6CF0108BE
:10AFA00070B50646B6FBF2F40846154614B12046C5
:10AFB000FFF7F6FF05FB1464024B1B5D00F8013B35
:10AFC00070BD00BF71BA010870B50124B0FBF4F583
:10AFD0008D4202D21CB91C7070BD4C43F6E7B0FB29
:10AFE000F4F6092E0BDD002A14BF3725572535440A
:10AFF00004FB160003F8015BB4FBF1F4EAE730252B
:10B00000F5E7026810B51146531C036011F8024BB6
:10B01000D31C01605178036093781B0443EA012339
:10B02000111D0160D078234343EA006010BD03681E
:10B030005A1C02601A4612F8021B0260587841EA54
:10B040000020704703685A1C026018787047036834
:10B050005A1C0260197003685A1C02600A0A1A70AE
:10B0600003685A1C02600A0C1A700368090E5A1C05
:10B0700002601970704703685A1C026019700368F7
:10B08000090A5A1C0260197070470FB437B50B4893
:10B0900006AB53F8042B8168C068019307F091FE5A
:10B0A0000446074D286806F080FD0028FAD02046A7
:10B0B00003B0BDE8304004B0704700BF841B0020DF
:10B0C000001F0020704738B50B4C0546014620682C
:10B0D00003F08CFE082341F22102A08880EA0520BB
:10B0E00010F4004F4FEA400018BF5040013B80B2BF
:10B0F000F6D1A08038BD00BF941B002010B5054CD0
:10B10000206806F05BFD0028FAD02068BDE81040FA
:10B1100006F04EBD941B002010B5FFF7EFFF41F283
:10B1200021040821074AD38883EA00239BB213F441
:10B13000004F4FEA430318BF634001399BB2F6D179
:10B14000D38010BD941B002010B50446204606F0A5
:10B150002CFD00B110BD0A20FFF757FAF6E70023D7
:10B160000C2130B5074C01FB03425568A84203D0BF
:10B170000133052BF7D130BD0023C3621381536027
:10B1800030BD00BF683500202DE9F04F604D00272D
:10B190004FF00C0CA94687B0044603919DF844007B
:10B1A00011461A469DF840300CFB07F606EB050EDB
:10B1B0007657A64200F099800137052FF4D1002080
:10B1C0007EE01E2C00F08C801F2CF8D10090012016
:10B1D00088E04FF480584FF0030B4E4E4E4DB3694C
:10B1E00005A943F00403B36128468DF816B0ADF805
:10B1F00014808DF81740FCF797FAC5F81480C82022
:10B20000FFF703FAC5F81080B36905A943F00403FA
:10B21000B3614FF4C053ADF814301C2328468DF8A9
:10B2200016B08DF81730FCF77FFA4FF480233B4DB2
:10B230003B4A4FF0010B53612B65082305F1500089
:10B2400085F8553085F856B005F0E2FF354B364AA3
:10B25000C3F800A0F369354943F40003F361022603
:10B26000334B13601E72334A334B1360334A1B68EF
:10B2700011609847324B334A05A8DA608DF81440C4
:10B280008DF815608DF816A08DF817B0FCF728FA28
:10B290002A238DF814309DF817308DF815B08DF8ED
:10B2A00016A083B105A8FCF71BFA274B2748AB6013
:10B2B0000C2303FB0797BDF80C3004713B817860C9
:10B2C00007B0BDE8F08F4FF48062214BC3F88420B3
:10B2D000EBE700901F4806F0EBFA0028E8D16EE794
:10B2E0000090504605F034FDF7E7BEF808A0BAF12B
:10B2F000000F7FF464AF142C3FF46BAF3FF761AFE6
:10B30000002CE6D0022C7FF45AAF00901248E2E7FE
:10B31000683500200010024000080140941B002006
:10B3200000040140D8004242282B00205002002097
:10B33000B83500209C1E00208C030020981E0020A1
:10B3400000ED00E00005FA05EC9D01089C1B0020C3
:10B3500000E100E0003801400048004038B10388B7
:10B3600013EA010003D08B420CBF0120022070477A
:10B37000F0B500250E4B0F491A6891F85840E3B21A
:10B38000042B04D90DB181F858300020F0BD32F8FB
:10B39000347001333842DBB204F101064FF001058D
:10B3A00004D081F8583002EBC400F0BD3446E6E723
:10B3B00064350020941B00200022024B83F85820A3
:10B3C000D6E700BF941B00204000142870B4A8BF2B
:10B3D0001420002302261425084A02F159015E5464
:10B3E0000233CC18984204F8015CF8DC1344FF22C5
:10B3F00083F859200F2070BC04F090BB941B0020F0
:10B4000010B50024002005F097FC064B1C70FEF7D9
:10B4100033FA054B83F86F401C67A3F874409C67B0
:10B4200010BD00BFCC1A0020941B00202DE9F04F66
:10B430009C4DD3B02860FFF7E3FFDFF8789209F165
:10B44000140A0024AC71EC71FFF766FE2F28F9D1C5
:10B45000012005F0CDFEADF81040FFF75DFE019034
:10B46000FFF75AFE8DF81D00FFF756FE8DF81E00FF
:10B47000FFF752FE002407460DF14808FFF74CFE87
:10B4800008F804000134E3B29F42F7D1FFF736FE1B
:10B490008DF81500FFF732FE8DF81400BDF814602A
:10B4A000EB8801209E4214BF0326002605F0A0FE73
:10B4B000002E43D1019BCDF82080303B0F2B00F2B2
:10B4C000CE81DFE813F015003D0047024100100077
:10B4D0009500CC01B8006F01A001C101FF01CC01B2
:10B4E000EB0122028C00012404AF4FF0010B35E088
:10B4F0006D4F3B7813B395F87C301BB1022B09D903
:10B50000032B17D000243C707C704FF0010B04AF6C
:10B510000F2623E0FD23002402210CA88DF83030F3
:10B520008DF8314006F0C9FD012006F0B5FDC128B7
:10B53000E8D1D9E7FEF7C0F90028E3D00024D3E72B
:10B540006A238DF81030F9E790238DF8103004232A
:10B5500000244FF0020B8DF8113004AF0020287149
:10B56000687105F045FE286806F017FB2E20FFF7EE
:10B57000AAFD0198FFF7A7FD9DF81D00FFF7A3FDA9
:10B580009DF81E00FFF79FFD5846FFF79CFD0BF14D
:10B59000FF385FFA88F808F10108B844286806F017
:10B5A0000AFB0028FAD017F8010BFFF78CFD47457E
:10B5B000F4D13046FFF787FD6979286803F016FC5F
:10B5C0002979286803F012FC286806F0E1FA0020C7
:10B5D00005F00EFE002C3FF434AF344CD4E198F863
:10B5E00000305A1E022A00F2BA8185F87C30A5E7A5
:10B5F00098F8003095F87D209A4205D8002404AFD1
:10B600004FF0010B0826A9E7294A274F137095F838
:10B610007C30013B012B0AD800238DF830308DF8A7
:10B620003130012302210CA83B7006F046FD0024B6
:10B630003C707C7058E798F8003095F87D201A4FE0
:10B640009A423E707E70B846D8D90324184A07F152
:10B65000010B1370FEF730F970B30121584606F064
:10B6600033F848B30221104806F02EF820B349F20F
:10B670000732B8F8003023F00801914207D049F2B0
:10B680000A32934203D049F20B42934214D103236E
:10B6900085F87C3095F87C300024FB704FF0040B6B
:10B6A000014F5BE7941B0020BF3A0020803A002046
:10B6B000B03A0020149E010899F80230B9F8001041
:10B6C00006AADFF8F8E2937011800CAB9C46DEF816
:10B6D0000000DEF804100EF1080EACE80300D645B9
:10B6E0006346F3D1DAF800009AF804100392CCF81C
:10B6F00000008CF804100CA8152106F0DEFC09AB44
:10B7000008211846029306F067FD00283FD000216B
:10B71000039A029B13F801E0505C864537D1013152
:10B720000329F7D1DA7888F802201A795B7988F84A
:10B7300001204FF2103288F80030B8F8003023F0C2
:10B740002001914211D04FF2104293420DD04FF29E
:10B750009032934209D04FF65002934205D003F540
:10B76000BA520F3292B2012A01D8012390E749F26E
:10B77000073123F008028A4207D049F20A32934285
:10B7800003D049F20B42934201D1022380E7013CEE
:10B7900014F0FF047FF45EAF3C707C704FF0040B3C
:10B7A000814FB5E695F87C30032B58D112247F4B9E
:10B7B0001C7006F0F5FB002006F08CFB072006F05D
:10B7C00089FB0E2006F086FB204606F083FB142042
:10B7D00006F080FB002006F07DFBAC2006F07AFB33
:10B7E000882006F077FB132006F074FB762006F025
:10B7F00071FB06F0B9FB6E4806F0D6FA00287FF41C
:10B800009DAE002481E695F87C40012C27D198F864
:10B81000003007A88DF810305B008DF81D30002334
:10B820008DF81E3006F0B4FC0028EAD002210CA8E6
:10B830008DF830108DF8314006F03FFC142006F0F2
:10B840002BFC3028DDD179E698F800308DF81C30DB
:10B8500095F87C301BB1022B07D9032B12D00024A2
:10B8600004AF4FF0010B022678E60CBF072003203F
:10B8700007A906F0F7FC0028C3D09DF81CB00024EF
:10B8800047466BE607A806F0D5FB0028B9D014227E
:10B89000464B07A81A7006F0A7FBECE798F80030B3
:10B8A0008DF81C3095F87C30022B08D0032BD6D1B4
:10B8B00007A806F0BFFB0028A3D01622E8E707A9D7
:10B8C0000420D6E795F87C308DF81C70002B3FF4EF
:10B8D00035AE022B0ED9032B7FF430AE07A806F04D
:10B8E000A9FB00288DD01322304B07A81A70FEF751
:10B8F00001F883E707A806F04BFC002881D014224A
:10B90000012007A906F00AFC78E795F87C308DF84D
:10B910001C70022B0BD0032B14D0012B4FF0000412
:10B9200004AF4FF0010B0CBF02260F2616E607A846
:10B9300006F02EFC00283FF464AF40F2DC5207A969
:10B940000520DFE707A806F075FB00283FF459AF94
:10B950001522C9E70024174F4FF0090BFEE500241C
:10B9600004AF4FF0010B0926F8E5013BDBB254F8B8
:10B9700023001A2185F87D3003F034FC95F87D30E2
:10B9800054F8230003F059FC95F87D30002BECD1DE
:10B99000D5F88030084A9B1A18BF012385F87E30FD
:10B9A00053B0BDE8F08F00BFBF3A0020A43500209F
:10B9B000A535002096BA0108B9EC0008189E0108C8
:10B9C00070B5314C0646D4F88430DB0402D50A2029
:10B9D00004F0A4F8A36F002B55D0226FB24252D8C6
:10B9E00094F86F00B4F87420596860BB01208A5C39
:10B9F00084F86F00002A38D01B78244A013BD2F823
:10BA0000CC2400FA03F3134201D105F095F9012289
:10BA10001F4B1A70FDF730FFB4F8743043B9A36FB1
:10BA20001B78053B012B03D8FEF79CFDC4F888006A
:10BA3000A36FB4F874205B689B5CFE2B10D10023CD
:10BA4000A4F8743070BD00258B5C84F86F5063B12E
:10BA5000284605F071F90E4B1D70FDF70DFFE7E765
:10BA6000FF2B07D1BDE87040CAE4A36FB4F874207F
:10BA70005B689B5C42F2107101FB03630132236738
:10BA8000A4F8742070BD70BD941B002018300020F5
:10BA9000CC1A0020304BF7B519684FF47A732F4851
:10BAA000B1FBF3F106F05AFCFCF7EEF82C4B2D4AF3
:10BAB0002D49127853F8203009882C4806F04EFCA6
:10BAC0002B4B2C4819682C4B2C4DB1FBF3F106F095
:10BAD00045FC2B4806F086FD2A4B2B4A1C882B4937
:10BAE0002B48A4B206F03AFC40F2EC422146294829
:10BAF00006F034FCAE6D6EB3304608F0DBF901465B
:10BB0000254808F0E3FA08F009FC0746D5F8F400E8
:10BB100038B108F0CFF901461F4808F0D7FA08F00D
:10BB2000FDFB0446686A38B108F0C4F901461A48BA
:10BB300008F0CCFA08F0F2FB184B32461988019055
:10BB4000642900943B46A8BF6421154806F006FC12
:10BB500003B0F0BD3746D9E708350020A0BA010888
:10BB6000309E0108EC140020F8140020BCBA010833
:10BB700074020020E4BA010840420F0018000020BF
:10BB800009C10108201C002000500020000800000E
:10BB9000F4BA01081ABB010800247449EC0F002014
:10BBA0003CBB01082DE9F0470546204FDFF88480B3
:10BBB000DFF87C90DFF898A0284607F01BFC0646CB
:10BBC00058B91B4B1B4A93F8B3321B48013B52F840
:10BBD0002310BDE8F04706F0C1BB024639462846AF
:10BBE0000DF05DFA28B1002458F8241091B91348DB
:10BBF0000CE0134806F0F6FC124C134D54F8041FE9
:10BC000019B1284606F0AAFBF8E71048BDE8F0474E
:10BC100006F0E8BC324628460DF041FA013400280F
:10BC2000E2D189F8B3425546C6E700BF90BB010890
:10BC30001830002044A1010884BB0108D8B80108CD
:10BC400095BB010840A1010837C0010809C10108DE
:10BC500058C401082DE9F74F824607F0CBFB494D48
:10BC60000446D5F8CC74F0B9474806F077FB0125B7
:10BC7000464EDFF82C8105FA04F33B4206D00C2334
:10BC800003FB04634046996806F068FB0134122CFC
:10BC9000F1D117B93E4806F0A5FC3E4803B0BDE817
:10BCA000F04F06F09FBC02463B4950460DF0F7F9B5
:10BCB000DFF8D890064668B9384806F093FC384D4E
:10BCC00009EB0603996828460C3606F047FBF02E70
:10BCD000F6D1E2E79AF800304FF000082D2B0CBFA8
:10BCE0004FF0010B4FF0000B4FF00C0304BF0AF1B3
:10BCF000010A04F1FF3403FB08929668504622467D
:10BD0000314601930DF0CBF9019B98BBBBF1000FBD
:10BD10001CD0B8F1120F0CD1224BC5F8CC342248FC
:10BD200006F060FC3146214803B0BDE8F04F06F054
:10BD300015BBB8F1130F02D1D5F8D034EDE70123CC
:10BD400003FA08F31F43C5F8CC74E8E7B8F1120F03
:10BD500003D1C5F8CCB41648E2E7B8F1130F1DBF04
:10BD6000012303FA08F39F43C5F8D07418BFC5F840
:10BD7000CC74F0E708F10108B8F1140FBBD10D48FD
:10BD80008CE700BF18300020A8BB0108A8A3010859
:10BD9000B2BB010809C1010890BB0108BEBB010884
:10BDA000B9BB0108FFFF0300C9BB01088ABB01083A
:10BDB000D2BB0108D8B801082DE9F84F002482460B
:10BDC0002546154EDFF85CB0144F54F806905146E6
:10BDD000484604EB06080DF0B0F988B149465846CC
:10BDE00006F0BCFA0021404606F034FB384606F067
:10BDF000F9FB404606F09EFC384606F0F3FB0135A1
:10BE00001034B4F5276FE0D125B9BDE8F84F0448E8
:10BE100006F0E8BBBDE8F88FBCA5010809C1010820
:10BE2000D8B8010820C601082DE9F74F064607F0EB
:10BE3000E1FA054620B101281ED133782A2B1BD107
:10BE4000744806F0CFFB0024734EDFF8EC91734F7B
:10BE5000A15904EB0608484606F080FA29464046F8
:10BE600006F0F8FA1034384606F0BCFBB4F5276F3C
:10BE7000EED103B0BDE8F08F3D2130460DF001F961
:10BE8000002800F0C180054615F8013C6A1E202BF1
:10BE900030D0AD1B013083469BF800300130202BA1
:10BEA000F9D04FF000085C4CEDB24FEA081959F890
:10BEB00004A009EB0407504607F09CFA51460246DD
:10BEC000009030460DF0EBF8002840F09180009B88
:10BED000AB4240F08D803D7915F0C0030CD0402B73
:10BEE00043D04F4806F07EFB384603B0BDE8F04F24
:10BEF00006F020BC1546C7E758460AF0C9FB0446C1
:10BF00005846FEF74DFF0646B7F90C0007F0D6FF7E
:10BF10000146304608F0D8F90028E2D0B7F90E0003
:10BF200007F0CCFF0146304608F0C4F90028D8D00D
:10BF300005F00F03052B00D02646374B05F03002E5
:10BF40009944102A3046D9F8083033D17421354A43
:10BF500092F81C2401FB023305F00F05052D38D89B
:10BF6000DFE805F03636424237442F4B97F80C8015
:10BF7000002603EBC80804460146034698F814203F
:10BF8000944202D3002BD8D1ABE70029FAD1D8F8DC
:10BF90001000594650F824008DE80C000DF044F8CC
:10BFA0009DE80C00002805BF264601210021012341
:10BFB0000134E5E7202ACFD11C491A4A8C780C219C
:10BFC0006143742492F81C2404FB02121344C3E757
:10BFD00018705146164806F0C1F90021384603B0E2
:10BFE000BDE8F04F06F036BA1880F2E71E60F0E7C1
:10BFF00008F10108B8F1A70F7FF457AF0D4803B05F
:10C00000BDE8F04F06F0EEBA304603B0BDE8F04FA1
:10C01000D2E600BFDABB0108BCA5010809C10108CE
:10C02000FABB010818300020309E0108201C0020B7
:10C03000EFBB0108D8B8010820C6010810B50A4CAA
:10C04000037833B9094B0A489978BDE8104006F0E7
:10C0500085B90AF01DFB022804D8C0B2FDF77CFDAB
:10C060002046EDE710BD00BF58C40108201C002089
:10C070000ABC010838B50C4D0C4C03783BB90A4B8F
:10C080000B4893F81C14BDE8384006F067B90AF075
:10C09000FFFA012807D885F81C04FEF7DDFDFEF73E
:10C0A0003BFC2046E9E738BD1830002058C40108A1
:10C0B0000EBC0108F7B503781BB906F0ADFA03B062
:10C0C000F0BD002401AA1E490AF05DFB2646254664
:10C0D0001B4F40B90B2D18D90B23024619491A489A
:10C0E00006F03CF9EBE744B1012C0AD001AA39462D
:10C0F000002001340AF047FBEBE70AF0C9FA0546D5
:10C10000F4E70AF0C5FA0646F0E7022C0ED1A6F5D0
:10C110007A73B3F57A7F05D94FF4FA634FF47A72E4
:10C120000A49DCE70A4B03EB45039E80084B29468E
:10C1300003EB45039A88074806F010F9BFE700BFF4
:10C1400046BA0108F3B80108B8B8010855CB010890
:10C15000201C00201BBC010870B5134C0546134879
:10C1600006F040FAE069FEF793FB206AFEF7ECFF69
:10C170000F4B1420197800231E4624348B420BDB0E
:10C1800040F2DC50FEF736FA0A4B0B4A15B10B4869
:10C190000B490860DA6070BD00FB03F2125902B16E
:10C1A00016800133EAE700BF201C00202ABC0108EA
:10C1B0005C25002000ED00E00400FA05EFBEADDED6
:10C1C000F04F002010B50C4CE069FEF761FB002336
:10C1D000B4F94A1184F81431C4F8443184F8483170
:10C1E000221D22F8131001330C2BFAD10020FFF787
:10C1F000B3FF0023E36110BD201C002008B5FEF74B
:10C2000073F8FEF729FDBDE808400020A4E708B553
:10C21000FEF722FDBDE8084000209DE701209BE7D6
:10C220002DE9FF41054607F0E5F808282BD16E1EE1
:10C23000EF1D74780AF034FA2044437803F00303C6
:10C24000022B08BF203C06F8014FBE42F1D12C461C
:10C25000DFF8708005F1080714F8016B404631469D
:10C260000CF00FFF20B1314620460CF00AFF20B140
:10C2700006F0D2F904B0BDE8F081A742ECD10E4936
:10C280002846FDF71FFA0D4806F0ACF900230C4CC8
:10C290000C481A1992F8542204A90A44195C013373
:10C2A000082B02F80C1CF4D1002301A906488DF8D4
:10C2B0000C3006F053F8DDE76C32002036BC010884
:10C2C00018300020A19D01088BBB01082DE9F84F13
:10C2D000054607F08FF8344F0446D7F80890B8B9F0
:10C2E000324806F07FF90126314D324F55F82410BF
:10C2F00049B106FA04F313EA090F02D0384606F0F2
:10C300002DF80134F2E72C48BDE8F84F06F06AB981
:10C3100002462A4928460CF0C2FE60B9284806F0B9
:10C3200061F9284C234D54F8041F0029EBD028460E
:10C3300006F014F8F7E72B7800262D2B0CBF4FF0F2
:10C34000010A4FF0000ADFF868B004BF013504F1BC
:10C35000FF345BF82680B8F1000F01D11A48D3E70B
:10C360002246414628460CF09AFED0B90120B04042
:10C37000020601D51548C7E78305FBD4BAF1000FC3
:10C380000AD0FEF791FA124806F02CF94146BDE8B2
:10C39000F84F104805F0E2BF40EA0900B8600E48C7
:10C3A000F2E70136D5E700BF183000203CBC010899
:10C3B000B0A1010837C0010809C1010890BB0108FC
:10C3C00046BC0108ACA10108D8B8010852BC01085C
:10C3D000C9BB01088ABB0108D2BB010810B50E4CCD
:10C3E0000E4805F0BBFFE069FEF752FA02F06EFB63
:10C3F000002384F84C3184F84D31C4F8503102F0F8
:10C4000017FA20B10648BDE8104005F0A7BF642028
:10C41000FEF7FBF8F3E700BF201C002060BC01081A
:10C420006BBC01082DE9FF410A488488C568C688AD
:10C430000789D0F8108002F0DBF98DE880010290C6
:10C4400033462A462146044805F088FF04B0BDE87B
:10C45000F08100BF7402002075BC010870B504466D
:10C4600008460E4606F0C6FF3146024620460CF04E
:10C4700016FE08B1002070BD0AF012F905463046DC
:10C4800006F0B8FF235C1D446B785B07F2D10130E6
:10C49000204470BD064B93F8D42403F2D443002A01
:10C4A000044A06BF012113460021034A06F00EB8D4
:10C4B00018300020D2BC0108D4BC010838B50546AC
:10C4C00006F098FF044690B1112200210A480CF0B2
:10C4D000A3FD2246094928460CF008FE38B1102C6D
:10C4E0002246294628BF102203480CF011FEBDE861
:10C4F00038400120CEE700BFEC340020D2BC010858
:10C500002DE9F04F074600262D4B87B0049103F12B
:10C51000AC0A16F80A302A4A012452F82380294B23
:10C52000DFF8ACB0DB430593274B621E99190B7AF9
:10C53000002B08BF0123934205DC0C36542EE8D1B2
:10C5400007B0BDE8F08F4B689D5C049A1344059AD0
:10C5500023449B5CEA1AD2F1000949EB020993B922
:10C5600000944346194A4946384605F08FFFC5B93D
:10C570007B0606D400944346144A4946384605F0E3
:10C58000A5FF0134D0E703F00F021B0940330292EC
:10C590000193009443465A464946384605F076FFD3
:10C5A000E5E705F00F032D09403502938DE83000D3
:10C5B00043465A464946384605F088FFE1E700BF42
:10C5C00044A0010818300020F0A0010835BF010880
:10C5D0004BBF010838B50C240A4B0D4604FB003450
:10C5E00094F8AC20084853F8221005F0B7FE94F8F0
:10C5F000B4302BB1691C0548BDE8384005F0AEBE2B
:10C6000038BD00BF44A00108BBBB010873CF0108BF
:10C610001FB5074B074A0293074B08490193084B84
:10C6200008480093084B05F099FE05B05DF804FB3F
:10C630002AB1010810B1010821B1010863B2010853
:10C6400015B1010863BF01085DB201082DE9F04F83
:10C6500000252F46A9465C4E8BB05C4B1A68002320
:10C66000934223DB01350A2D06F13406F5D1584BF0
:10C6700093F8FA31BBB14FF47A73564991E805004B
:10C680008968B0FBF3F35209534805F067FE97FB46
:10C69000F5F399FBF5F105FB137705FB1192009774
:10C6A0004E4805F05BFE0BB0BDE8F08F4C4951F8E9
:10C6B00023108E4263D00133D2E74346079A01210B
:10C6C000484805F04BFE5C46BAF1000F50D041F2ED
:10C6D00088314FF47A700AFB0411B1FBF0F0099B2A
:10C6E0005B091DBF41F288324FF47A7103FB0422CB
:10C6F0001A4618BFB2FBF1F23549052D91F8FA112F
:10C700001CBF8144BF18002934D04FF47A7E0899A9
:10C71000B1FBFEF104910A2192FBF1FE01FB1E2206
:10C72000039290FBF1F201FB120100920191CDF80E
:10C7300008E0524621462C4805F010FE012D91D10B
:10C74000234B93F8F831012B8CD95A460799274887
:10C7500005F004FE86E738B107F0ACFB014624483B
:10C7600007F0B4FC07F0DAFD04464246294627E00C
:10C770005046B4E721461F4805F0F0FDDEE7736838
:10C78000012D0793336BD6F800800893B36AD6F86F
:10C790002CA00993706ADED138B107F08BFB0146FB
:10C7A000134807F093FC07F0B9FD094B834693F853
:10C7B000F831012B90FBF3F47FF67FAF4246012165
:10C7C0000D4805F0CBFD7FE7180000200C15002078
:10C7D00018300020741D0020D8BF0108FABF0108DE
:10C7E000101500208EBF0108A0BF0108C6BF0108B8
:10C7F00000247449D2BF01087FBF01082DE9F04F22
:10C8000089B0044606F0F6FD074630B901464120DE
:10C81000FFF776FE09B0BDE8F08F02468E4920464C
:10C820000CF03DFC8D4D064600284DD18C4805F09E
:10C8300095FD8C4CDFF86C92DFF86CA2DFF86C820F
:10C8400004F58477A2882168B2FA82F201F14041AE
:10C85000A379A1F58431890A413155F82330C2F119
:10C860001F02484605F07AFDE17911B1504605F006
:10C8700075FD4046083405F071FDA742E2D17A48C3
:10C8800005F06CFD794805F069FD794CDFF82082F0
:10C89000DFF82092DFF820A2237E01363246012104
:10C8A000404655F8237005F059FD627E39463AB18D
:10C8B000504605F053FD072E04F11C04ECD1A9E706
:10C8C000484605F04BFDF6E707AA6A49204609F0FD
:10C8D0005AFF4FF0000806464FF00C0A05F1AC096C
:10C8E0000AFB08F414F809303A4655F8231030468C
:10C8F0000CF0D5FB40B108F10108B8F1070FEFD1FA
:10C900005D4805F06FFE85E707AA5A4909F03BFF2D
:10C91000064609F0BDFE2C4494F8B4300746BBB976
:10C92000002823DC0C2303FB0855D5F8B0303478FD
:10C930003B440193002C00F08C80504930460CF0B1
:10C9400073FBE8B9019B18704D4805F007FD61E7DE
:10C95000002805DD1A46BA420ADA002B08BF012377
:10C9600001224849484805F0F9FC53E70122F2E763
:10C9700007AA4049002009F006FF013F0646D1E71B
:10C98000A4F14105EDB2072D04D9A4F16105EDB282
:10C99000072D5ED8701C09F07BFEC3B20F2B8146B9
:10C9A00057D86C1C40EA0414E4B2204602F0F8FBAD
:10C9B00000284ED04FF0000B23094033049304F0BD
:10C9C0000F0305930C21314A002601FB0B2A2AE0B4
:10C9D000DAF804209119925DA24223D1D84504D1FE
:10C9E000FAB2B2421ED000220A70059A0499284871
:10C9F00005F0B4FC5FFA8BF30293F3B21946029888
:10CA00000393FFF7E7FDD84509D1224805F0A6FCBE
:10CA100002980399FFF7DEFD1F4805F09FFC1F48B1
:10CA200005F0E0FD01369AF80820002A08BF01222F
:10CA30009642CDDB0BF1010BBBF1070FC2D15FFAC0
:10CA400089F205F14101164805F088FC019B1C7034
:10CA5000E0E605F0E1FDDDE690BB010844A0010839
:10CA60002AC00108801D002007C101083BC0010841
:10CA70008802002046BA01085DC0010854BD0108C3
:10CA800067C00108F3B80108B8B80108F0A00108B0
:10CA90006FC0010893C0010896C001087FB9010862
:10CAA000A0C001082FC0010874CF010809C1010806
:10CAB00042C001088ABB010854C001082DE9F04FAB
:10CAC0000E4695B073490446FFF7C8FC054600289A
:10CAD00040F0BB8070492046FFF7C0FC05460028A7
:10CAE00040F0B5806D492046FFF7B8FC05460028A8
:10CAF00040F0AF8020466A49FFF7B0FC00280546A9
:10CB000012BF0824254601240EB144F010046548E4
:10CB1000FDF78EF964492846FFF7A0FC08B144F000
:10CB2000200414F0090F00F0DD820020FFF770FDF3
:10CB300004F01803182B02D15C4805F053FDDFF810
:10CB400064815B4D2046FFF7A5FC41462046FFF778
:10CB5000D7FC98F8B33295F8B362564FA6EB0309A9
:10CB6000D9F1000646EB090607EB83033146D3F8FB
:10CB7000FC30514A204605F089FC95F8B332314625
:10CB800007EB8303D3F8FC304B4A204605F09EFCAC
:10CB90000021E86807F07AFB4FF00106CDF820800D
:10CBA0000795099700B90646444A06F00101204658
:10CBB00005F08CFC4249204604F005FC4149204622
:10CBC000FBF76EFE079B002793F904113E4AB1FA6A
:10CBD00081F12046490905F079FC32492046FBF7EE
:10CBE00011FC079BDFF8E4B0D3F80880089BDFF85E
:10CBF000E0A09D685BF827606EBBDFF8D8A068EA0C
:10CC0000050B324B53F82690B9F1000F64D0012781
:10CC1000B7403D4209D01BEA070F4B46524614BFAE
:10CC200001210021204605F031FC17EA080F0AD047
:10CC300065EA08033B4252464B4614BF01210021DE
:10CC4000204605F043FC0136DBE701245CE70224C3
:10CC50005AE7042458E74FF0010965EA080309FA86
:10CC600007F913EA090F14BF012100213346524688
:10CC7000204605F00BFC68EA050313EA090F52464B
:10CC8000334614BF01210021204605F01FFC013767
:10CC9000B0E700BFC7C00108C3C40108CEC0010887
:10CCA000D4C001082C2B0020D8C00108E5C0010821
:10CCB0001830002044A00108F0C00108FBC00108A2
:10CCC000382B00209E2C00200CC10108B0A10108C7
:10CCD0001BC1010829C10108079B4D46D3F8CC743C
:10CCE000089BDFF89893D3F8CC34DFF894A37B400B
:10CCF000DB430B9301260B9A06FA05F31A4214BF85
:10CD0000B0464FF000083B400A934FF00C03D34A63
:10CD1000414603FB0523D3F808B014BF4A465246E8
:10CD20005B46204605F0B2FB0A9A5B46002A14BF18
:10CD300052464A4641462046354405F0C7FB122D6F
:10CD4000D8D14FF41573C64D079AA3F51571D25C6F
:10CD5000485D14A9114401F8200C089914AFC95C6E
:10CD60000F4407F8100C2EB1A2EB0108D8F1000611
:10CD700046EB08060133B3F5177FE5D14FF0000805
:10CD800010ABB84A314620468DF83880B64F05F0D2
:10CD90007DFBDFF8F0B20CABB24A3146204605F01D
:10CDA00095FBB249204604F091FBD9463D464FF031
:10CDB000190A95F81D3499F81D24934299F82034E6
:10CDC00040F0A58195F81E0499F81E14884240F0A1
:10CDD0009E8195F81F0499F81F14884240F09781AE
:10CDE00095F82064A6EB030CDCF1000646EB0C067C
:10CDF0000AFB03F303F56173039399F81F3431467B
:10CE00000AFB03F303F56173029399F81E3420467D
:10CE10008DE80C004346964A05F038FB95F820341F
:10CE2000934A0AFB03F303F56173039395F81F34E8
:10CE300031460AFB03F303F56173029395F81E3440
:10CE40002046019395F81D3409F1040900934346E7
:10CE500008F1010805F03AFBB8F1140F05F10405DB
:10CE6000A7D14FF000094FF0190A089E7E4D95F8A2
:10CE70006D3496F86D24934296F8713440F04981F0
:10CE800095F86E0496F86E14884240F0428195F849
:10CE90006F0496F86F14884240F03B8195F8700457
:10CEA00096F87014884240F0348195F871149942D4
:10CEB00040F02F8195F8728496F87214A8EB010E59
:10CEC000DEF1000848EB0E08059396F870344146F1
:10CED000049396F86F3420460AFB03F303F561735D
:10CEE000039396F86E3401920AFB03F303F5617322
:10CEF000029396F872345F4A00934B4605F0C6FAE7
:10CF000095F871345B4A059395F870344146049363
:10CF100095F86F3420460AFB03F303F5617303931E
:10CF200095F86E3406360AFB03F303F5617302933A
:10CF300095F86D340635019395F86C3400934B46A3
:10CF400009F1010905F0C2FAB9F10F0F8FD14FF0C5
:10CF50000009089DDFF81081DFF82CA1B8F8A022A5
:10CF6000B5F8A0329A42B5F8A22240F0D580B8F8C0
:10CF7000A262B01A464246410192009352464B4685
:10CF80003146204605F082FAB8F8A23252460193A3
:10CF9000B8F8A0323146009320464B4609F101090A
:10CFA00005F094FAB9F1040F08F1040805F104053D
:10CFB000D4D10026DFF8D490DFF8D4A097F87C22F3
:10CFC0009BF87C329A4240F0A98097F87D529BF8FA
:10CFD0007D12691A4D424D41022A40F0A1804FF066
:10CFE00019089BF87D22294608FB02F202F2EE2284
:10CFF0000192099A2046134493F8E0315246009377
:10D00000334605F043FA97F87D32099A08FB03F896
:10D0100008F2EE23019397F87C322946134493F8E3
:10D02000E031524600932046334605F04FFA013670
:10D03000122E07F102070BF1020BBFD1214600208F
:10D0400004F0CEFA14F0080F0B4E00F08280002599
:10D05000079BDFF8408093F81C741DE0A8A301082B
:10D06000A19D010836C1010818300020042E0020BF
:10D070003FC10108F9B80108741D0020AEC00108C5
:10D08000BAC001082C2B00209FB8010866C1010816
:10D0900054C1010858C40108E8B2214604F0E4FA7A
:10D0A000D6F814312146002093F84C9004F0F6FA9B
:10D0B0002146012004F0F2FA2146022004F0EEFAA3
:10D0C0004846FCF749FD01354046FEF7B7FF022D03
:10D0D000E2D13846FCF75EFD2548FEF7CBFF254838
:10D0E00005F080FAA20705D5234B214693F81C04CE
:10D0F00004F0BAFA630707D5204B2146D3F8143160
:10D1000093F84C0004F0CAFA15B0BDE8F08F002681
:10D110006EE64FF00008D7E600262DE700255BE716
:10D12000099A2946134493F8E0314A460093204671
:10D13000334605F0ABF997F87C32099A2946134437
:10D1400093F8E0314A4600932046334605F0BEF995
:10D150006DE7079B214693F81C0404F085FAD6F886
:10D160001431214693F84C0004F098FABAE700BF56
:10D1700058C4010875C1010818300020741D002032
:10D1800070472DE9F0412D4D2C68228AD2B9267ABC
:10D19000042E17D12A480378012B0FD1294B196887
:10D1A000294B89B221F007010B445B001A60302340
:10D1B000027043802B681E72BDE8F08110230726A1
:10D1C0004380F7E7B4F81480A36942458CBF022678
:10D1D0000426904528BF90461FFA88F7384698479E
:10D1E0000021184B08F101021B6852109BB223F07A
:10D1F000070303F1005303F540535B001B689BB228
:10D2000003F1005303F540535B008A4210D13946C5
:10D210000020FAF74BF83022238ADB1B2382638A33
:10D220001F44074B67825A804FF440529A80C1E7EF
:10D2300030F802EB23F821E00131E6E7282B00204B
:10D240008C1E0020505C00400230002008B50B4BC3
:10D25000002093F82C10FAF707F8094B1B68187A8E
:10D26000082805D14FF48052064B9A8010225A802C
:10D27000A0F109035842584108BD00BF8C030020AB
:10D28000282B00208C1E0020704770477047FEE757
:10D29000FEE7FEE77047202938B50C461DD8D1B10E
:10D2A000631C124AA1B25B100432C3B90120F9F722
:10D2B000FDFF0F4A1368234413600E4A136823F4DA
:10D2C000E04323F040039BB283F0300343F4004378
:10D2D00043F080031360204638BD2024E0E730F897
:10D2E000025B013B22F8045CDEE700BF8061004086
:10D2F0000C350020045C0040002330B51D46DCB234
:10D30000A24200D830BD040F092C94BF303437340A
:10D3100001F8134001EB4304000165700133EEE7AF
:10D3200070B5002240F60F7648F2800502F1805376
:10D3300003F5B8539B00196842EA050431400132F5
:10D340002143042A1960F1D1024B40F0800018609B
:10D3500070BD00BF4C5C00402DE9F347994D9A4CDD
:10D360002B689A4E9BB2E380E3883288134098057D
:10D3700006D54FF6FF532B60237A0133DBB22372BD
:10D38000E3881A40110440F11382002348F60F7815
:10D390008F4FDFF85092ADF802302B689AB2190423
:10D3A000E28040F10582E38803F00F036372002BF3
:10D3B00040F0FD82D9F800309BB2A380A38803F02F
:10D3C00030036380A38803F44053A380D9F800306E
:10D3D00023F4804323F040031B041B0C83F400530D
:10D3E00083F0200343F4004343F08003C9F8003086
:10D3F000E38813F0100FD9F8003028D123F4E1436B
:10D4000023F070031B04734F1B0CC9F800303B68FA
:10D410001A7A022A01D0042A06D1FFF7B2FE3B682D
:10D420001B7A3A6813729CE1062A0ED15A78052AB3
:10D4300008D11A78520605D1D878FFF771FFE36852
:10D440001B6A984723699B6898470823E9E79BB2C2
:10D45000ADF80230BDF80230180540F11982D9F854
:10D4600000305D4923F070031B051B0DC9F8003027
:10D470000A685A4B92B222F007021344554F5B00E0
:10D480001A683B688846187A092817D092B2520069
:10D4900002F1804202F5C04211781970517859703A
:10D4A0009088C1B2090241EA102159801089C1B2A5
:10D4B000090241EA102199809289DA8001221A72C8
:10D4C000DA8893F80190002A40F0DC801A7812F094
:10D4D0007F0258D1B9F1090F16D1DA78012A08D99B
:10D4E000236948465B699847032840F0C7800923B1
:10D4F00097E799780029F3D199880029F0D19A7299
:10D50000E3685B6898470FE0B9F1050F1AD193F90A
:10D510000320002A99DB9A78002A96D19A88002A5B
:10D5200093D19B7A002B90D1D8F800202C4B92B24B
:10D5300022F00702134400225B001A60302363804C
:10D5400006236EE7B9F1030F0CD1DA78012AC7D1AF
:10D550009A88002AC4D15A7A42F020025A72E368AB
:10D56000DB69CFE7B9F1010FBAD1DA78012AB7D177
:10D570009A88002AB4D15B7A9906B1D508F0E4FF05
:10D580000028D1D0ACE7012A2ED1B9F10B0FA7D1D9
:10D590002269D9789269587990473B689A7A002A2B
:10D5A0009ED000289CD11A79002A99D19B78002B13
:10D5B00096D1E368DB6898473B685A79DA72DA7883
:10D5C0001A73B1E7445C00408C1E0020CA3A002068
:10D5D00038A20108282B0020505C004004300020B5
:10D5E00002300020005C0040022A7FF479AFB9F1DC
:10D5F000010FC3D0B9F1030F7FF472AF587920F057
:10D60000800E4FEA8E0202F1804101F5B8410968AF
:10D6100040B20028B4BF01F0300101F44051BEF126
:10D62000030F3FF65DAFB3F802E0BEF1000F7FF4E9
:10D6300057AF00293FF454AF9B7A002B3FF450AF13
:10D6400002F1804202F5B84213680028B5BF23F406
:10D65000E04323F4804323F0400323F07003B5BF7D
:10D660009BB29BB283F0100383F4805343F40043D6
:10D6700043F080031360E3689B6943E700287FF46D
:10D68000E4AE51E7B9F1060F13D11A7852065ED114
:10D690009B78012B03D12369DB69FBB957E0022B8F
:10D6A00002D123691B6AF8E7032B50D123695B6A17
:10D6B000F3E7B9F1000F40F09D805988002946D169
:10D6C0005A6822F47F42B2F5003F40D11A7812F036
:10D6D0007F0219D19B88002B39D1A84B4FF000084D
:10D6E0003A684046A2F812809361984740464FF648
:10D6F000FF713B681A8A8A4231D0022802D0002A80
:10D7000040F09C8008222BE0012A09D12269587937
:10D7100092699047D8B93B689B7A002BDDD116E01F
:10D72000022A14D15A7902F00F018B0003F18043D1
:10D7300003F5B8431B6812F0800F14BF03F03003E9
:10D7400003F44053032902D812F0700FE5D03A6871
:10D75000236950781B6998470328C8D13B68092280
:10D760001A72FFF773FD864B1B68A28823F480436F
:10D7700023F04003D1044FEA0343A2884FEA134346
:10D7800048BF83F480539204628848BF83F40053F7
:10D79000D706628848BF83F01003900648BF83F025
:10D7A000200343F4004343F08003754A9BB21360A7
:10D7B0003288E38813405A0505D54FF6FF332B60B6
:10D7C000704B5B689847E38832881340DB0440F174
:10D7D00028814EF6FF732B6000232375237D052BD4
:10D7E00000F21481DFE813F00E011701200124017B
:10D7F0002D013801B9F1080F04D11B785B06A6D1C1
:10D80000614B6BE7B9F10A0FA1D11A7802F07F02E0
:10D81000012A9CD19A7A002A99D05988002996D158
:10D820005A6822F47F42B2F5803F90D1226958793C
:10D830009269904700288AD1544B4FE793F9001022
:10D8400000291FDAD98801910198824208D9019AEA
:10D850001A82226992F82C209A82FFF792FC80E7C4
:10D860008A42F6D2216991F82C00824202D200222B
:10D870002270EEE792FBF0F100FB1122002AE8D1C2
:10D880000122F5E703221A724FF44053A38068E7A0
:10D89000BDF8023018047FF580ADD9F800303C4A5D
:10D8A00023F070031B051B0D1768C9F800303B7A85
:10D8B0009146022B79D0042B77D0032B01D0052B76
:10D8C0006ED1BB693A8AC3B93B8A43B100214FF498
:10D8D00040530846A380F9F7E9FC30236380BB8AF4
:10D8E000398A8B42D9F8003036D803221A72D9F817
:10D8F00000301B7AD9F8002094E5002AE4D0B7F86C
:10D900001480904528BF90461FFA88FA50469847E1
:10D9100000213B8A08F10108A3EB0A033B827B8AC2
:10D920004FEA68089A441B4BA7F812A01A681A4BD2
:10D9300092B222F0070213445B001B689BB203F112
:10D94000005303F540535B008845BDD053F82120B8
:10D9500020F811200131F7E709B10522C6E70622B8
:10D960001A720C4B1A680D4B92B222F00702134444
:10D970005B00196030236380B9E700BF497100087C
:10D98000005C00408C030020FD710008D971000884
:10D99000282B0020505C0040043000200230002082
:10D9A000072B02D12369DB6898470823A2E79A0076
:10D9B00002F1804202F5B842116889B2ADF8021056
:10D9C000BDF80210090409D51168013B21F070016E
:10D9D0000905090D116057F823309847BDF802304A
:10D9E00018067FF5DAAC627A930003F1804303F501
:10D9F000B843196807EB820201EA080119609369CC
:10DA00009847CAE4A3691BB903F0A2FE062300E00D
:10DA10000523237505E003F09BFE042323750123F2
:10DA2000A36102B0BDE8F087022363750323F0E72A
:10DA3000637D013BDBB26375637D002BF1D1042371
:10DA4000E7E70F4A13689BB243F010031360052306
:10DA500023750A236375E4E7637D013BDBB26375DD
:10DA6000637D03F0FF01002BDBD14FF6EF73044A17
:10DA700010680340136006232375A161D1E700BF3E
:10DA8000405C00402DE9F843A14EA24A33680546A8
:10DA90001A4278D045F207229F4C2368C31A93425A
:10DAA00071DDA3792060B4F8048043B94CF25032A0
:10DAB0009A4904F1080005F07FFB0123A371984BFC
:10DAC0009A78984B33F8129094F824301FFA89F919
:10DAD000022B08BFA4F82690484606F0EBF9014651
:10DAE000914805F031F906F03FFC80B2FAF70AF9E7
:10DAF0008E4B074618804846FAF704F98C4A94F88A
:10DB000024E01378BEF1020F08BF2785032BA08005
:10DB1000884B894957D11B785B070AD40B681B7C5B
:10DB2000BB421DD2A0EB080808F10208B8F1040FAF
:10DB300016D80023D1F800C013709CF8033090FB76
:10DB4000F3F001300828A8BF08207C4B18709CF81F
:10DB5000053080B24343E3859CF804305843208667
:10DB6000BEF1020F04D113786385744B1B78A38533
:10DB700009684B7C3BB11378012B44D03BD3022B7B
:10DB80004DD0FAF78FF8D6F8008018F0082F00F083
:10DB9000BC8045F20723604E746B2C1B9C4240F303
:10DBA000B4807563FAF770F8032800F0A980624F1B
:10DBB000D7F8009099F80C30032B00F2A680DFE82C
:10DBC00003F09F32739F93F800C01CF0040CC7D180
:10DBD0000B681B7CBB42C3D3A0EB080002300428B7
:10DBE000BED803231370554BA4F82EC083F800C091
:10DBF000A4F830C0B4E7E38D89795B1A9F42C0DC9A
:10DC000001231370BDE7238E89795B1A9F4201DCE3
:10DC10000223F6E7E38DBB42B3D20023F1E7238E64
:10DC2000BB42EDD3ADE796F8383043B94CF25032F1
:10DC30003A49434805F0C0FA012386F8383040F6E7
:10DC4000E4464FF47A75364BDA79364B33F81200E6
:10DC50003A6880B206FB00F1B2F90A30B2F9082046
:10DC6000C3EB11336B4393FBF2F3364A136006F0B8
:10DC700021F90146324805F067F806F075FB80B2DD
:10DC80003A687043B2F90A30C3EB10304543B2F939
:10DC9000083095FBF3F52C4B1D602046F9F7DAFFB1
:10DCA000BDE8F843FAF70DB8224B28481B78B9F9BC
:10DCB0000A60244D5B07B0F8EE102E601CD500F50D
:10DCC000157004F0B3FD224BB3F90620A2F57A7269
:10DCD00018B918F0100F18BF0022322102FB02F30E
:10DCE00093FBF1F31A44B9F9083053434FF47A72B5
:10DCF00093FBF2F333442B602A68134B1A60CCE792
:10DD00000023114A13600F4A1360BDE8F88300BF77
:10DD10000017002002000008A81E0020CDCCCC3E39
:10DD2000240B0020380B0020B01E0020F814002027
:10DD30000415002028260020F0140020EC140020F8
:10DD4000E41E0020FC140020600C0020183000208D
:10DD5000500C00202DE9F04FBD4E8DB03578002DD0
:10DD600000F0B580BB4B1868002870D0FCF790FD20
:10DD7000DFF81083B84DD8F8000003F01FFF00282B
:10DD800065D0D8F8000003F013FF0928B34C01D088
:10DD90003F2853D14FF0000B5F46DFF8D092D4F804
:10DDA00000A009F58073BAF1000F08D05246D9F8E7
:10DDB0000010284601930BF072F9019B08B9CB467D
:10DDC0007FB309F108099945EDD397B1D7F800E081
:10DDD000DBF800C023681EF803001CF80310814222
:10DDE00007D15A1CF9B92D2B1DD820202260E854E8
:10DDF000A95423680BB15F4509D0994804F0F2FBA0
:10DE00005F4513D9974804F0EDFB4FF0000A2368F3
:10DE10009A45B0D215F80A0004F027FB0AF1010A6E
:10DE2000F5E74F46CDE7E8542260D3E757F8080BF3
:10DE300004F0D8FB092004F018FBE1E72368002B6D
:10DE400040F0B181042805D18348FEF7BBF90DB03D
:10DE5000BDE8F08F0C2840F0D181834804F0C2FB6C
:10DE6000804804F0BFFB86E701220B46AEE1591E55
:10DE7000685C2028F8D002B1236000227B4FEA546E
:10DE800007F5807939682846FEF7E8FA30B908378F
:10DE90004F45F7D3764804F0A5FB03E04F45F9D290
:10DEA0007B689847002395E12F2B3FF664AFA0F1E4
:10DEB0002002D2B25E2A3FF65EAF13B920283FF4AB
:10DEC0005AAF5A1C2260E85404F0CFFA53E7694F66
:10DED000694C97F80080DFF8B09108F0040854F816
:10DEE000093C002B40F046810135032D04F1CC04A0
:10DEF000F5D1ACE7012A05D14D2808BF022318BF90
:10DF000000234DE1022A03D13C2808BF0323F6E792
:10DF1000032A40F0C380C0284FF0000240F2B680D0
:10DF200004F8012C14F8013C062B40F025814FF039
:10DF3000000A524B0DF1180E93E8070014F8043C48
:10DF40008EE8070023440A930CAA14F8023C42F816
:10DF500024AD714609A80994ADF82C30ADF82EA077
:10DF6000F2F7D6F8002862D0069A54F8090C079206
:10DF7000434A069203F011FE2423069A07998DF86E
:10DF80001030A1EB020B4D235A468DF81130BDF92C
:10DF90002230FF2AA8BFFF22591C14BF3E23212391
:10DFA000BBF1FE0FCDF814A0CCBF4FF0070A4FF025
:10DFB000050A8DF81230BDF820308DF813208DF849
:10DFC00014305246C8BF4FEA2B2304A954F8090C59
:10DFD000C4BF8DF816308DF815B000F00AFF04AB01
:10DFE00003EB0A0200230DF11301914240F0BA80C5
:10DFF000BBF1000F8DF80B300EDD5A46069954F830
:10E00000090C00F0F6FE069B9DF80B209B445B4537
:10E0100040F0AC808DF80B2054F8090C01220DF172
:10E020000B0100F0E6FE54F8090C03F0B1FD0023EB
:10E03000DDF80CB004F8013CBBF1000F3FF454AF25
:10E0400054F8090CFDF780F854F8090CD8474BE751
:10E05000681D00203C1C0020341D0020641D002091
:10E0600024C4010829C401082EC40108A8A201087B
:10E0700039C40108282600207118002074A2010864
:10E08000D83A0020401C0020F04F002004F8040C77
:10E0900004F8052C04F8030C042381E0042A09D1B8
:10E0A00014F8032C04F8020C80EA020304F8033C81
:10E0B000052375E0052A7FF435AF14F8050C14F834
:10E0C000042C14F8031C82420ED9421C04F8052CBF
:10E0D000CC228AEA010104F8031C4A4902FB05121A
:10E0E000024482F809A01DE7514501D1062357E0FB
:10E0F000002355E0B8F1000F3ED1232825D101229D
:10E1000054F8091C3270404A40481160404A9165F9
:10E110001166802182F864103E49D06502F15C00EE
:10E1200008603D4982F8658091F8FA113B4800315A
:10E1300018BF012182F8E81004F054FA384804F0BE
:10E1400051FA3A7842F002023A70364A126892F86E
:10E150002A20524501BF344BC9F80030334BC3F875
:10E160000CB0DFE611F8010B43403EE713F8011B4A
:10E170004A404CE7DFF8C0B054F8090C03F01EFD2C
:10E1800000283FF4B1AE54F8090C03F011FD14F867
:10E19000012C8246002A7FF4ADAE2428AAD10123A7
:10E1A00004F8013CBEE60C283FF457AE0A2801D023
:10E1B0000D281AD11E4804F015FA232128460AF02A
:10E1C00060FF08B1401B206000222368002B7FF411
:10E1D0004EAE02B123603022002128460AF01CFF17
:10E1E0003378002B7FF43CAE31E67F287FF45CAEC1
:10E1F0000022013B2360EA540E4832E67F287FF478
:10E2000056AEB8E568180020401C002085170108AC
:10E21000A81E00203C1C00201830002059C4010812
:10E2200029C4010864350020EFBEADDE00ED00E03A
:10E2300009C1010855C401080400FA052DE9F84395
:10E240008A4D6B6828469847002800F00C8101230E
:10E2500005F12C0785F83C3039460023844C05F144
:10E260000A0294F8246004F1260E042E04BF1088DC
:10E270002EF8130032F9020B0133032B41F8040F7F
:10E28000F3D1B4F8EA30002B40F0A580794E697CD8
:10E290007948F9F7BBFB3388002B44D00023BC46F8
:10E2A0001A46D4F840E1DFF8F08131884FEA83095B
:10E2B000B1F5C87F08BF48F8232058F80910084670
:10E2C000DCF804104CF8042F084448F809002EF834
:10E2D00013200133032BE8D13388012B20D14FF4D5
:10E2E000C870D4F8443103F1C80191FBF0F1AEF8E5
:10E2F0000010D4F84811C83191FBF0F1AEF80210CB
:10E30000D4F84C312989C83393FBF0F35B1AAEF88B
:10E3100004305A4BA3F82022A3F82222FBF74EFC2C
:10E320003388013B3380564B1B685B0740F18A8082
:10E33000544E3388322B63D1D4F840311A88A4F874
:10E3400050215A889B88A4F85221A4F854314B4B91
:10E35000B3F82022B3F82232A4F85621A4F8583199
:10E360000020D4F84031484AA3F1020E03F1040C16
:10E370003188322908BF10601368796847F8040FA4
:10E380000B4442F8043B2EF8020FF445F0D13388D9
:10E39000012B1CD14FF000013C4A0C2011703C4A6B
:10E3A000137001F0BBFBD4F84031B4F850211A804F
:10E3B000B4F852215A80B4F854219A802F4BB4F803
:10E3C0005621A3F82022B4F85821A3F8222233883A
:10E3D000013B338016E0B8460026DFF8C090D8F83D
:10E3E000040005F06BFD014609EB060004F0ACFCEF
:10E3F00008F03CFB1C36542E48F8040FEFD145E7DB
:10E40000002BADD1234B1A78E2B1002232201A70D2
:10E41000D4F85C31D4F8401193FBF0F30B80D4F8BE
:10E42000603193FBF0F34B80D4F8643193FBF0F34D
:10E4300028891B1A8B80114BA3F82022A3F82222D3
:10E44000FBF7BCFBD4F840312A6BB3F90010521A29
:10E450002A63B3F902106A6B521A6A63B3F9042093
:10E46000AB6B9B1AAB63BDE8F88300BFB0250020FF
:10E47000A81E0020780B0020E02500201830002086
:10E48000001700207A0B0020042000207C0B0020C5
:10E49000740B0020750B0020EC1F0020941F00203F
:10E4A0004FF400630381704738B5054600BF064C42
:10E4B000206800F0C2FE2946044800F010FF2068E2
:10E4C00000F0C0FE00BF38BD00070020003800404B
:10E4D0002DE9F041804616460F460B4C0B4D206847
:10E4E00000F0ABFE48F08001284600F0F8FE3B4605
:10E4F00000223146284600F0C4FE206800F0A2FE4B
:10E500000120BDE8F08100BFDC06002000300140A2
:10E510002DE9F043C36A85B004460BB3187800F0C8
:10E520003FFE0027202305468371C771062100F0B6
:10E5300059FE8E4B6361AB88B3FA83F3C3F11F03BB
:10E540005A1C40F0C080AB880122B3FA83F3C3F1B8
:10E550001F0312FA03F31FBF85490A6813430B60B8
:10E56000844E3778002F70D1834D80212B886B200B
:10E5700023F040031B041B0C2B802B8823F0380353
:10E580001B041B0C43F038032B802B889BB243F0F9
:10E5900040032B80F6F708FF9620FCF736F803219E
:10E5A0006820F6F701FF9620FCF72FF803216B2077
:10E5B000F6F7FAFE0F20FCF71DF810216A20F6F797
:10E5C000F3FE0F20FCF716F839466C20F6F7ECFE48
:10E5D0000F20FCF70FF894F824101920F6F7E4FE4A
:10E5E0000F20FCF707F818211B20F6F7DDFE0F209F
:10E5F000FCF700F818211C20F6F7D6FE0F20FBF7D9
:10E60000F9FF10213720F6F7CFFE0F20FBF7F2FFBE
:10E6100001213820F6F7C8FE0F20FBF7EBFF2B880F
:10E62000012023F040031B041B0C2B802B8823F0BC
:10E6300038031B041B0C2B802B889BB243F0400338
:10E640002B80FBF7D7FF012333704B4D1A202B880B
:10E6500023F040031B041B0C2B802B8823F0380372
:10E660001B041B0C43F038032B802B889BB243F018
:10E6700040032B8094F82210F6F796FE0120FBF75A
:10E68000B9FF2B88204623F040031B041B0C2B8072
:10E690002B8823F038031B041B0C2B802B889BB288
:10E6A00043F040032B80F6F7C3FCE38B5BB20133EE
:10E6B00006D1A38B5BB2013302D10620FBF7D6FF54
:10E6C00005B0BDE8F0834FF00F0C4FF00109DFF803
:10E6D000B4802A4908EB0302D67904F1140241F808
:10E6E0002320DAB202F0030002F0FC0202F18042C1
:10E6F00002F580322968D2F808E080000CFA00FCAC
:10E700002EEA0C0E01F14041C2F808E0A1F5843177
:10E71000D2F808E0C1F38721814041EA0E019160FF
:10E72000134A09FA03F35361029308230DEB030024
:10E730008DF80D308DF80C708DF80E9002F068FD9C
:10E740000F4B9A5DF02A7FF7FEAEF0229A5518F82B
:10E75000063001A88DF8043003238DF806708DF87B
:10E7600005308DF80790F8F7BBFFECE6B7500008CE
:10E7700000040140102000200030014064200020EF
:10E78000E805002080A20108094A0A4913781844C4
:10E79000C0B210F0800F18BF803810701078134688
:10E7A0000A78904202BF00220A701A70704700BFB8
:10E7B0006D1D00206C1D002010B50A4B0A4A1B7805
:10E7C00042609C18094A0460127893429DBFD31A94
:10E7D0000B600023C3F1800392BF4B600B604A6063
:10E7E00010BD00BF6D1D00204D2100206C1D0020BC
:10E7F0001FB502A86946FFF7DFFF044B00981B68AE
:10E800001844019B184405B05DF804FB701D0020FE
:10E81000054B1878054B1B78984236BFC3F180032F
:10E82000C01AC018704700BF6C1D00206D1D00206D
:10E8300037B5104C2078C0B105238DF80030002387
:10E840008DF8013000BF0C4D286800F0F6FC022363
:10E850006A4601A9094800F014FD286800F0F2FC9E
:10E8600000BF9DF8050000F00100207080F001005D
:10E8700003B030BD0407002000070020003800402E
:10E8800070B50646044C2568FFF7D2FF18B9236817
:10E890005B1BB342F8D970BD083500202DE9F04F5D
:10E8A00087B0019300238246029103920093039A5A
:10E8B00093420CDB019B002B40F08880FFF7B8FFF0
:10E8C000002840F08380019807B0BDE8F08F029ADD
:10E8D000009952F82320013311440091E7E7022206
:10E8E0008DF814201A0C8DF8152006201A0A8DF8C0
:10E8F00016208DF81730FFF7C3FF0620FFF7D4FD71
:10E900000123334A137000BF4FF00008D146274659
:10E91000304B186800F091FC042305AA00212E4812
:10E9200000F0AFFC029D039B984515DA2B684FEA77
:10E93000880B002B44D09F4233D83B465AF80B201B
:10E940000021254800F09DFC5AF80B303B444AF862
:10E950000B302B68DF1B2F601E4B186800F072FC19
:10E9600000BF1E4B361B1B681C441C4B1C60019BCC
:10E97000A3B19EB1194B1B68DCB23219B2F5807F8E
:10E98000174A88BFC4F58074D26898BF3446934252
:10E99000A5D30023134A1370134A1370009B981BCE
:10E9A00092E7D9F8002000210B4800F06AFC2A68A1
:10E9B000D9F80030BF1A1344C9F8003000232B6087
:10E9C00008F10108043509F10409ACE7009ED0E71D
:10E9D000040700200007002000380040701D0020C0
:10E9E000780200206C1D00206D1D002030B50B4CFE
:10E9F0000B4D22782B7885B09A420CD002A968463C
:10EA0000FFF7DAFE0123022202A96846FFF746FF5C
:10EA100000232B70237005B030BD00BF6D1D00209A
:10EA20006C1D002030B50E4D0E4C2A78237885B031
:10EA30009A4212D002A96846FFF7BEFE00230222C6
:10EA400002A96846FFF72AFFFFF79EFE2878237881
:10EA5000C31A5842584105B030BD0120FBE700BF42
:10EA60006D1D00206C1D0020032373B58DF804304C
:10EA7000030C8DF805308DF80700030A06200E46BA
:10EA800014468DF80630FFF7FBFEC0B100BF0D4DF8
:10EA9000286800F0D2FB042300210DEB03020A4892
:10EAA00000F0EFFB234600223146074800F0E9FB67
:10EAB000286800F0C7FB00BF204602B070BD0446C6
:10EAC000FAE700BF000700200038004008B545F213
:10EAD0000820FFF7D5FE0620FFF7E6FC0122034BD6
:10EAE000C7201A70BDE80840DEE400BF040700201C
:10EAF00010F80A3C0133DBB20A2B00F80A3C07D9B4
:10EB0000002310F8131C034A22F8113000F80A3CC5
:10EB1000704700BF0C17002070B51424454B1A78BD
:10EB20000132B2FBF4F004FB102298681A705A6CA0
:10EB30008142DC680A4404D293F84C0008B102F523
:10EB400080323D480678B2FBF6F2944223D293F825
:10EB50004C501DB14FF4803595FBF6F5101B451B4D
:10EB60001D61DA6040F68C2200209960196983F8F3
:10EB70004C00914241D9187993F94920904230D103
:10EB8000021F082A2DD893F84A20182A0BD80132E0
:10EB900083F84A2009E04FF4803090FBF6F0001B28
:10EBA00010441861DDE783F8480093F9482090424B
:10EBB0000FD193F84B1061B10021204C204D9142B0
:10EBC00011DB00241E490B2A13DD1E490A7801328D
:10EBD0000A70012283F84B20002283F849001A7141
:10EBE00070BD0022D4E754F8046F25F8116001319C
:10EBF000E5E721F812400132E5E793F84B20C2B176
:10EC000040F2DA52A1F2EF20904207D81A790B2A8B
:10EC100004D803EB820041610132E0E7002283F86F
:10EC20004B20114613460848C2180433302B11619B
:10EC3000FAD170BD142000204C03002024200020B5
:10EC40000C170020041700201820002010B51424F1
:10EC5000094B1A780132B2FBF4F004FB10221A704F
:10EC60005A6C01320A445A644FF6FF72914204BF53
:10EC7000012283F84C2010BD14200020704714237B
:10EC80005843024B1B581980704700BF441C00209A
:10EC900014235843074A10B514181358A1F57A7273
:10ECA000618951434FF47A7291FBF2F189B2198074
:10ECB00010BD00BF441C002070472DE9F04714250B
:10ECC00050264FF028084FF00009144C144F05FB54
:10ECD0000045A54201D1BDE8F087237ACBB1D4F835
:10ECE00004A05046FBF7CEFBEFF3128386F31288A5
:10ECF000BAF8242008FB007092B201324262BAF8DE
:10ED00001420DBB292B242F00102AAF8142083F37D
:10ED1000118854F8143BA3F80090DAE7441C002053
:10ED2000D81A002014235843084B10B51C58A1F5DD
:10ED30007A7005F0C3F8064905F014F9054905F0A5
:10ED400009F807F093FE80B2208010BD441C00201B
:10ED5000EC51B83F0000B44314235843074B10B59F
:10ED60001C581820484305F0A9F8054905F0FAF8A1
:10ED700007F07CFE80B2208010BD00BF441C002044
:10ED8000ABAA2A3D14235843074B10B51C58C800A2
:10ED900005F094F84FF0785105F0E4F807F066FEBE
:10EDA00080B2208010BD00BF441C00202DE9F0413E
:10EDB00001270C4DDFF830802C686A6914400CB9CB
:10EDC000BDE8F081B4FA84F3C3F11F0307FA03F638
:10EDD00008EB8303186D24EA0604036898476E6104
:10EDE000EDE700BF000401401420002003681B6809
:10EDF000184703682DE9F041DB6905460E461746C2
:10EE00008BB90C463B1B3344002B01DCBDE8F08181
:10EE1000284602F0D0FE0028FAD014F8011B28463C
:10EE2000FFF7E4FFEEE7BDE8F04118471FB5012307
:10EE3000ADF808300023ADF80C30ADF80A30094BBE
:10EE4000ADF8041093F8903001A9012B08BF0323FB
:10EE5000ADF8062008BFADF80C30F8F72AFB05B076
:10EE60005DF804FB1420002038B510F80E2C044681
:10EE700050F8043C52B9012220F80C1C00F80E2C6A
:10EE8000597918680222BDE83840CFE7002530F8EC
:10EE90000C2C20F80A1C891A89B220F8081C074A91
:10EEA00010F80F0C22F8101004F80E5C2A4659795D
:10EEB0001868FFF7BBFF04F8065C38BD0C1700208C
:10EEC000072807D81422044B02FB0030D0F89430F6
:10EED00003B11980704700BF142000202DE9F84FBE
:10EEE0000F460546194638681E46BDF82840FBF710
:10EEF0003BFA97F807A03A681AF0040197F805E082
:10EF00000AF0020A1ED00020BAF1000F14BF4FF021
:10EF100000094FF0080982464FF0040C8346BEF109
:10EF20000C0F00F21A81DFE81EF01400180118011E
:10EF300018017300180118011801AD00180118011B
:10EF40001801E7004FF4807089468C464FF0010BA2
:10EF5000E5E7138C914923F001031B041B0C138478
:10EF6000138CB2F80480178B23F0020327F0730789
:10EF70003F041B043F0C1B0C4BEA0A0A8A421FFA8F
:10EF800088F847F0600743EA0A030FD001F50061F3
:10EF90008A420BD001F540618A4207D001F58061B9
:10EFA0008A4203D001F580618A420AD14FF6F3719B
:10EFB000194041EA090128F4407841EA0C0348EA83
:10EFC0000008A2F80480178394861384138B23F01F
:10EFD00008031B041B0C43F008031383B2F84430EE
:10EFE00011466FEA43436FEA53439BB2A2F84430A1
:10EFF00013889BB243F0010321F8343B01EB0E036D
:10F000002B6000236E816A6021F80E30BDE8F88F16
:10F01000138C624923F010031B041B0C1384138C04
:10F02000B2F80480178B23F0200327F4E6473F044F
:10F030001B043F0C1B0C4AEA0B0A8A421FFA88F891
:10F0400047F4C04743EA0A1303D001F500618A423E
:10F050000BD123F0800343EA091323F0400328F483
:10F06000406843EA0C1348EA8008A2F8048017833A
:10F0700014871384138B23F400631B041B0C43F4C9
:10F080000063AAE7138C4AEA0B0A23F480731B047B
:10F090001B0C1384B2F820809788938B28F400719E
:10F0A00023F07303DFF8F4801B0409041B0C090C24
:10F0B0004245BFB243F0600341EA0A2103D008F59C
:10F0C000006842450BD121F4006141EA092121F495
:10F0D000806127F4405741EA0C2147EA00179780E6
:10F0E000938394871184938B23F008031B041B0CD8
:10F0F00043F00803938371E7138CDFF8A0C023F477
:10F1000080531B041B0C1384138C9788918B23F45E
:10F11000005321F4E64109041B04090C1B0C4AEAC4
:10F120000B0A6245BFB241F4C04143EA0A3303D03F
:10F130000CF5006C624503D127F4804747EA80173D
:10F1400097809183A2F840401384938B23F400634B
:10F150001B041B0C43F40063CCE7BEF10C0F3FF61D
:10F160003DAF01A353F82EF0CDEF0008DDEF00080E
:10F17000DDEF0008DDEF000875F00008DDEF0008A6
:10F18000DDEF0008DDEF0008E7F00008DDEF000824
:10F19000DDEF0008DDEF00084BF10008002C014016
:10F1A00038B50409013C022C00F00F0214DC0B4DB1
:10F1B00035F8141041FA02F313F001000DD00120CC
:10F1C00090400138084005F0EFF82C44A37903443F
:10F1D000034800EBC30038BD002038BD98A20108E9
:10F1E000801D002037B50D460446C8B103680D4A9E
:10F1F00003F14043A3F5843302EB9323587A01F0E3
:10F20000D9FFA38801A9ADF80430206805F00303F5
:10F2100005F07C058DF806308DF80750F8F784FA74
:10F2200003B030BD98A2010830B102688388D1686C
:10F230000B4218BF1B041361704710B1036882882A
:10F240005A61704710B1036882881A61704738B1FB
:10F25000002914BF00211021838802688B401361AC
:10F26000704730B1036882889B681A4214BF01203E
:10F27000002070479AE599E598E597E596E595E5CC
:10F2800094E5F8B584894FF6FF764FF47A740BB99C
:10F290000120F8BD92B1157801320789BF070FD55B
:10F2A0004FF47A74ADB285810589ED0712D5858951
:10F2B000ADB209B10D700131013BE8E7FF25ECE784
:10F2C000013CA4B2B442E8D1FBF714FA003018BFF5
:10F2D0000120F8BD013CA4B2B442E5D1F4E708B581
:10F2E00040F2E9330289920708D540F2E93389B246
:10F2F00081810289D20709D5808905E0013B9BB253
:10F30000002BEFD1FBF7F6F9C0B208BD013B9BB271
:10F31000002BEED1F6E700BF022803D0431E58426F
:10F3200058417047064B1B681B7823B1054B186882
:10F33000C0F3C0407047044B1878C0F3800070479A
:10F34000841B0020181C002028260020A0F17D032B
:10F35000012B70B504460D460A4E11D87D21306848
:10F36000FFF744FD84F020013068FFF73FFD35B121
:10F370002888204400EB102000F0FF00288070BD9A
:10F380000146F1E7C00C00205E2810B50146094C8B
:10F3900009D15D212068FFF729FD3E212068BDE8E5
:10F3A0001040FFF723BD5D292068F8D1FFF71EFD4F
:10F3B0003D21F3E7482100200846F7F77DB9034BCC
:10F3C0001979034B1868FFF711BD00BF48210020D1
:10F3D000400E002010B50446044B01461868FFF7A4
:10F3E00005FD034B1A7954401C7110BD400E0020DE
:10F3F0004821002010B50446C0B2FFF7EBFF200AF9
:10F40000BDE81040E6E7002238B50546084C094B38
:10F41000206824211A71FFF7E9FC20685421FFF7C6
:10F42000E5FC29462068BDE83840FFF7DFBC00BF97
:10F43000400E002048210020074B198107490A4649
:10F4400002F8010B4FF6F67083E80600012258819E
:10F45000034B1A70704700BF200D00202C0D0020B8
:10F460002C0E0020002373B502AD25F8023D0C469A
:10F470002946FFF76BFFA61D14F8010B2946FFF77D
:10F4800065FFB442F8D19DF806000021C043C0B228
:10F49000FFF75CFF02B070BD07B50B0A8DF80000E6
:10F4A0008DF802108DF80330000A0B0C090E8DF850
:10F4B00001008DF80510102069468DF80430FFF723
:10F4C000D1FF03B05DF804FB73B5094C0646206814
:10F4D0000D46FBF744FE002296F9000001920095CC
:10F4E0004FF496430821FBF74FFE206002B070BD39
:10F4F000A80C002010B5054C206802F05FFB00B995
:10F5000010BD206802F054FBF6E700BFA80C0020F5
:10F510000028114AB8BF404290FBF2F330B53C25B9
:10F520000E4C04FB030068430D4D90FBF2F22D6876
:10F530002D7B75B903EB830303EB830302EB83039A
:10F540000B804FF47A7304FB020292FBF3F24A80C1
:10F5500030BDC3EB0313F1E780969800806967FF25
:10F560005C0C002010B50446C0B2FFF70DFFC4F3D9
:10F570000720BDE8104007E7024B5E211868FFF73F
:10F5800035BC00BF4821002038B50546054C5E213A
:10F590002068FFF72BFC29462068BDE83840FFF7BC
:10F5A00025BC00BF48210020038813F0400004D090
:10F5B00013F4057F14BF012000207047674B73B51B
:10F5C0001A68674C6AB11046FFF7EEFF48B123781E
:10F5D0003BBB644B1B6823B3634A13600123237056
:10F5E0001FE0624B1878FFF797FE237805468342A9
:10F5F00017D0002874D0A2B15D4B92F902001B68AD
:10F6000000225B780421003318BF012301930223F9
:10F6100000934FF41653FBF7B7FD534B18600028C7
:10F62000DCD1544B544D1878FFF776FE2B78044606
:10F63000834213D000285AD0504B1B6873B100226C
:10F64000012493F9020008214FF49643019200949B
:10F65000FBF79AFD4A4B186000B12C70494B4A4D9C
:10F660001878FFF759FE2B78044683422E4623D0A4
:10F67000002842D0454B1A68F2B1454B19688B7887
:10F680004978002B0CBF0023082309B143F0010384
:10F6900092F90200019303230022009320214FF4EA
:10F6A0006143FBF771FD3B4B186028B101233A4AD7
:10F6B00033701370394B1B68394B3A4C1A682AB3B4
:10F6C0001046FFF771FF08B32378002B3CD1254B80
:10F6D0001B68002B38D0344A13600123237033E0B9
:10F6E000214E3068FBF73BFD3560257099E7244ECD
:10F6F0003068FBF734FD3460AFE7264E3068FBF727
:10F700002EFD254B34601C702C70D5E7274B1878E4
:10F71000FFF702FE23780546834215D0B0B19AB1B7
:10F72000937992F9020002210022002B08BF0223E4
:10F730008DE806001E4951F823301021FBF724FD07
:10F74000194B18600028C8D102B070BD164E306841
:10F75000FBF705FD35602570F6E700BFE8060020E1
:10F76000450C0020E006002048210020EC06002087
:10F770005C0C0020ED060020640C0020B80C00207A
:10F78000A80C0020F4060020BE0C0020F00600208B
:10F79000300E0020C00C0020C40C002008350020D2
:10F7A000F80600203C0E0020400E0020FC06002041
:10F7B0007CA5010838B5124B05461B6883421CDA4C
:10F7C000104B93F8C9441CB1012C0AD0022038BD5B
:10F7D0000D4B1B68186970B18542B4BF012002202F
:10F7E00038BD7F28F2DCFFF713F8C0F17F008542B7
:10F7F00001DDFFF717F9012038BD002038BD00BF3B
:10F80000880700201830002084070020074B93F859
:10F81000C934012B08D1064B1868064BDB689842A7
:10F8200034BF0020012070470020704718300020AE
:10F83000701D002078020020F8B500230646011F45
:10F84000083051F8042F02F120043F2C3BD802F17C
:10F8500008040F2C1CD80232032A02D9002B08BF3F
:10F8600001238842EDD1012B306813D0022B1FD029
:10F87000736800019B0000F0300003F00C030343A9
:10F88000B06800F003001843BDE8F840F6F714BF75
:10F890000223E6E700F00F0040F04000F6F70CFF0F
:10F8A000B068736800F00F0040EA0310C0B2EBE7E5
:10F8B00000F03F0040F08000F6F7FEFE3079F6F7EA
:10F8C000FBFE307AE0E706F10C073C46002554F8D1
:10F8D000043DAD0003F18002FF2A06D903F5004282
:10F8E000B2F5803F19D245F00105B442EFD165F081
:10F8F0003F00C0B2F6F7E0FE05F00303022B2078CC
:10F9000019D0032B1ED0012B11D00434F6F7D4FEEE
:10F91000A7424FEAA505EFD1F8BD03F50003B3F107
:10F92000807F34BF45F0020545F00305DDE7F6F7BB
:10F93000C3FE6078E9E7F6F7BFFE6078F6F7BCFE35
:10F94000A078E2E7F6F7B8FE6078F6F7B5FEA078A3
:10F95000F6F7B2FEE078D8E710B504467F2C04D85D
:10F96000E0B2BDE81040F6F7A7BE64F07F00C0B279
:10F97000F6F7A2FEE409F1E7C31783EA4000EBE7DC
:10F9800070B506460D460024AC4200DB70BD36F96A
:10F990001400FFF7F1FF0134F6E72DE9F047324B91
:10F9A00086B093F8C9340546012B08D004462F4F82
:10F9B000264616F8011B002951D1641B48E003F0CC
:10F9C00019FD0446074603A96846FEF7F5FE049AAA
:10F9D000039B0295134423443F2B059417D900231E
:10F9E000032203A96846FEF759FF039BA3BB049BB0
:10F9F00093BB1F4A13701F4A1370059B43B3049AAD
:10FA0000039B059F13443B447F2B21D8029DDFF8C5
:10FA10006090DFF864A099F800602946C6F180087C
:10FA2000B84528BFB8460AEB06004644F6B242463F
:10FA300009F0CDFA802E89F8006009D1A7EB0807FC
:10FA40003A4605EB0801504609F0C1FA89F8007002
:10FA5000204606B0BDE8F087FEF796FECFE738688F
:10FA6000FFF7C4F93446A3E71830002084070020CC
:10FA70006C1D00206D1D00204D2100200FB437B5F6
:10FA800006AC54F8045B4820F6F716FE2020F6F783
:10FA900013FE23462A4609490020019403F091F9F8
:10FAA00004460A20F6F708FE054A033413681B1BB8
:10FAB000136003B0BDE8304004B07047B9F30008EC
:10FAC000880700200FB407B504AB53F8042B054991
:10FAD0000020019303F075F903B05DF804EB04B066
:10FAE000704700BFB9F3000870B50024064E074DFB
:10FAF00056F8340002F076FD0134284602F072FD1B
:10FB0000202CF5D170BD00BFA8A2010809C10108D1
:10FB10000121FCF7D3BF0021FCF7D0BFF0B468B1DE
:10FB2000184BD3F8CC3413F400330BD0164B1B68AE
:10FB300013F0020306D0154B1B7813B9F0BCFBF78A
:10FB40005FBC0023124A0C2602F58075294606FB8D
:10FB500003F4675D874204D00133142BF7D1F0BC66
:10FB600070470C4B186828B1224492F80151427832
:10FB70009542F4D2214419600023074A1380074AB2
:10FB80001360ECE71830002000170020EC14002070
:10FB9000A8A201080C1C0020081C0020041C002046
:10FBA00038B5104D00242846214600F8014B70223C
:10FBB00009F032FA284621466C1C436F0B4493F936
:10FBC00002206AB11D680A190D519D880731958080
:10FBD0009B7970299371037803F101030370ECD1D1
:10FBE00038BD00BFD0210020094B9A6F0E2303FBC4
:10FBF0000020437AFF2B07D0064A12789A4203D995
:10FC0000054A32F913007047B0F90400704700BF8D
:10FC1000D021002028170020181800202DE9F74FC8
:10FC2000054600273D4CDFF810B1DFF81091461E65
:10FC300004F17C0A04F1880804F1940216F8010F1B
:10FC4000019204F03BF9594604F08CF94AF8270078
:10FC5000B07A04F033F9494604F084F948F82700F3
:10FC6000307D04F02BF92E4904F07CF9019A42F81A
:10FC700027000137032FE1D195F8410004F01EF968
:10FC8000284904F06FF9C4F8A00095F8400004F08A
:10FC900015F90146244804F019FAC4F8A400E879DB
:10FCA00004F00CF9214904F05DF9C4F8A800687C5F
:10FCB00004F004F91D4904F055F9C4F8AC00E87EDD
:10FCC00004F0F8F81A49C4F8B000D4F8B40004F00D
:10FCD00049F9A96C064604F045F93146C4F8BC0060
:10FCE000C4F8B800686C04F03DF9C4F8C00095F899
:10FCF000280004F0DFF80F4904F034F901464FF012
:10FD00007E5004F025F801464FF07E5004F0DEF9F5
:10FD1000C4F8C40003B0BDE8F08F00BFD0210020BC
:10FD200097AC0A3A0402013C0000C842CDCCCC3D5D
:10FD300000007A440AD7233CD730033D033F7A3E84
:10FD40002DE9F347664C0546D4F8B4104FF07C50CB
:10FD500004F0BCF904F008FBAE8C07460EB1B042CB
:10FD600014D2604BC4F8C830288C08B1874238D20E
:10FD70005C4BC4F81031688C10B1874280F09180E0
:10FD8000584BC4F8743302B0BDE8F087564BE98C89
:10FD90003046C4F8C83003F01BFA04F1D40A804698
:10FDA000C4F8CCA0304604F085F84FF00109434672
:10FDB000D4F80C21014604F1F0065046CDF800902D
:10FDC00003F07CF9A88CC4F8D06004F073F8CDF887
:10FDD000009001464346D4F80C21304603F06EF9FA
:10FDE000C2E7AB7F012B41D018D3022BC0D13F4ECD
:10FDF0003F4BB4F80C21C1B23046C4F81031C4F8FE
:10FE0000146103F03DF906F58070B4F80C2195F803
:10FE10002010C4F8180103F033F9ACE7354BC0B239
:10FE2000C4F8103104F04AF80146334804F04EF9A2
:10FE3000D4F8B46080460146304603F08BFF01469B
:10FE4000304604F043F92D4BC4F82481C4F8143132
:10FE50001033C4F82861C4F82001C4F81831C4F87C
:10FE60003481C4F83861C4F8300184E71E4B244E55
:10FE7000C4F81031C4F8146104F01CF8D4F80C2153
:10FE8000014630461C3603F097F9C4F81861288CF7
:10FE900004F010F8D4F80C210146304603F08CF938
:10FEA00069E7144BC0B2C4F87433164BD4F8B4509D
:10FEB000C4F8783304F002F801460F4804F006F95C
:10FEC000C4F888530146C4F88403284603F042FF6F
:10FED0000146284604F0FAF8C4F8800353E700BF4F
:10FEE000D0210020BF2D0108492D01084423002006
:10FEF000E52C0108A12D010883F9223EEC22002007
:10FF00000C2300204C2500200D4B2DE9F0411B78DF
:10FF10000C4D3BB100240C4F05F5657695F88C33FC
:10FF20009C4206DBD5F8903395F88C03BDE8F04190
:10FF3000184736F81410E0B23B6898470134EDE7F3
:10FF4000121C0020D0210020141C00202DE9F74FA6
:10FF50004C4B4D4CD3F80090D4F8AC53494628464E
:10FF600004F000F8D4F8B07380464946384603F0F0
:10FF7000F9FFD4F8B46300904946304603F0F2FF2D
:10FF800039468246284603F0EDFF3146834628462F
:10FF900003F0E8FF31468146384603F0E3FF394677
:10FFA0000190384603F0DEFF014603F0D3FE3146F0
:10FFB0000746304603F0D6FF014603F0CBFE064667
:10FFC0000146384603F0C6FE01464FF07E5003F06E
:10FFD000BFFE5146C4F8B803584603F0B9FE0146C7
:10FFE00003F0B8FE4946C4F8BC03009803F0B2FE23
:10FFF000014603F0AFFE5946C4F8C003504603F073
:020000040801F1
:10000000A9FE014603F0A6FE2946C4F8C40328460B
:1000100003F0A8FF014603F09DFE00F100453146C4
:10002000284603F095FE4FF07E5103F093FE4146C3
:10003000C4F8C803019803F08BFE014603F08AFE62
:100040000099C4F8CC03484603F082FE014603F051
:1000500081FE0199C4F8D003404603F07BFE0146BF
:1000600003F078FE3946C4F8D403284603F070FE46
:100070004FF07E5103F06EFEC4F8D80303B0BDE824
:10008000F08F00BF50030020D02100202DE9F04F59
:10009000B54C89B0D4F8DC339A0740F1078494F862
:1000A0001C24002A00F00284D4F82024D4F8107410
:1000B000821A059207FB07F2D4F81464D4F81814D6
:1000C00006FB0622069101FB012164224A43B4F893
:1000D000E81313F0080801FB01F192FBF1F2A2F121
:1000E0005202C4F82004079210D0D4F83034002B08
:1000F00000F0C683D4F83434002B00F0C183D4F868
:10010000383413F1000818BF4FF00108059803F0C8
:10011000D1FE964903F026FF954D01909549E86C74
:1001200003F020FF93490290286D03F01BFF9149D3
:100130000390686D03F016FF00250490B8F1000FDE
:1001400000F0A083D4F8300403F0B8FE8346D4F85E
:10015000340403F0B3FE8246D4F8380403F0AEFE54
:1001600051468046504603F0FDFE414681464046DA
:1001700003F0F8FE0146484603F0ECFD594681467F
:10018000584603F0EFFE0146484603F0E3FD7A4986
:10019000814604F0A3F8002800F07483484606F076
:1001A00025FF01464FF07E5003F090FF8146014647
:1001B000584603F0D7FE49468346504603F0D2FE28
:1001C00049468246404603F0CDFED4F8B813804637
:1001D000584603F0C7FED4F8BC138146504603F0DE
:1001E000C1FE0146484603F0B5FDD4F8C013814670
:1001F000404603F0B7FE0146484603F0ABFDD4F895
:10020000C4138146584603F0ADFED4F8C8138346A4
:10021000504603F0A7FE0146584603F09BFDD4F874
:10022000CC138246404603F09DFE0146504603F043
:1002300091FD49468046484603F094FE414681467A
:10024000404603F08FFE0146484603F083FD06F06A
:10025000CDFE0146404603F085FE00F1004AD4F889
:10026000D013504603F07EFED4F8D4138146504696
:1002700003F078FED4F8D8138046504603F072FE9F
:100280008246079B262B00F28B80384603F016FE31
:100290000746304603F012FE0646069803F00EFEAF
:1002A00031460446304603F05DFE21468346204633
:1002B00003F058FE0146584603F04CFD394683468C
:1002C000384603F04FFE0146584603F043FD2A49E5
:1002D000834604F003F8002862D0584606F086FEF4
:1002E00001464FF07E5003F0F1FE8346014638464A
:1002F00003F038FE59460746304603F033FE5946B0
:100300000646204603F02EFE174B8346D3F8D8232B
:1003100030461146D3F8D4430792069303F022FEE9
:10032000494603F017FD21468146584603F01AFE60
:100330000146484603F00CFD069B8146D3F8D033B6
:1003400058461946069303F00DFE414603F002FDA0
:10035000079A80461146384603F004FE014640469F
:1003600003F0F6FC214609E0D0210020BD37863598
:10037000F80F002035FA8E3C0AD7233C80463846D9
:1003800003F0F0FD514603F0E5FC069B04461946D8
:10039000304603F0E7FD0146204603F0D9FC8246D3
:1003A000AE4C0021D4F84064304603F097FF00289B
:1003B00000F06C820399084603F0D4FD04990546C9
:1003C000084603F0CFFD0146284603F0C3FC02991E
:1003D0000546084603F0C6FD0146284603F0BAFC70
:1003E0009F4903F05DFF08B33146019803F0BAFD61
:1003F0004946054603F0B6FDD4F84C1403F0AAFCB8
:100400004146C4F84C04284603F0ACFDD4F850141F
:1004100003F0A0FC5146C4F85004284603F0A2FDA6
:10042000D4F8541403F096FCC4F8540494F85834E7
:10043000D4F8440413F00403069340F02E82894B51
:100440001A6844F61F639A4200F22782864903F035
:1004500089FDD4F84C140546029803F07BFC29462C
:100460000646484603F07EFD0146304603F072FC26
:10047000D4F850148146039803F06CFC29460646D4
:10048000404603F06FFD0146304603F063FCD4F8AC
:1004900054140746049803F05DFC2946064650466E
:1004A00003F060FD0146304603F054FC4FF07C51F0
:1004B0008246019803F056FD4946064603F052FD78
:1004C00039460546304603F04DFD514680463046DC
:1004D00003F048FDD4F8AC93644B8246294609F1F9
:1004E0000040D3F800B0079303F03CFDD4F8B063AC
:1004F00002903146404603F035FD029A014610460F
:1005000003F026FCD4F8B47302903946504603F049
:1005100029FD029A0146104603F01AFC594603F0E1
:1005200019FC59460290284603F01CFD3146039001
:10053000504603F017FD039A0146104603F00AFCEB
:10054000494603F007FC39460390404603F00AFD94
:10055000039A0146104603F0FBFB594604904046BF
:1005600003F000FD39460390284603F0FBFC0146EA
:10057000039803F0EFFB314603F0ECFB4946039090
:10058000504603F0EFFC0146039803F0E1FB5946A7
:100590000390504603F0E6FC49468246404603F08D
:1005A000E1FC0146504603F0D5FB394603F0D2FB8F
:1005B00031460746284603F0D5FC0146384603F08D
:1005C000C7FB02990646084603F0CCFC049A054690
:1005D0001146104603F0C6FC0146284603F0BAFB5C
:1005E00003990546084603F0BDFC0146284603F082
:1005F000B1FB31460546304603F0B4FC01462846BF
:1006000003F0A8FB06F0F2FC01464FF07E5003F029
:100610005DFD05460146029803F0A4FC049A079B81
:1006200029461860104603F09DFC2946C4F8AC0327
:10063000039803F097FC2946C4F8B003304603F052
:1006400091FCC4F8B403FFF781FCD4F8D863D4F864
:10065000D4833146404606F0D1FA09E0D02100208B
:10066000E68AF93D083500200000204150030020B3
:10067000924903F077FC06F0F9F9D4F8D093A4F886
:100680005A0409F1004006F069FA01468C4803F06B
:100690005FFB8A4903F066FC06F0E8F9D4F8C4333E
:1006A000D4F8B8A3A4F85C0451461846029306F0A7
:1006B000A5FA824900F1004003F054FC06F0D6F997
:1006C00003B2002B7F4FBABF00F56160A4F85E044F
:1006D000A4F85E34D7F86014304603F0FFFD97F8B5
:1006E0006424002800F0DC8042F0080287F86424CB
:1006F000D7F8100403F0E2FB0546D7F8140403F022
:10070000DDFB8346D7F8180403F0D8FBD7F8BC13F9
:100710000446584603F026FC51460390284603F051
:1007200021FC039A0146104603F014FBD7F8C013CE
:100730008246204603F016FC0146504603F00AFBB1
:1007400049468246284603F00DFC414681465846FC
:1007500003F008FC0146484603F0FCFA31468046A7
:10076000204603F0FFFB0146404603F0F3FAD7F8BA
:10077000C8130646584603F0F5FB02998046284602
:1007800003F0F0FB0146404603F0E4FAD7F8CC133F
:100790000546204603F0E6FB0146284603F0DAFA58
:1007A00097F8482400F10045012A464C7BD1069B6E
:1007B00073B94022D7F8680490FBF2F2801A03F074
:1007C0007DFB314603F0C6FA03F0A8FDC7F86804C4
:1007D0004023D4F8680490FBF3F003F06FFB01466C
:1007E000304603F0B5FAD4F870140746019803F0C8
:1007F000B1FA0146019803F069FCD4F86C648046B4
:100800003146384603F0A4FA0146404603F0AAFBFD
:10081000314603F09FFA0646C4F86C04504606F0D1
:1008200025F994F84A74394602F0B4FBD4F87434CC
:100830001844C4F87404284606F018F9394602F042
:10084000A9FBD4F878341844C4F87804304606F08C
:100850000DF994F84B1402F09DFBD4F87C34059A02
:100860001844D4F88034C4F87C041344C4F88034A9
:10087000D4F884340133C4F8843409B0BDE8F08F6F
:10088000984643E4AA46A846A946FAE4C4F84C545C
:10089000C4F85054C4F85454C8E54FF07E51D6E51E
:1008A00022F0080222E7B7F8E80396E70023C4F82D
:1008B0001034C4F81434C4F81834DEE74C3D0F4447
:1008C000DB0FC93FD0210020012310B50B4C4FF4A2
:1008D0008060E370022384F8203001F073FF64210C
:1008E000074B1A68074BD3F888345B7801FB032366
:1008F000636123880133238010BD00BF44180020AA
:1009000008350020D0210020426A806A131A58421C
:10091000584170474171704743799B070AD5436A34
:100920008269D154436A01690133B3FBF1F201FBDF
:10093000123343627047437913F0020308D003690E
:10094000426A806A013B101A1840C0B2181A7047F8
:1009500018467047437913F001031FBFC369026A49
:10096000C0689B1A1ABF00F1FF3018401846704744
:1009700010B54379014613F001030ED0FFF7EAFFEB
:1009800060B10B6A4A69CC68D05C0133B3FBF4F206
:1009900004FB1233C0B20B6210BD184610BD90F8B4
:1009A000433230B53BB9012490F8411290F84232FD
:1009B000DAB2914200D830BDB0F84A5204FA03F2DC
:1009C0002A43A0F84A220133F2E710B5046B03462C
:1009D000C168406944B11A6C8C1A013A08BF0A46D2
:1009E000005D1A64C0B210BD1A6A805C01328A428E
:1009F00028BF2246C0B21A6210BD436B13B190F8F3
:100A000044007047836A406A1B1A58425841704735
:100A1000416A836A0269994238BF8918CB1A416BCF
:100A200021B149680B44511E8B4202D2501EC01A9C
:100A3000704700207047036B4BB1026C5B689342B8
:100A4000A3EB02032EBF1846C068C0187047C269E6
:100A5000036A9A422FBFD01AC0688018C01A704724
:100A600038B5A0F517746379A579DB0744D594F8F8
:100A700040321BB3A06B0268938DC3F34E03938483
:100A800094F85132012B07D094F8453223B1B4F8D1
:100A90004C320133A4F84C32E94301F0010100F07B
:100AA00009FC012384F84332002384F8413284F89E
:100AB000423284F84032A4F84A3238BD94F84332C6
:100AC0002046012B04BF94F8413284F84232FFF7EC
:100AD00066FF94F843324BB90123E94384F843326B
:100AE0001940A06BBDE8384000F0E4BB002305F0DE
:100AF000010184F84332F4E738BD10B58379044628
:100B0000DB074CBF2A214A21006BFEF76BFB00225A
:100B1000012384F84122A26B84F8443284F84032E5
:100B20001168527993400A8C9BB292B222EA030276
:100B30000A840A8C92B213430B8410BD0A4B10B482
:100B40001A681346B3FBF1F4B4F5803F03D3012BCD
:100B5000FAD95B08F6E7054BA1B2B2FBF3F210BC81
:100B6000D2B2F9F755BC00BF7402002040420F001A
:100B70008160806BE2E78379406BDB0744BFB1FAA9
:100B800081F1490909B1FEF75DBBFEF756BB10B50F
:100B9000A0F5157463799A0714D594F84522002AB4
:100BA00059D1A36A616A994221D194F844324BB970
:100BB000A3791B0706D5606B0621FEF713FB2046C1
:100BC000FFF79BFF6379D90740F1978094F8403293
:100BD000002B40F0928094F841320133DBB2092BB4
:100BE00084F841324DD12046BDE81040D7E6591C6B
:100BF000A069A162C35C2069DBB25B0043F40073AF
:100C0000A4F848320A2381424FF0010184F84632A9
:100C100094F8443228BFA26284F84512002BD1D048
:100C2000A3791807CED5A06B02684079138C814058
:100C30009BB223EA01031384138C206B9BB21384B1
:100C40000621FEF7CFFA0023122184F84432606BAC
:100C5000FEF7C8FAB6E794F946327BB1B4F8481209
:100C600020464B08A4F8483201F00101FFF783FF4A
:100C700094F84632013B84F84632A3E784F84532C3
:100C8000A0E70A2B39D194F843322BB9B4F84A3291
:100C900043F00103A4F84A32B4F84A02820501D4B1
:100CA000C30718D4B4F84E320133A4F84E320122EF
:100CB000002384F8402294F8432284F84132012A28
:100CC0001BD1A17984F84332A06B01F00101BDE88A
:100CD000104000F0EFBAE36AC0F347000BB1984749
:100CE000E5E7E3696269D054E369E1680133B3FB86
:100CF000F1F201FB1233E361D9E710BD417100F05D
:100D000043BD816000F040BDEFF31283102282F3F7
:100D100012880649DBB20A6801320A600021044ADF
:100D20001160044A126883F3118870470835002067
:100D3000781B002010E000E0044B014618681B7986
:100D40000BB981F00101FEF782BA00BF5C260020DA
:100D50002DE9F04F4FF4187489B098469DF848304B
:100D600004910293794B4443034493F8CC12054613
:100D7000084693F8C0B20192039100F0B4FA0790CC
:100D8000584600F0B0FA0399814608460691FEF7EE
:100D900007FA05905846FEF703FA6D4E029B06F1DE
:100DA000080713F00803039307EB040A059B069951
:100DB000079A00F09580B9F1000F03D1002009B027
:100DC000BDE8F08F3319C3F84090D86398630B23C4
:100DD0008371EB18C3714FF418794FF0000B4FF487
:100DE000807209FB05695B4BC9F81420C9F808300B
:100DF000019BC9F81820C9F810309DF808300199F6
:100E000089F80E30049BD9F84000C9F8343004F159
:100E100040033B44C9F81C3004F5A0733B44C9F8B7
:100E2000203089F80D80C9F828B0C9F824B0C9F875
:100E300030B0C9F82CB089F85852A9F854B2A9F8C2
:100E400056B289F84CB289F84DB2FFF777FE029B93
:100E5000D9F8400003F0010100F02CFA3E4A04F5F5
:100E60001773C9F864223D4A04F5157418F0020F8F
:100E70003B44C9F85C222744C9F860B25BD0D9F87A
:100E80004400002857D0D9F84010026809688A4207
:100E900051D00122019989F859220293FFF74EFEA1
:100EA0003A465946D9F84400F9F708FB029B5A46DE
:100EB0001946D9F84000F9F701FB039B5BB94FF4E1
:100EC000187303FB05651221E86BFEF78BF901210E
:100ED0005046FFF750FE5046FFF70FFE50466EE7B4
:100EE00018F0010E0DD000293FF468AF002A3FF43E
:100EF00065AF31190A640C228B639A7105F10B02FC
:100F0000DA7118F0020F3FF466AFBBF1000F3FF447
:100F100055AF4FF4187303FB0563D863BEF1000FA0
:100F200006D1B9F1000F3FF449AFC3F840904EE746
:100F3000C3F844904BE74FF41870002200FB0560A3
:100F4000194680F859223A46006CB4E72230002056
:100F50005C260020F4A40108610A01088F0B010837
:100F6000836A8169426B1944D160416A8B4229BF0F
:100F70000169CB1ACB1A53602ABF002353608362E6
:100F80004FF0000380F84430136838BF816243F0AB
:100F9000010313607047436A8269D154436A02694E
:100FA0000133934228BF00234362436B1BB11B688C
:100FB000DB0705D4D4E7026DD36843F08003D36028
:100FC000704700BFFF207047012380F8453070470D
:100FD000014B1868704700BF242B00200120704788
:100FE0007047704720B90822024B5B681A8270472D
:100FF00001487047242B00205403002010B50446FC
:1010000001F08BF92379134A03F00F03052B1FD846
:10101000DFE803F003090D101E140378805C1B1A2F
:101020005842584110BD90F900308056F7E70388C8
:10103000805AF4E7B0F90030805EF0E7815800682C
:101040004FF0010403F022F900B90446E0B210BDEC
:10105000002010BD14FBFFFFF8B5002390F844609A
:1010600080F844300EB3144DD5F8E029FAB1D5F824
:10107000E029052A1DD1D5F8E47900F13004D5F82E
:10108000E83983B931462046FCF705F9D5F8E4394B
:10109000361ADB1B322B044401D8002EEFD1B6FAEE
:1010A00086F04009F8BD0020F0E70120F8BD1046A9
:1010B000F8BD1846F8BD00BF242B0020002280F8A0
:1010C0004520C9E790F84420531CDBB2024480F865
:1010D000443082F8301090F845200AB1132B00D923
:1010E000BAE77047F8B50F4C1646D4F8E039B3B1FB
:1010F000D4F8E039052B12D10D46D4F8E479002E4E
:101100000DDDD4F8E8395BB931462846FCF7C3F861
:10111000D4F8E439361ADB1B322B0544EFD9F8BD7D
:101120000020F5E7242B00202DE9F3411F4E204F2E
:101130003446336873BB3568002294F8EC196018A4
:10114000D3B29D4202F1010226D8236829445B1BD9
:101150002360D4F8008084F8EC19B8F1000F12D1A4
:1011600040210320F6F780F83B6823F4804323F006
:1011700070039BB283F4405343F4004343F0800375
:101180003B6084F8EC89002DD3D09DF8040002B0B8
:10119000BDE8F0810125CFE70DF1080E9E44034420
:1011A00093F8ED390EF8043CCAE700BF242B002069
:1011B0000C5C0040012300F01F024009022803FAE2
:1011C00002F308D003280BD001280DD1074A51693A
:1011D0000B4353617047054A91690B439361704714
:1011E000024AD1690B43D361704700BF001002402F
:1011F000064B93F82D1AD3F8303A20B101F00101D3
:101200001846FEF724B8C943F8E700BF242B002096
:101210000168154BCA4310B51C6814401C605C681B
:1012200022405A60027902F1804202F5823214684B
:101230002143116002689C68D1430C409C60DC68CB
:101240002140D9604179102906D1996811439960EC
:10125000D9680A43DA6010BD01F1804303F5823397
:1012600019680A431A6010BD0004014010B5044615
:101270000068FEF781FB6068FEF77EFBA068BDE8B2
:101280001040FEF779BB10B5094B03F1500293F8FB
:101290001D14814205D193F81F4493F820148C4209
:1012A00004D304339342F2D1002010BD012010BDBD
:1012B000183000201FB50123ADF808300023ADF829
:1012C0000A30ADF80C3043790029ADF8043014BF72
:1012D0000023022301A90068ADF80630F6F7E9F80B
:1012E00005B05DF804FB10B560B10022064901EBC2
:1012F000C2031C79844204D001320C2AF7D10020A9
:1013000010BD184610BD00BF1CA50108F0B5002493
:101310004FF00C0E164B93F83C2AD3F8401A03F604
:10132000442701EBC201042A04D90CB183F83C2AFA
:101330000020F0BD0132D2B281B10C88E5070DD595
:1013400020420BD0002491F902600EFB04F515F940
:1013500007C0B44505D00134052CF6D1083101246D
:10136000E1E783F83C2A2B44D3F8480AF0BD00BFDC
:10137000242B00200022024B83F83C2AC6E700BF42
:10138000242B002008B50020FEF724F80020FEF7EB
:1013900021F80020FEF71EF8BDE808400020FEF707
:1013A00019B8031EB8BF2D2210B5B8BF58420C465D
:1013B000AEBF0A2201F8012B0A22F9F7F1FD002342
:1013C0000370204610BD2DE9F04F0D46002793B065
:1013D0003C4E08900991D6F80C800021404602F05E
:1013E00055FF0446002869D1336904937369059356
:1013F000B3690693099B002B3DD0D5F800B0EB688C
:1014000059464046D5F804A0D5F80890079302F055
:101410003DFF80B15146049802F038FF58B149466B
:10142000059802F033FF30B10799069802F02EFFBD
:10143000041C18BF01240AA95846F9F74DFD0CA950
:1014400083465046F9F748FD0EA982464846F9F70B
:1014500043FD10A981460798F9F73EFDCDF80890A5
:101460000390CDF804A0CDF800B03B46164A2146C3
:10147000089801F00BF80AA94046F9F72DFD0CA9D0
:1014800004460498F9F728FD0EA980460598F9F757
:1014900023FD10A981460698F9F71EFD3B460390EF
:1014A0008DE81003084A00210898013701F00EF872
:1014B0000C2F06F1100605F110058CD113B0BDE814
:1014C000F08F00BF18300020E7C501082DE9F04F6C
:1014D000814688460E463F4C89B001F128033E4FB5
:1014E000DFF8F8A0079304F5AA6B002394F9DA2239
:1014F00013F90B10914267D00C333C2BF8D1079BAA
:1015000008369E4204F10804EFD109B0BDE8F08F1F
:1015100096F9023031889A42727953D1B4F8D802E0
:1015200088424FD194F8DB52F07885424AD194F842
:10153000DC523079854245D194F8DE52B07985424B
:1015400040D194F8DD52A81A4542454107EB82028A
:10155000126E48460492B27907EB8202126E039231
:10156000327907EB8202126E0292F27807EB820266
:10157000126E8DE806005246294600F087FF94F867
:10158000DD2294F9DA3207EB8202126E29460492C8
:1015900094F8DE22484607EB8202126E039294F81A
:1015A000DC2207EB8202126E029294F8DB2207EB38
:1015B0008202126E0192B4F8D8220092524600F0D4
:1015C00085FF9CE70025C1E7B8F1000FA0D1454693
:1015D000D5E700BF183000201CA50108FDC5010893
:1015E0002DE9F84380460E460025DFF878901A4F23
:1015F0007C19237903F03003434527D12046FFF7B8
:10160000FDFCEF5901463B46144A304600F03EFFD0
:1016100058B1204600F081FE002200EB090120466F
:1016200000F0B4FE0E4800F0DDFF2046FFF7E6FCB8
:101630003B460146094A304600F048FF30B120469B
:10164000002100F007FF064800F0CCFF1035B5F58B
:10165000276FCCD1BDE8F883BCA501081CC60108E2
:1016600009C1010814FBFFFF012810B50C4610D872
:10167000F8F790FA0748FAF7FDFC074800F0B2FFC8
:1016800021461020FFF7ACFFBDE810400148FAF7F3
:10169000D5BC10BD58C4010809C10108022810B505
:1016A0000C460CD8F8F758FA0548FAF7C7FC054875
:1016B00000F098FF2146BDE81040202090E710BDC3
:1016C00058C4010809C10108F8B51D250F461F4C73
:1016D000064684F8805A00F063FC002000F0FAFB14
:1016E000082000F0F7FB0E2000F0F4FB284600F085
:1016F000F1FB042000F0EEFB042000F0EBFB0020E7
:1017000000F0E8FB302000F0E5FB002000F0E2FBF9
:10171000384600F0DFFB002000F0DCFB00F024FC8A
:1017200004F6812000F040FB234670B194F8812A32
:1017300052B994F8822A302A00D02AB993F8832A21
:1017400012B993F8843A33700120F8BD242B00209D
:101750004FF6FB7210B5094C21680A402260084A16
:1017600092F89E1A41B10523C2F8E039F6F72EF837
:101770004FF41643236010BD0123F5E7405C0040A1
:10178000242B0020FDF735BBF0B50446056D8668B7
:10179000AB8987B023F400531B041B0CAB81837906
:1017A00013F004010CBF00274FF4805713F0020F11
:1017B00014BF4FF4005200220029617914BF4FF486
:1017C0008060002011F0010F14BF0423002389075B
:1017D000298A48BF43F0080389B221F440511143DC
:1017E0002982AA8922F4B05222F00C021204120CAF
:1017F0003A4302431343AB81AA8A01A822F4407200
:101800001204120CAA82F5F7F9FD284A039B0499E9
:10181000954218BF19461922AB894A4313F4004F69
:1018200014BF7100B100B2FBF1F16426B1FBF6F315
:10183000AA891801120406FB13132CD5DA003232E0
:10184000B2FBF6F202F0070242EA00039BB22B81E0
:10185000A379DB0709D5226D144B9A4223D12220AC
:10186000FDF79EFC0121FDF7F2FCA379226D13F038
:10187000080F938A0BBF23F008039BB21B0443F0AD
:10188000080308BF1B0C938293899BB243F4005357
:10189000938107B0F0BD1B013233B3FBF6F303F0C5
:1018A0000F030343D2E70020DCE700BF003801400C
:1018B0002DE9F0431D46AC4B8DB098428846174643
:1018C0009DF8506040F0EB80A84CA94B2065236048
:1018D00004F1A803636104F5D473A3614FF480732A
:1018E000E3602361A34B4E206363A3F54843403B71
:1018F000A260A364FFF75EFC310740F1B8801920B5
:10190000FDF74EFC0B2216F0100F82714FF0010212
:1019100014BF1A211E21C271FDF764FC964B974A31
:10192000596E50694FF00109084350610B2083F84C
:101930006D9083F86C005069014351619C660024EE
:101940008F4A01A8DA6593F861308DF806408DF86A
:1019500004308DF805908DF80790F5F7C1FE25232A
:1019600001A88DF806408DF804308DF805908DF8AB
:101970000790F5F7B5FE7D4C4FF000090123C4F840
:10198000209084F84430C4F81C90C4F82890C4F81F
:101990002490C4F82C806571A760A6712046FFF7DB
:1019A000F3FEEA072ED5206B002800F0CB80E36C15
:1019B000CDF80C9001934FF480530A938023069343
:1019C000E368CDF814900493202309936369CDF85C
:1019D0001C900293CDF82090CDF82C90F5F794FC54
:1019E00001A9206BF5F772FC226B216D136843F09F
:1019F000010313608B8A9BB243F040038B825368D0
:101A00009BB22364AB0728D5606B002800F0A3804D
:101A1000A36C002501934FF480530A93802306930F
:101A20002369029504931023059503930795089560
:101A300009950B95F5F768FC01A9606BF5F746FC75
:101A4000636B1A6842F002021A60226D5D605D608D
:101A5000938A9BB243F0800393822046226D938940
:101A60009BB243F4005393810DB0BDE8F083AA0705
:101A700009D51920FDF794FB0B22827101221A214E
:101A8000C271FDF7AFFBEB077FF548AF1A20FDF7FA
:101A900087FB0C22827101224A21C2713CE7394B3B
:101AA00098425ED1314B324AC3F8A4005A6503F51F
:101AB0002A729A6603F56A72DA664FF480721A66C1
:101AC0005A66314A7220DF65C3F89C20C3F8A02013
:101AD000FFF770FB34071ED52A20FDF761FB0B22B0
:101AE00016F0100F82714FF0030214BF1A211E214D
:101AF000C271FDF777FB272300228DF80430012304
:101B000001A88DF805308DF806208DF807301F4CA0
:101B1000F5F7E6FD30E7A80709D52A20FDF740FBD9
:101B20000B22827103221A21C271FDF75BFBE907C8
:101B3000E1D52B20FDF734FB0C22827103224A21D0
:101B4000C271D6E74FF6DF72236D1A80DA6842F071
:101B50002002DA6056E7226DD36843F08003D36039
:101B60007BE7002080E700BF00380140D43500202B
:101B70002CB00108440002408802002000100240FE
:101B8000DD5300080048004004480040283600208B
:101B900003685B6A03B11847704703681B6A03B1A7
:101BA0001847704703689B69184703685B691847C3
:101BB0000368DB68184703689B68184703685B681D
:101BC000184700BF30B508224AF2010409490B88C2
:101BD00080EA030515F0010F4FEA530302F1FF32CB
:101BE00014BF63409BB212F0FF024FEA5000EFD1E6
:101BF0000B8030BD7C3A0020F8B5F8F7B3FC244EDA
